:020000040800F2
:1080000028EE0020A1810008A981000889AB0008A2
:10801000AD810008AF810008B181000800000000B8
:10802000000000000000000000000000B381000814
:10803000B581000800000000B7810008B981000880
:10804000BB810008BB810008BB810008BB81000820
:10805000BB810008BB810008199E0008299E00080A
:10806000BB810008BB810008BB810008BB81000800
:10807000BB810008BB810008AB990008B3990008D8
:10808000BB810008BB990008BB810008BB810008C8
:10809000BB810008BB810008BB810008BB810008D0
:1080A000BB810008BB810008BB810008BB810008C0
:1080B00001450308BB810008BB810008BB810008A3
:1080C000BB810008BB810008BB810008BB810008A0
:1080D000BB810008235403082B54030833540308BE
:1080E000219E0008BB810008BB810008BB810008FD
:1080F000BB810008BB810008BB810008C399000850
:10810000BB810008BB810008BB810008BB8100085F
:10811000135403081B540308BB810008BB810008EB
:10812000BB810008BB810008BB810008BB8100083F
:10813000BB810008BB810008BB810008BB8100082F
:10814000BB810008BB810008BB810008BB8100081F
:10815000BB810008CB990008D39900083B54030861
:10816000BB810008BB810008BB810008BB810008FF
:10817000BB810008BB810008BB810008BB810008EF
:10818000BB810008BB810008DFF810D000F058FC6C
:108190000048004781720308AFF3008028EE0020FA
:1081A0000648804706480047FEE7FEE7FEE7FEE791
:1081B000FEE7FEE7FEE7FEE7FEE7FEE79944030879
:1081C000898100082DE9F0410024061B254671F144
:1081D000000605DA01240027D0EB070067EB010158
:1081E000161E73F1000605DA0027D2EB07020125FF
:1081F00067EB030300F0C1FA86460E4617469C461D
:10820000AC4204D00025D0EB050E65EB010624B18D
:108210000020D2EB000760EB030C704631463A4673
:108220006346BDE8F081202A06DBCB17203A41FAED
:1082300002F043EAE07306E041FA02F3D040C2F1F3
:108240002002914008431946704740EA01039B070A
:1082500003D009E008C9121F08C0042AFAD203E0BB
:1082600011F8013B00F8013B521EF9D27047421E43
:1082700012F8013F002BFBD111F8013B02F8013B42
:10828000002BF9D17047421C10F8011B0029FBD1CB
:10829000801A704730B505460020034600E05B1C9D
:1082A000934205D2EC5CC85C201A01D1002CF6D1B7
:1082B00030BD2DE9FE4F804681EA0300C00F0C4619
:1082C000009021F0004123F00045B8EB0200A941E5
:1082D00005D24046214690461C460B46024623F0F6
:1082E0000040104347D0270DC7F30A00C3F30A51DB
:1082F0000290401A019040286BDAC3F3130040F457
:10830000801B0098924620B10023D2EB030A63EB56
:108310000B0B01985946C0F14002504600F05EFA3E
:1083200006460D4650465946019AFFF77CFF10EB72
:1083300008006141002487EA115284EAE7731A4376
:1083400040D0009A62B3019A012A4FEA075215DC25
:10835000001B61EB02014FF0004202EA0752CDE937
:108360000042001C41F5801132462B4600F0EAFA2B
:1083700003B0BDE8F08F40462146F9E7001B61EBF2
:108380000201001C41F5801300185B412018A2F582
:10839000001747EB030140EAD570B6196D4111E0B3
:1083A0006D084FEA360645EAC0754FEA0752001BD2
:1083B00061EB0201001C41F5801149084FEA3000D1
:1083C0000019514132462B4603B0BDE8F04F00F092
:1083D000AABA0098012240000023D0EB020263EB0E
:1083E000E073009821464FEAE074B8EB000061EBBF
:1083F0000401E9E783F000435BE781F0004158E7BF
:108400002DE9FE4F81EA030404F0004421F000410D
:1084100000944FF0000B23F0004350EA01045ED0BB
:1084200052EA03045BD0C3F30A54C1F30A552C4447
:10843000A4F2F3340194A0FB0254C1F3130141F4FC
:108440008011C3F3130343F4801301FB024400FBC8
:10845000034E840A970A44EA815447EA8357A4FBEF
:10846000076802958D0A05FB07854FEA932C04FBEC
:108470000C542705029D4FEA065847EA1637B5EB1C
:1084800008056EEB070C870E920E47EA811742EA49
:108490008312A7FB0201B6EB0B0164EB00042B0D6A
:1084A00043EA0C335E1844EB1C50DA465146E7FBB6
:1084B0000201C5F313044FEA0B3343EA14534FEAA6
:1084C0000432019C43EA0603A4F10C040294009CCC
:1084D000CDE900B400F036FA03B0BDE8F08F00201B
:1084E0000146F9E72DE9F04D81EA030404F0004B61
:1084F00021F0004514464FF0000A23F0004150EAF5
:10850000050220D054EA01021DD0C5F30A570246E5
:10851000C5F31303C1F31300C1F30A5640F48015E9
:1085200043F48013A7EB0608101BD64608F2FD386B
:1085300073EB050002D308F1010801E092185B41DA
:10854000B8F1000F03DA00200146BDE8F08D0020ED
:108550004FF48011064684460EE0171B73EB0507A7
:1085600005D3121B63EB050306434CEA010C4908D3
:108570004FEA300092185B4150EA0107EDD152EA10
:10858000030012D082EA040083EA0501084305D003
:10859000101BAB4106D20122002306E000224FF05F
:1085A000004302E06FF0010253101AEB06004CEB9F
:1085B000085110EB0A0041EB0B01BDE8F04D00F053
:1085C000B2B9F0B4CA17CB0F50405140C61841F1B0
:1085D00000054FEAC372314628004FF0960303D0DE
:1085E000B623F0BC00F071B930460021F9E70EB5B2
:1085F000C10F80EAE0700844CA07002140F233430B
:108600008DE80E000A460B4600F09CF903B000BD51
:108610000EB540F2334102910021CDE900110A4626
:108620000B4600F08FF903B000BD3EB5CA17CB0F63
:10863000002450405140C0186141DA0740F23343F2
:108640000094CDE901232246234600F07BF903B0D4
:1086500030BD10B500F0004420F00040C20DC0F362
:10866000160040F400007F2A02DA0020014610BD07
:108670000021962A03DCC2F19602D04002E0963A2D
:1086800000F0ACF8002CF2D00023D0EB030063EB39
:10869000010110BD70B5C1F30A5201F0004500247C
:1086A000C1F3130140F2FF3341F480119A4201DA21
:1086B000002070BD40F233439A42A2F2334203DC01
:1086C000524200F09AF800E090402C43F1D0404232
:1086D00070BD70B5C1F30A5201F000450024C1F32A
:1086E000130140F2FF3341F480119A4202DA002074
:1086F000014670BD40F233439A42A2F2334203DC9A
:10870000524200F07AF801E000F068F82C43F0D013
:108710000023D0EB030063EB010170BD00F00042C9
:1087200030F000400AD0C10D01F56071C0F31600B1
:1087300042EA0151C2084007114370470020014638
:10874000704701F0004330B421F0004150EA0102CB
:1087500006D00A0DA2F56072C1F31301002A02DCF3
:1087600030BC00207047440F44EAC104C100E01847
:1087700030BC00EBC25000F09FB82DE9F05F054619
:10878000002092469B4688460646814640241BE0D0
:10879000284641464746224600F02FF853465A469F
:1087A000C01A914110D311461846224600F016F81F
:1087B0002D1A67EB01084F4622460120002100F0E8
:1087C0000DF817EB00094E41201EA4F10104DFDC77
:1087D000484631462A464346BDE8F09F202A04DB3E
:1087E000203A00FA02F1002070479140C2F12003C4
:1087F00020FA03F3194390407047202A04DB203A03
:1088000021FA02F00021704721FA02F3D040C2F1B0
:108810002002914008431946704700000FB400231E
:1088200000B589B00CA900910B996FF00042CB60A4
:108830001E4B06931E4B07930423CDE901321D4ABC
:10884000089202466B46002000F0A6F909B05DF8D8
:1088500014FB70B586B006464FF0FF300091CDE9AD
:108860000101002015460C4604903246694604A8D2
:10887000FFF7D4FF02460498211825B108B1084635
:1088800000E020462860049800280DD0002A02DD70
:108890000098884208D0081B0094CDE901043246B4
:1088A000694604A8FFF7BAFF06B070BDD18D000875
:1088B000EF8D0008658A00080029A8BF7047401C9A
:1088C000490008BF20F00100704710B4B0FA80FCE6
:1088D00000FA0CF050EA010404BF10BC704749B123
:1088E000CCF1200421FA04F411FA0CF118BF012193
:1088F00021430843A3EB0C01CB1D4FEA00614FEA73
:10890000102042BF002010BC704700EBC350104441
:108910000029A4BF10BC7047401C490008BF20F0CC
:10892000010010BC704710B5141E73F1000408DA82
:10893000401C41F1000192185B411A4301D120F023
:10894000010010BD2DE9F04D92469B4611B1B1FAE0
:1089500081F202E0B0FA80F220329046FFF73EFF4B
:1089600004460F4640EA0A0041EA0B0153465A46C4
:10897000084313D0114653EA010019D0C8F1400250
:108980005046FFF73AFF05460E46504659464246C6
:10899000FFF724FF084305D0012004E020463946B4
:1089A000BDE8F08D0020054346EAE0762C433743CE
:1089B0000A986305E40AA0EB08000022FD0A44EAD5
:1089C00047540A3002D500200146E9E70105101995
:1089D0006941DDE9084500196941BDE8F04DA2E7AC
:1089E00070B521F0004303430CD0C1F30A550024B5
:1089F000D5EB040564EB0403D617AD1AB34102DBD3
:108A00000020014670BD201841EB025170BD0000EE
:108A100030B5041E71F1000404DB4FF00044404205
:108A200064EB0101141E73F1000405DB1C464FF0DA
:108A30000043524263EB0403994208BF904230BDA9
:108A4000064C074D06E0E06840F0010394E807009B
:108A500098471034AC42F6D3FFF79AFB78F8030836
:108A600098F80308C0B24FF4F05100F03BBA000090
:108A70002DE9FF4F087883B09946FF2805D0491C9F
:108A80002D2804D00024002008E000200BE0012461
:108A9000F9E700EB800003EB4000491C0B78FF2B4B
:108AA000F7D104B1404200230293147819461D46C1
:108AB0002D2C01D02B2C04D1521C2D2C13D0002492
:108AC0000294AA461478FF2C0FD00A25A3FB057840
:108AD00001FB05814FF0000C03FB0C11521CE31944
:108AE0004AEB0101EEE70124EAE7814453EA010081
:108AF00002D019F5C87F06DA03980021C0E90011F9
:108B000007B0BDE8F08F0025AE4E2F46DFF8B882E3
:108B1000184600F0FBF9CDE90001B9F1000002DAD6
:108B2000C9F1000400E004460023A74A1AEB030B36
:108B300042EB045A12E0E00707D02A463346384693
:108B40004146FFF75DFC074688462A4633461046F5
:108B50001946FFF755FC05460E466410002CEAD175
:108B6000DDE90001B9F1000F5A46534606DAFFF776
:108B7000B9FC3A464346FFF7B5FC05E0FFF740FC79
:108B80003A464346FFF73CFC029A0AB181F00041A5
:108B9000039AC2E90001B3E72DE9FF4F1F468DB0EC
:108BA000D7E901464FF0FF382E2045464FF0000927
:108BB0000B90B9696D1C0E988847396A82468847C0
:108BC0000028F6D1BAF1FF3F0AD024F4D064002E79
:108BD00011DDBAF12B0F08D0BAF12D0F0BD102E045
:108BE000404611B08DE744F48064B9696D1C0E985D
:108BF00088478246761E6946600501D52D2000E033
:108C00002B208DF8000001F1010B0DF1200809E087
:108C1000B9696D1C0E98884782460F9844F4007419
:108C2000761E0560002E02DDBAF1300FF0D00B99F0
:108C30008A453ED144F0800406E00F99681CA9F1F2
:108C4000010944F400740860B9696D1C761E0E9821
:108C5000884782463028F0D02BE00B998A4505D111
:108C6000200603D444F08004761E18E050462DF010
:108C700021FF08B30DF11301761E44F400748B45F7
:108C800008D2AAF130000BF8010B200607D5A9F194
:108C9000010003E0200602D409F101008146A0058D
:108CA00002D50F99681C0860B9696D1C0E98884739
:108CB0008246002ED1DC53E0002E51DDBAF1650F63
:108CC00002D0BAF1450F4BD1A00549D5B9696D1C49
:108CD00024F44074761E0E9888478246002E0CDDE0
:108CE0002B2804D0BAF12D0F07D144F48074B96950
:108CF0006D1C0E9888478246761EE00501D52D2111
:108D000000E02B2108F8011BCDF82C8021E00DF1AB
:108D10002901761E44F4007488450CD2AAF1300073
:108D200010F0FF0088F8000002D10B99884509D99E
:108D300008F1010806E0E00501D5244801E042F20F
:108D40000F708146B9696D1C0E98884782460F984E
:108D50000560002E04DD50462DF0ACFE0028D6D173
:108D6000F9690E988847FF208BF8000088F800000A
:108D70000020069007904B466A4608A906A8FFF710
:108D800077FEA00502D46FF001002AE714F0240F4B
:108D90000AD0E00714D1DDE906123868031D3B60F4
:108DA0000068C0E900120BE0DDE90601FFF7C9FC2D
:108DB0000146E00704D13868021D3A60006801608E
:108DC00028460EE7000014400000F03FF1D8FFFFF6
:108DD000426842B1016811F8013B23B1521EC0E95B
:108DE0000012184670470121C160881E7047426812
:108DF0005AB1C368016843B983688B4205D0491EE4
:108E0000521CC0E90012002070474FF0FF3070473D
:108E10002DE9F04D00231A461B1A8A4103DB00207E
:108E20000146BDE8F08DC1F30A52C1F3130141F4CC
:108E300080154FF0000BD10702D100186D41521E72
:108E40000027044640F2FF11384601EB620A3E4615
:108E50008046024600204FF48011FFF7CEFCC21975
:108E60007141BB1846EB0100B4EB030C75EB000C31
:108E700004D3E41A65EB000517460E46241908F1E1
:108E800001006D4180463428E3DDF91946EB060008
:108E9000091BA84103D24FF0FF32134601E0002224
:108EA00013461BEB070046EB0A51BDE8F04DFFF7F8
:108EB0003ABD000030B5041E71F1000404DB4FF030
:108EC0000044404264EB0101141E73F1000405DB11
:108ED0001C464FF00043524263EB04038B4208BF31
:108EE000824230BD7F2801D9002208E0064A02EB09
:108EF0005002C007127800D1120902F00F020120BF
:108F0000904008407047000038F803080EB540F262
:108F1000334202920022CDE900221346FFF712FDF0
:108F200003B000BD70B58C1810F8015B15F0070395
:108F300001D110F8013B2A1106D110F8012B03E0F2
:108F400010F8016B01F8016B5B1EF9D12B0705D4FA
:108F50000023521E0DD401F8013BFAE710F8013B43
:108F6000CB1A921C03E013F8015B01F8015B521E5F
:108F7000F9D5A142D8D3002070BD10B502461078B3
:108F800003E012F8014B2318D8B20B1EA1F1010423
:108F9000A1B2F6D110BD000070B5ADF5287D044634
:108FA0000D460020A790A690002604EB44004549FA
:108FB00001EBC000408AA84203DC00200DF5287DAB
:108FC00070BD0020A69077E004EB44003D4B03EB1E
:108FD000C000028A04EB440003EBC00080892844EF
:108FE00081B2394800F010F90020A79011E004EB9D
:108FF0004400344901EBC0004068BDF89C12405C5D
:1090000001A9BDF89C228854BDF89C02401C80B286
:10901000A79004EB44002B4901EBC000008ABDF887
:109020009C128842E3DC04EB4400264A02EBC000B9
:10903000008A401E81B201A8FFF79FFF23490870F4
:1090400004EB44001F4901EBC000008A401E01A947
:10905000085C1E490978884226D10020A79016E0B6
:1090600004EB4400174901EBC0004068BDF89C12B6
:10907000405C04EB4401134A02EBC1018968BDF86E
:109080009C228854BDF89C02401C80B2A79004EB3F
:1090900044000C4901EBC000008A401EBDF89C1240
:1090A0008842DDDC012089E764202DF041FFBDF816
:1090B0009802401C80B2A690BDF89802062883DB77
:1090C00000207BE774D0030890A70020310A00201D
:1090D0002DE9F043ADF5257D04460E460025002719
:1090E000A846A94604EB4400324901EBC000408A7F
:1090F000B04204DC00200DF5257DBDE8F08300259D
:1091000018E004EB44002B4901EBC0008068405D8F
:1091100004EB4401274A02EBC1014968485504EBBE
:109120004400114601EBC0004068405D0DF80500A9
:10913000681C85B204EB44001E4901EBC000008AA4
:10914000401EA842DDDC04EB44000A4602EBC000EE
:10915000008A401E81B26846FFF70FFF04EB44010E
:10916000144A02EBC101098A491E0DF801000027CB
:109170001BE004EB44000F4B03EBC000028A04EB3E
:10918000440003EBC0008089304481B2684600F09F
:109190004FF931462046FFF7FFFE012800D1AAE72C
:1091A00064202DF0C5FE781C87B2062FE1DB00207D
:1091B000A1E7000074D0030808B50020009028F053
:1091C0001FFC0F49087000F09BF80D480078242818
:1091D00004D0272807D028280FD109E0002109480A
:1091E00080F8081D09E00121064880F8081D04E008
:1091F0000221044880F8081D00BF00BF08BD000020
:109200002C0A0020BC2200202DE9F04106460D4624
:109210001746002401202DF043FC00202849088037
:109220000DE028F0CFFB00F0800000B10BE0012042
:109230002DF07EFE22480088401C214908802048ED
:109240000088C828EDDB00BF1D480088C82832DA36
:1092500010211C4801F08CFC08211A4801F08AFCFE
:10926000E82000F031F8C5F3871000F02DF8A906CA
:10927000080E00F029F8002000F026F8002404E091
:10928000002000F021F8601C84B2042CF8DB0024DC
:1092900005E0FF2000F018F83055601C84B2BC4295
:1092A000F7DB1021074801F065FC00202DF0F8FBEA
:1092B0000120BDE8F08100202DF0F2FB0020F8E74E
:1092C0002E0A00200000024010B5044600BF022113
:1092D0000A4828F0A5FC0028F9D02146074828F0C4
:1092E000ABFC00BF0121054828F09AFC0028F9D00A
:1092F000024828F09EFCC0B210BD000000300140C2
:1093000010B501202DF0CCFB00201E4908800DE097
:1093100028F058FB00F0800000B10BE001202DF098
:1093200007FE18480088401C164908801548008828
:10933000C828EDDB00BF13480088C8281CDA1021BC
:10934000114801F015FC08210F4801F013FC3D20E5
:10935000FFF7BAFF2A20FFF7B7FF8020FFF7B4FF1F
:10936000A720FFF7B1FF1021074801F003FC002000
:109370002DF096FB012010BD00202DF091FB002068
:10938000F9E700002E0A00200000024070B50546F3
:109390000E46002401202DF083FB00202249088086
:1093A0000DE028F00FFB00F0800000B10BE0012081
:1093B0002DF0BEFD1C480088401C1B4908801A483F
:1093C0000088C828EDDB00BF17480088C82825DAC8
:1093D0001021164801F0CCFB0821144801F0CAFB0B
:1093E0008420FFF771FF0020FFF76EFF0020FFF7DA
:1093F0006BFF0020FFF768FF002404E0285DFFF703
:1094000063FF601C84B2B442F8DB1021074801F00E
:10941000B1FB00202DF044FB012070BD00202DF099
:109420003FFB0020F9E700002E0A00200000024068
:1094300070B506460C46154601202DF031FB294635
:109440003046FFF7A3FF08B9002070BD00201F4978
:1094500008800DE028F0B6FA00F0800000B10BE0C3
:1094600001202DF065FD19480088401C174908802F
:1094700016480088C828EDDB00BF14480088C828BB
:109480001EDA1021124801F073FB0821104801F088
:1094900071FB8320FFF718FFC4F38710FFF714FF59
:1094A000A106080EFFF710FF0020FFF70DFF1021A7
:1094B000074801F05FFB00202DF0F2FA0120C4E71D
:1094C00000202DF0EDFA0020BFE700002E0A00205A
:1094D0000000024030B502460020002304E012F8EC
:1094E000014B60405C1CE3B28B42F8DB30BD70B5D1
:1094F00004460D46164632462946204600F001F83D
:1095000070BDF8B503460C460020002100BF06E000
:10951000C50022FA05F5EDB20DF80050401C0428F4
:10952000F6DB00201AE0064600EBD6777F100FB975
:10953000012701E04FF0FF373D4600210BE01E5CA4
:10954000012D01D10F4601E0C1F103071DF807709D
:109550007E401E54491C0429F1DB401CA042E2D38A
:10956000F8BD000010B5044639202DF023FFE0B20D
:109570002DF040FFC4F307202DF03CFFC4F307405B
:109580002DF038FF200E2DF035FF4FF480510348A9
:1095900001F0F0FA2CF094F810BD00000004024035
:1095A0002DE9F04107460E4614463A202DF002FF01
:1095B000F0B22DF01FFF30122DF01CFF4FF4805140
:1095C0000F4801F0D7FA19E02CF07AF805461D2D66
:1095D00011D1384600F0ACF805463B202DF0EAFEEC
:1095E0004FF48051064801F0C5FA2F4434B1208869
:1095F0002844208002E02846BDE8F081E4E700002E
:10960000000402402DE9F04107460E4614463C2076
:109610002DF0D0FEF0B22DF0EDFE30122DF0EAFE6E
:109620004FF48051104801F0A5FA0CB100202080C1
:1096300019E02CF045F805461E2D11D1384600F0F2
:109640002BF905463D202DF0B5FE4FF4805106481C
:1096500001F090FA2F4434B120882844208002E0A1
:109660002846BDE8F081E4E70004024010B528F088
:10967000A1F808B100F02EF8302000F0A9F810BDD4
:1096800010B504462146362000F08EF810BD10B506
:10969000044614B1204600F0ABF8342000F098F8EE
:1096A00010BD10B50446204600F0A2F820785C28D2
:1096B00002D020782F2803D10021642000F008F97F
:1096C000322000F085F810BD10B5682000F04CF88D
:1096D00010BD000010B522202DF06CFE2DF05FFEB5
:1096E00004464FF48051024801F044FA204610BD70
:1096F000000402402DE9F0412DF051FE04462DF00A
:109700004EFE05462DF04BFE06462DF048FE074660
:109710004FF48051054801F02DFA44EA052040EA53
:10972000064040EA0760BDE8F08100000004024006
:1097300070B5044627202DF03DFE2DF030FE064684
:10974000054646B100BF2DF02AFE2070641C701E35
:10975000C0B2061EF7D14FF48051024801F00AFA58
:10976000284670BD0004024010B504460C202DF0C0
:1097700021FE20462DF03EFEFFF7BCFF10BD00008D
:1097800070B504460A202DF015FE20462DF032FE5D
:109790002DF005FE05464FF48051024801F0EAF92C
:1097A000284670BD0004024070B505460C462846A8
:1097B0002DF000FE20462DF01DFE4FF48051034891
:1097C00001F0D8F92BF07CFF70BD000000040240CE
:1097D00010B5044620462DF0EDFD4FF480510348AE
:1097E00001F0C8F92BF06CFF10BD0000000402402E
:1097F0002DE9F041064601202DF0DCFD2DF0CFFDD6
:1098000043282BDA2B20FFF7BBFF102826DA2F2066
:109810002DF0D0FD00202DF0EDFD3220FFF7D8FF18
:109820000446142C1AD1CF20FFF7AAFF0446ACB18E
:109830004C20FFF799FF00EB042739464C2000F03D
:1098400047F85020FFF790FF00EB042739465020DF
:1098500000F03EF80021702000F03AF82F202DF0A3
:10986000A9FD357828462DF0C5FD09E0761C357830
:109870005C2D01D02F2D00D1002528462DF0BAFDFA
:10988000002DF3D14FF48051024801F073F9BDE887
:10989000F08100000004024070B504462D202DF038
:1098A00089FD2DF07CFD0646054646B100BF2078B7
:1098B0002DF0A0FD641C701EC0B2061EF7D14FF43F
:1098C0008051024801F056F9284670BD000402405C
:1098D00070B505460C460D202DF06CFD28462DF088
:1098E00089FDE0B22DF086FDC4F307202DF082FD46
:1098F000C4F307402DF07EFD200E2DF07BFD4FF4CC
:109900008051024801F036F970BD000000040240A9
:1099100070B502460C46FF25FF2309E012F8010B43
:1099200080EA05010648405C80EA03050548435C7F
:10993000201EA4F10106B4B2F0D145EA032070BDA7
:10994000DCCD0308DCCE03082DE9F04103460C46CC
:1099500000200146024606E013F8010B411842F1CF
:109960000002601E84B2002CF6DC080C40EA024CB7
:10997000100C8DB21CEB050140F10002080C40EA0E
:10998000024041186FEA010080B2BDE8F08130B5B5
:1099900002460020002305E012F8015B2C18E0B21B
:1099A0005C1CE3B28B42F7DB30BD10B51DF0ECFA66
:1099B00010BD10B51DF086FA10BD10B51DF052FA9D
:1099C00010BD10B51DF0AEFA10BD10B51FF0C8FDEA
:1099D00010BD10B527F02AFA10BD00000246094B51
:1099E0009A4201D2084801E00648103801F00053BD
:1099F0001BB1064B0B40C36002E0044B0B4083607D
:109A00007047000010640240006002407D0F7D0F2F
:109A100021B1026842F00102026003E0026822F014
:109A20000102026070470000016821F0010101603D
:109A30000021016041608160C160016121214161BB
:109A40004A49884204D13D21484A103A91608CE04D
:109A500046491831884205D14FF47461434A103A9F
:109A6000916082E041493031884205D14FF4741150
:109A70003E4A103A916078E03C494831884205D12D
:109A80004FF07461394A103A91606EE037496031A5
:109A9000884204D13649354A103AD16065E03349ED
:109AA0007831884204D13349304A103AD1605CE0C1
:109AB0002E499031884204D12F492C4A103AD16066
:109AC00053E02A49A831884205D14FF03D51274A39
:109AD000103AD16049E02949884204D13D21274A02
:109AE000083A116041E025491831884205D14FF408
:109AF0007461224A083A116037E0204930318842C7
:109B000005D14FF474111D4A083A11602DE01B492C
:109B10004831884205D14FF07461184A083A116003
:109B200023E016496031884204D11149134A121FBB
:109B300011601AE011497831884204D10D490F4A69
:109B4000121F116011E00D499031884204D10A4979
:109B50000A4A121F116008E00849A831884204D15E
:109B60004FF03D51054A121F1160704710600240CE
:109B70003D000020400F002000003D201064024006
:109B800010B501F080034BB122B1436943F080036B
:109B9000436103E0436923F08003436180290BD0D4
:109BA0002AB1036801F01E042343036004E0036844
:109BB00001F01E04A343036010BD000010B5002295
:109BC0000268134B1A40CC680B6823434C6923434B
:109BD0008C692343CC6923430C6A23434C6A234397
:109BE0008C6A23434C6B23438C6B23431A430260E0
:109BF000426922F00702D1E90B3423431A43426140
:109C00000B6943604B6883608B68C36010BD0000C4
:109C10003F801CF01CB500240121202027F0D6FD38
:109C20003020009001208DF8040000208DF80600FF
:109C300003208DF8050000208DF8070069461748BD
:109C400000F022FF3021154800F094FF0021144855
:109C500080F8841600201349887001204870C8706D
:109C60004FF4FA70886000F021F80F4890F80B0F5D
:109C7000592811DD24200A49F53948710820087156
:109C80003020C870142088702020487000210648B9
:109C900080F80B1F00F04EF81CBD000000140240BD
:109CA000BC32002040390020BC2200201CB52DF021
:109CB00047FAD0202DF010FA2DF076FA00202DF082
:109CC0000BFA2DF071FA2DF03BFAD1202DF004FAA9
:109CD0002DF06AFA00240EE0062C05DA01202DF0A2
:109CE000CBF90DF8040004E000202DF0C5F90DF8C3
:109CF0000400601CC4B2072CEEDB2DF03BFA9DF88B
:109D000006000A4948719DF8050008719DF8040095
:109D1000C8709DF8020088709DF8010048709DF899
:109D20000010034880F80B1F1CBD0000C731002045
:109D3000BC2200201CB500241B4890F80B0F8DF8A6
:109D400000001A4840788DF80100184880788DF896
:109D5000020001208DF803001448C0788DF804003B
:109D6000124800798DF80500104840798DF80600FA
:109D70002DF0E6F9D0202DF0AFF92DF015FA0020E6
:109D80002DF0AAF92DF010FA00BF07E01DF804002D
:109D90002DF0A2F92DF008FA601CC4B2072CF5DBF7
:109DA0002DF0E8F91CBD0000BC220020C7310020C6
:109DB00070B502460C460025002309E012F8010B9D
:109DC00080EA05010648405C80EA03050548435CDB
:109DD000201EA4F10106B4B2F0D145EA032070BD03
:109DE000DCCD0308DCCE030810B504460B46002189
:109DF000072A00DD072244EA042001462BB901FAB4
:109E000002F081B20912084610BD012B02D11141A6
:109E1000C8B2F9E700BFF7E710B527F0FBFA10BDAD
:109E200010B527F0F7FA10BD10B527F0F3FA10BD02
:109E30000149086070470000143C014001460020C1
:109E40000022074B1B6803EA0102054B14331B6811
:109E50000B4013B10AB1012000E000207047000060
:109E6000003C0140002123498279002A3AD00A4669
:109E7000126803689A430B461A600A1D1268036849
:109E80009A430B1D1A60027911440A6803681A4349
:109E90000A60184A0832126803689A43154B08335F
:109EA0001A601A1D126803689A43124B0C331A6029
:109EB0004279102A0ED11A1F126803681A430D4BFB
:109EC00008331A601A1D126803681A43094B0C33D1
:109ED0001A600DE00749427911440A6803681A4381
:109EE0000A6005E0027911440A6803689A430A602F
:109EF00070470000003C014010B504460B460021AD
:109F0000072A00DD072244EA0420014613B9114163
:109F1000C8B210BD012B05D101FA02F081B20912BD
:109F20000846F6E700BFF4E7F0B5ADF21C5D044665
:109F30000D460020CDF81805CDF81405002604EBD9
:109F40004400584901EBC000408AA84203DC0020CD
:109F50000DF21C5DF0BD0020CDF814059AE05148CB
:109F60000122C168504800F0A9FA4E4840680078C4
:109F70008DF800009DF8000038287DD104EB4400E6
:109F8000484B03EBC000C06804EB4403454F07EBAC
:109F9000C3031B8A03FB050104EB44003B4603EBB0
:109FA000C000028A404800F089FA0020CDF8180568
:109FB00012E004EB44003B4901EBC0004068BDF8EF
:109FC0001815405CBDF818250DF80200BDF81805FD
:109FD000401C80B2CDF8180504EB4400314901EB78
:109FE000C000008ABDF818158842E2DC04EB44008A
:109FF0002C4A02EBC000008A401E81B2684600F085
:10A0000023FB064604EB4400264901EBC000008A0E
:10A01000401E1DF80000B04233D10020CDF81805D5
:10A0200020E004EB44001F4901EBC0004068BDF88C
:10A030001815415C04EB44001A4A02EBC00080682A
:10A04000BDF81825024404EB4400164B03EBC00096
:10A05000008A401E68431154BDF81805401C80B2A8
:10A06000CDF8180504EB44000E4901EBC000008A4E
:10A07000401EBDF8181500E003E08842D1DC012045
:10A0800066E764202CF054FFBDF81405401C80B234
:10A09000CDF81405BDF814050628FFF660AF0020C2
:10A0A00056E70000C87E0308E07900202DE9F04162
:10A0B000ADF5A36D04460E4600250027A8460020F6
:10A0C000009004EB4400494901EBC000408AB042D3
:10A0D00004DC00200DF5A36DBDE8F0814448807BD1
:10A0E000002878D100210846FFF71EFF01287AD109
:10A0F000002520E004EB44003C4901EBC0008068EF
:10A10000411904EB4400394A02EBC000008A401EAA
:10A110007043085C04EB440102EBC10149684855F7
:10A1200004EB4400114601EBC0004068405D01A90A
:10A130004855681C85B204EB44002C4901EBC00073
:10A14000008AA842D6DC00274BE004EB4400274BF2
:10A1500003EBC000C06804EB4403DFF890C00CEBD5
:10A16000C3031B8A03FB060104EB4400634603EBB5
:10A17000C000008A401E82B21E4800F021FA04EBA3
:10A1800044001A4A02EBC000008A401E81B201A8B6
:10A1900000F05AFA009004EB4400144A02EBC000AD
:10A1A000C06804EB4402114B03EBC202128A104454
:10A1B00004EB440203EBC202128A02FB0600411EBA
:10A1C0000122684600F0FCF931462046FFF7ACFE5C
:10A1D000012801D17EE706E064202CF0A9FE781C5E
:10A1E00087B2062FB1DB002074E70000C87E0308A9
:10A1F000BC120020E0790020F0B5ADF21C5D002516
:10A20000002400200190002600210120FFF78CFE91
:10A210004B4890F8FC6C00204A49088080E00025FB
:10A220006FE0002414E04748008800EB40004649F6
:10A2300051F83000005D4349098801EB4101424A71
:10A2400002EBC1014968085502A90855601C84B297
:10A250003C48008800EB40003B4901EBC000008A0D
:10A26000401EA042DFDC3748008800EB40000A4671
:10A2700002EBC000008A401E81B202A800F0E4F99F
:10A2800001903048008800EB40002F4B03EBC000EA
:10A29000C0682C4B1B8803EB43032B4F07EBC30316
:10A2A0001B8A03FB05012748008800EB40003B4662
:10A2B00003EBC000008A401E82B2244800F080F9FF
:10A2C0002048008800EB40003A4602EBC000C0681E
:10A2D0001C4A128802EB42023B4603EBC202128A7E
:10A2E0001044184A128802EB420203EBC202128A9F
:10A2F00002FB0500411E012201A800F061F9681C63
:10A3000085B21048008800EB40000F4901EBC00007
:10A31000408AA84285DC0B480088401C0949088017
:10A32000084800880D28FFF67AAF054880F8FC6CD5
:10A3300000210120FFF7BAFE0DF21C5DF0BD000008
:10A34000BC22002010000020C87E0308E079002015
:10A350001CB50121084627F039FA01208DF80400C8
:10A3600002208DF8050000208DF8060001208DF8F0
:10A370000700182000906946144800F085FB05226C
:10A380001146124800F0C8FB052206210F4800F0D4
:10A39000C3FB052207210D4800F0BEFBA020009062
:10A3A00002208DF8040003208DF8050000208DF8B0
:10A3B00006008DF807006946044800F065FB402060
:10A3C00000906946014800F05FFB1CBD00000240A0
:10A3D0002DE9F84300240025002700200090804646
:10A3E000FFF7B6FF00F0BCF80A202CF0A1FD6E4686
:10A3F00008212D4800F0BCFB10212B4800F0BAFBCF
:10A40000062000F091F80821274800F0B3FB08214E
:10A41000254800F0ADFB1021234800F0ABFB0120E4
:10A4200000F082F8002000F07FF808211E4800F0BC
:10A43000A1FB1E48D0F82C11B0F83021B0F8320141
:10A4400002FB0010B0F5003F02D900BE00BFFEE7DE
:10A450001748006808B9FFF7CFFE002015490880AB
:10A4600017E0002406E0134908782146FFF75CFD59
:10A47000601C84B20F48008800EB40000B4901EBE0
:10A48000C000408AA042EEDC0A480088401C09490E
:10A490000880084800880D28E3DB0748D0F80C0244
:10A4A0000549C873BDE8F88300000240C87E030870
:10A4B0001C02434210000020BC1200202DE9F04194
:10A4C00005460C461646002701202CF0E6FA082126
:10A4D000144800F04DFB1021124800F04BFB032004
:10A4E00000F022F8C4F3074000F01EF8C4F3072080
:10A4F00000F01AF8E0B200F017F800BF06E0002004
:10A5000000F012F828706D1C781C87B2B742F6DB99
:10A510000821044800F02EFB00202CF0BEFABDE814
:10A52000F08100000000024010B5044600BF022187
:10A530000A4827F075FB0028F9D02146074827F084
:10A540007BFB00BF0121054827F06AFB0028F9D0FA
:10A55000024827F06EFBC0B210BD00000030014081
:10A5600000B585B00121080327F080F9134827F0D2
:10A570002BFB0020ADF80000ADF80400ADF806009C
:10A58000ADF808004FF40070ADF80A000820ADF8EF
:10A590000C000020ADF80E000720ADF810004FF4BD
:10A5A0008270ADF802006946044827F047FB01219C
:10A5B000024827F0FDFA05B000BD00000030014060
:10A5C0002DE9F04105460C461646002701202CF0E7
:10A5D00064FA08211B4800F0CBFA1021194800F05A
:10A5E000C9FA0620FFF7A0FF0821164800F0C2FABA
:10A5F0000821144800F0BCFA1021124800F0BAFA01
:10A600000220FFF791FFC4F30740FFF78DFFC4F36B
:10A610000720FFF789FFE0B2FFF786FF00BF05E0E4
:10A620002878FFF781FF6D1C781C87B2B742F7DBF3
:10A630000821044800F09EFA00202CF02EFABDE814
:10A64000F08100000000024010B50246107803E0DF
:10A6500012F8014B2318D8B20B1EA1F10104A1B2CC
:10A66000F6D110BD2C48807F012854D100212A4802
:10A6700081772A480078C0B9012028490870284805
:10A680000068C0002749D1F8301240EA810025490E
:10A69000D1F82C1240EA41002249D1F8281208438F
:10A6A0000F2181432048017017E000201B490870EA
:10A6B0001B480068C0001B49D1F8301240EA8100F5
:10A6C0001849D1F82C1240EA41001649D1F8281255
:10A6D00008430F218143154801701348007813493E
:10A6E0000978884217D11048007811490870084647
:10A6F00000781049097888420DD00D480078064945
:10A7000008760B4800780B4908700948007810B1AA
:10A7100001200149C8757047BC120020DE0A0020E4
:10A720003402424200004242DF0A0020E00A0020D8
:10A73000E10A0020DD0A002010B5ADF57C7D002483
:10A740007DA00068FB9000200090FEF78FFF14288A
:10A750007CD17A48FEF7A5FF794908700846007851
:10A76000142874D1FEF7B0FF0021764A03C2BDF869
:10A770000000FEF7F7FE6A464FF4FA7101A8FEF7F3
:10A780000FFF71A101A82CF0B1FD714908800846A6
:10A79000008810B300BF04E000216E480155601C22
:10A7A00084B2282CF8DB01A9694A128888186AA1AA
:10A7B0002CF09CFD69490880002409E06448008869
:10A7C000C01C204401A9095C62480155601C84B288
:10A7D00062480088001FA042F0DC61A101A82CF0B3
:10A7E00085FD5B4908800846008820B3002405E009
:10A7F0000021584828300155601C84B2282CF7DB12
:10A8000001A9534A1288881853A12CF06FFD5349AF
:10A81000088000240AE04E4800880830204401A93E
:10A82000095C4C4828300155601C84B24B480088B4
:10A830000938A042EFDC4DA101A82CF057FD444996
:10A8400008800846008830B3002407E06BE05BE036
:10A850000021404850300155601C84B2142CF7DBB5
:10A8600001A93B4A128888183BA12CF03FFD3B49C7
:10A87000088000240AE0364800880C30204401A9F2
:10A88000095C344850300155601C84B2334800885C
:10A890000D38A042EFDC39A101A82CF027FD2C498E
:10A8A00008800846008820B3002405E000202949DC
:10A8B00046390855601C84B2322CF7DB01A9244AC2
:10A8C0001288881824A12CF011FD24490880002446
:10A8D0000AE01F480088801D204401A9085C1D492A
:10A8E00046390855601C84B21C480088C01FA0422D
:10A8F000EFDC00210320FFF7D9FB0120FEF7C0FEAB
:10A9000001200DF57C7D10BD0D480078422803D153
:10A910000A48FEF7BCFE0CE00120FEF7B1FE002065
:10A920000749087005E00021164880F80A1F2CF03E
:10A9300071FC00BFE5E700000D0A0000480A002096
:10A94000380A0020400A002041504E3D000000001F
:10A950005E0A0020203A00203B0000005C0A002034
:10A96000574946494E414D453D000000574946492B
:10A9700050415353574F52443D00000053455256E7
:10A9800045523D00BC22002010B5044635488442A3
:10A9900008D10121084626F029FF0021012026F0D8
:10A9A00025FF5EE03048844208D10121022026F0D4
:10A9B0001DFF0021022026F019FF52E02B4884429F
:10A9C00008D10121042026F011FF0021042026F0E7
:10A9D0000DFF46E02648844208D10121082026F0D8
:10A9E00005FF0021082026F001FF3AE021488442BB
:10A9F00008D10121102026F0F9FE0021102026F0B8
:10AA0000F5FE2EE01C48844208D10121202026F0CA
:10AA1000EDFE0021202026F0E9FE22E017488442C6
:10AA200008D10121402026F0E1FE0021402026F03F
:10AA3000DDFE16E01248844208D10121802026F074
:10AA4000D5FE0021802026F0D1FE0AE00D48844288
:10AA500007D10121801526F0C9FE0021A01526F09E
:10AA6000C5FE10BD00000240000402400008024084
:10AA7000000C024000100240001402400018024086
:10AA8000001C024000200240F0B50A4600210023CD
:10AA9000002400BF3DE0012505FA01F3156805EA31
:10AAA00003049C4234D105684F000326BE40B543E1
:10AAB000056015794E00B540066835430560157987
:10AAC000012D02D01579022D16D185684F0003267D
:10AAD000BE40B543856055794E00B5408668354324
:10AAE0008560456801268E40B54345604568967986
:10AAF0008E40B6B235434560C5684F000326BE4060
:10AB0000B543C560D5794E00B540C6683543C560CC
:10AB1000491C1029BFD3F0BDF0B5002300244D0718
:10AB2000ED0E02FA05F3CE1000F1200555F826507F
:10AB30004E07F70E0F26BE40B543CF1000F120069A
:10AB400046F82750CE1000F1200555F8265045EA6A
:10AB50000304CE1000F1200545F82640F0BD024662
:10AB6000002013690B400BB1012000E0002070476A
:10AB700041837047018370470249087E0021014AE2
:10AB800011767047BC1200200E48006800F00100EA
:10AB900000B100BE012080F3138800BF00BFBFF3E7
:10ABA0004F8F0848E438006800F4E0600649084325
:10ABB000001D0449E4390860BFF34F8F00BF00BF98
:10ABC000FEE70000F0ED00E00000FA054AF6AA20DA
:10ABD00001490860704700000030004030B502466F
:10ABE0000024002305E012F8015B2819C4B2581CA8
:10ABF000C3B28B42F7DB6042C0B230BD10B5002457
:10AC00002CF008FB64202CF093F910BD2DE9F043E3
:10AC1000ADF2DC7D07460D46164698460024A14657
:10AC20008EA00068CDF8D80700200190042E7CDCAF
:10AC30008B480079302101EB101006EBC60101EBC7
:10AC40000611884A114408718548007900F00F0008
:10AC5000303006EBC60101EB061111444871804803
:10AC6000C078302101EB101006EBC60101EB061194
:10AC7000114488717A48C07800F00F00303006EB3C
:10AC8000C60101EB06111144C871FEF7EFFC142850
:10AC900071D175480078142809D006EBC60101EB84
:10ACA0000611704A8818FEF7FCFC6F4908706E4860
:10ACB0000078142872D1B5F57A7F01DD4FF47A75EA
:10ACC000FEF702FD0021694A03C268480068FEF7EA
:10ACD00049FC6348C078302101EB10108DF8080062
:10ACE0005F48C07800F00F0030308DF809005C48F4
:10ACF000807801EB10108DF80A005948807800F038
:10AD00000F0030308DF80B005548407801EB1010E3
:10AD10008DF80C005248407800F00F0030308DF86C
:10AD20000D00534890F80B0F00E093E001EB10107A
:10AD30008DF80E004E4890F80B0F00F00F003030E9
:10AD40008DF80F00B8F1020F16D13A208DF81000DF
:10AD5000002406E0395D02AA04F109001154601CC8
:10AD600084B2AC42F6DB05F1090081B201AA02A867
:10AD7000FEF748FC47E067E0B8F1000F03D154202C
:10AD80008DF8100005E0B8F1010F02D152208DF8C6
:10AD900010003A208DF81100002429E040E0204600
:10ADA00004EBD0714910795C4FEA21190A2099FB14
:10ADB000F0F0C0EBC00109F130000844C1B202AAB2
:10ADC00004F10A001154204604EBD0714910795C5B
:10ADD00001F00F090A2099FBF0F0C0EBC00109F166
:10ADE00030000844C1B204F10B001154A01C84B21D
:10ADF000B4EB450FD3DB0A2000EB450081B201AA7A
:10AE000002A8FEF7FFFB01AA02210DF5FB60FEF789
:10AE1000F9FB0120FEF734FC00201349087019E00B
:10AE200011480078422808D106EBC60101EB061153
:10AE30000C4A8818FEF72BFC0CE00120FEF720FCE2
:10AE400000200949087005E00021094880F80A1F20
:10AE50002CF0E0F90DF2DC7DBDE8F0830D0A000076
:10AE6000C7310020600A0020380A0020400A002074
:10AE7000BC22002070B5BAB00021399138913791C9
:10AE80003691359134913391329100223092319242
:10AE90002E922F922D912C912B912A9129912891CC
:10AEA0002791269125912491239115911491139125
:10AEB0001291119110910F919FEDFE0A8DED0E0AE6
:10AEC000FDA006C8CDE90C12FDA006C8CDE90A1206
:10AED000BAE0FD48807858B30020FB498870FB48F1
:10AEE000B0F8C406FA490968C1F57A7188421FD1E1
:10AEF000F7480068C0F57A7081B2F448A0F8BC1633
:10AF00000021F348001FFEF783FDF249F048001FBF
:10AF1000FEF764FD0120F04908704FF47A70EC49A7
:10AF20008C39C1F88C000121E948001FFEF770FD43
:10AF3000E548807B50B30021E3488173E7484088AF
:10AF4000E3498C39496CC1F57A7188421ED1E048D9
:10AF50008C38406CC0F57A70E0490839488000218F
:10AF6000DB484C38FEF754FDDD49D9484C38FEF734
:10AF700035FD0120DB4908704FF47A70D4498C39D3
:10AF800048640121D2484C38FEF742FDCE48807E0D
:10AF900050B30021CC488176D0488088CC498C3988
:10AFA0004969C1F57A7188421ED1C9488C38406917
:10AFB000C0F57A70C949083988800021C4487C38B6
:10AFC000FEF726FDC849C2487C38FEF707FD012080
:10AFD000C64908704FF47A70BD498C394861012127
:10AFE000BB487C38FEF714FDB74890F8260058B3EC
:10AFF0000021B54880F82610B848C088B4498C397B
:10B00000C96AC1F57A7188421ED1B1488C38C06ACC
:10B01000C0F57A70B1490839C8800021AC4864385D
:10B02000FEF7F6FCB249AA486438FEF7D7FC0120C7
:10B03000B04908704FF47A70A5498C39C862012173
:10B04000A3486438FEF7E4FC9F488178807B014484
:10B050009D48807E01449C4890F8260008440028C2
:10B060007FF437AF13F093BA9B48007820B10020EB
:10B07000994908702D9019E09A48007828B100206D
:10B080009849087001202D9010E09848007828B168
:10B0900000209649087002202D9007E0954800781E
:10B0A00020B100209349087003202D909DF8B41022
:10B0B00001EB4100C0EBC1108F4911F83000C128ED
:10B0C00036D19DF8B41001EB4100C0EBC1108A49A4
:10B0D00001EBC000807808282AD101217B4880F844
:10B0E00014179DF8B40030B101280AD002280ED000
:10B0F000032818D111E04FF480418048FFF738FD54
:10B1000011E04FF400517D48FFF732FD0BE04FF4A2
:10B1100080517A48FFF72CFD05E04FF40061774835
:10B12000FFF726FD00BF00BF00217548016099E7C9
:10B1300065480C389DF8B41010F811000121B1EBEE
:10B14000D01F53F080806F4890F80A0FB8B1634960
:10B1500008399DF8B40031F8101009919DF8B40039
:10B1600000EB4001C1EBC010634901EBC0010123BA
:10B1700008919DF8B420DDE90801FFF747FD9DF82F
:10B18000B41001EB410000EB01105F4901EB00102E
:10B1900081792C919DF8B0000C2893F03980DFE87C
:10B1A00010F0FD960C003D17E22A023B363D4D4162
:10B1B0000550605E1D6EAB83FE969DF8B41001EBEA
:10B1C0004100C0EBC1104C4901EBC000417808467A
:10B1D000099100211BF064FDC1B228910021369134
:10B1E0001CE09DF8B41001EB410000EB0110464952
:10B1F00001EB00113031BDF8D80001EB00104178AF
:10B200009DF8A000814204D1BDF8D800C1B22891B8
:10B2100012E0BDF8D800401C81B236919DF8B40010
:10B2200000EB400101EB0010374901EB0010C17940
:10B23000BDF8D8008142D4DC00BF9DF8B40000EB1B
:10B240004001C1EBC0102C4901EBC000807800F038
:10B25000F000A0280DD19DF8B41001EB4100C0EB27
:10B26000C110254901EBC000807800F00F01299141
:10B270000AE09DF8B41001EB4100C0EBC1111E487B
:10B2800000EBC10081782991BDF8A40008B9102015
:10B2900029909DF8B41001EB4100C0EBC110164994
:10B2A00001EBC001BDF8A400401C095C2591BDF86C
:10B2B000A4002BE000000000016932303130300082
:10B2C0000169323045303000283E0020BC72002039
:10B2D0008C6002400088002012000020807900204D
:10B2E0000080201013000020208000101400002097
:10B2F0000088001015000020F88700200018024088
:10B3000088024242BC22002098400020401C81B2AA
:10B3100009919DF8B41001EB4100C0EBC111FE484A
:10B3200000EBC1010891DDE908011CF049F93790F3
:10B330009DF8B41001EB4100C0EBC110F64901EBE0
:10B34000C001BDF8A400801C095CBDF8DC0081428E
:10B3500042F062869DF8B41001EB4100C0EBC110D1
:10B36000ED4901EBC0004078002842F355869DF876
:10B37000B41001EB4100C0EBC110E74901EBC00183
:10B38000BDF8A400C01C0A5C9DF8B40040F2A111F5
:10B3900010FB01F0E14901EBC00101F562719DF87C
:10B3A000A00000EB400303EB001001EBC00080F8AD
:10B3B00044200021DA4A9DF8B40002EB00129DF807
:10B3C000A0001154D74890F82800012840D19DF8DA
:10B3D000B40000EB400101EB0010D34901EB001079
:10B3E00030309DF8A01000EB0110801C099000780F
:10B3F00020F08000803009990870BDF89400B628CC
:10B4000014D0C52819D0D52802D0D9281CD106E0DF
:10B41000BDF8A400032801DA0020259017E0BDF84C
:10B42000A400032801DA0020259010E0BDF8A40054
:10B43000032801DA0020259009E0BDF8A4000328C4
:10B4400001DA0020259002E00020259000BF00BF17
:10B45000BDF89400C3287CD01EDCB32801F0A4837F
:10B460000DDC112802F09A84122802F0DF841328E0
:10B4700002F07185B22842F0CE8501F0E5BDB52815
:10B4800001F0A883B62801F09584B92801F01A8448
:10B49000BA28F0D101F061BBD9287CD00ADCC528DC
:10B4A00001F00986CA2877D0CE2802F06D83D5280E
:10B4B000E1D109E0E12802F07D83E52802F09A83DA
:10B4C000E728D8D102F050BC9DF8B41001EB410040
:10B4D000C0EBC110904901EBC000C178934880F8DF
:10B4E000021D9DF8B41040F2A11011FB00F08B4931
:10B4F00001EBC00101F562719DF8A00000EB400274
:10B5000002EB001011F830109DF8B40040F2A112C7
:10B5100010FB02F0814A02EBC000407981427DDAE3
:10B520009DF8B41001EB410000EB01107E4901EBE6
:10B53000001030309DF8A01000EB0110801C099025
:10B540007A4890F8020D0121A1EBD01009990978F1
:10B5500000E0FDE360F3000109980170734890F882
:10B56000020DC0F34010E0BB9DF8B40000EB4001B9
:10B5700001EB00106C4901EB001030309DF8A01079
:10B5800000EB01108078C0F3401050B39DF8B40078
:10B5900000EB400101E0FDE3FDE301EB0010624937
:10B5A00001EB001030309DF8A01000EB0110801C62
:10B5B0000990007820F00200801C099908709DF81D
:10B5C000B41040F2A11011FB00F0114601EBC000D5
:10B5D00000F562709DF8A01001EB410202EB011131
:10B5E00000E00EE000EBC10018300990007820F078
:10B5F0000200801C099908709DF8B4100220FEF723
:10B6000055FD00219DF8B40040F2A11210FB02F09C
:10B61000424A02EBC0000171022200E028E09DF8DE
:10B62000B40040F2A11110FB01F03C4901EBC00154
:10B6300001F562719DF8A00000EB400303EB0010E0
:10B6400001F83020B6229DF8B40040F2A11110FBA1
:10B6500001F0324901EBC00000F562709DF8A010C6
:10B6600001EB410303EB011100EBC1004271FDE36B
:10B670002E4890F8020DC0F3C000A8B9E5229DF84D
:10B68000B40040F2A11110FB01F0244901EBC0000D
:10B6900000F562709DF8A01001EB410303EB01116E
:10B6A00000EBC1004271E2E79DF8B41001EB4100EC
:10B6B00000EB01101C4901EB001030309DF8A01088
:10B6C00000EB0110801C0990184890F8020D012130
:10B6D000A1EBD01009990A7860F300020A709DF876
:10B6E000B40000EB400101EB00100F4901EB00102A
:10B6F00030309DF8A01000EB0110801C09900B4821
:10B7000090F8020D42090998007862F34100099906
:10B7100008709DF8B4100BE0F88700205845002011
:10B72000883E0020BC12002098400020BC2200204F
:10B7300001EB410000EB0110FE4901EB001030303D
:10B740009DF8A01000EB01108078C0F340029DF836
:10B75000B40040F2A11110FB01F0F74901EBC00069
:10B7600000F562709DF8A01001EB410303EB01119D
:10B7700000EBC100007EC0F3400082427BD09DF808
:10B78000B41040F2A11011FB00F0EB4901EBC00036
:10B7900000F562709DF8A01001EB410202EB01116F
:10B7A00000EBC100183009909DF8B40000EB400197
:10B7B00001EB0011DF4800EB011030309DF8A010C4
:10B7C00000EB0110807842080998007862F341008C
:10B7D000099908709DF8B41001EB410000EB0110CD
:10B7E000D44901EB001030309DF8A01000EB01109F
:10B7F0008078C0F34000E8B3D9229DF8B40040F24D
:10B80000A11110FB01F0CC4901EBC00000F5627002
:10B810009DF8A01001EB410303EB011100EBC10007
:10B820004271C64890F8E00700287CD19DF8B4101A
:10B8300040F2A11011FB00F0BF4901EBC00000F580
:10B8400062709DF8A01001EB410202EB011100EBC8
:10B85000C10090F87F00002865D011239DF8B40046
:10B8600040F2A11110FB01F0B34901EBC00101F559
:10B87000627101E06EE088E19DF8A00000EB4002FB
:10B8800002EB001001EBC00090F8800040F2A11123
:10B8900010FB01F0A84901EBC00101F562719DF8B0
:10B8A000B40040F2A11210FB02F0A34A02EBC00266
:10B8B00002F562729DF8A00000EB400404EB00105A
:10B8C00002EBC00090F8810000EB400202EB001098
:10B8D00001EBC00080F87E30F3239DF8B40040F205
:10B8E000A11110FB01F0944901EBC00101F5627157
:10B8F0009DF8A00000EB400202EB001001EBC0003D
:10B9000090F8800040F2A11110FB01F08A4901EB90
:10B91000C00101F562719DF8B40040F2A11210FB64
:10B9200002F0854A00E096E002EBC00000F562708C
:10B930009DF8A02002EB420404EB021200EBC200CF
:10B9400090F8810000EB400202EB001001EBC00018
:10B95000437115E101229DF8B40040F2A11110FBE2
:10B9600001F0754901EBC00101F562719DF8A0007D
:10B9700000EB400303EB001001EBC0004273D9223F
:10B980009DF8B40040F2A11110FB01F06A4901EBEF
:10B99000C00101F562719DF8A00000EB400303EBCC
:10B9A000001001EBC000427101229DF8B40040F28A
:10B9B000A11110FB01F0604901EBC00000F56270BD
:10B9C0009DF8A01001EB410303EB011100EBC10056
:10B9D00080F84620594890F8E007E0BB9DF8B40095
:10B9E00040F2A11110FB01F0534901EBC00000F53A
:10B9F00062709DF8A01001EB410202EB011100EB17
:10BA0000C10090F87F0030B39DF8B41040F2A1104F
:10BA100011FB00F0484901EBC00101F562719DF88E
:10BA2000A00000EB400202EB001001EBC00090F818
:10BA3000801001EB410000EB01103E4901EB0012C8
:10BA400030329DF8B40040F2A11110FB01F03A49E8
:10BA500001EBC00100E093E001F562719DF8A000E8
:10BA600000EB400303EB001001EBC00090F88100F5
:10BA700002EB0010801C0990007820F00402099865
:10BA8000027000239DF8B40040F2A11110FB01F0F8
:10BA9000294901EBC00000F562709DF8A01001EB90
:10BAA000410202EB011100EBC10090F8800040F26E
:10BAB000A11110FB01F0204901EBC00000F56270FC
:10BAC0009DF8B41040F2A11211FB02F11A4A02EBE8
:10BAD000C10202F562729DF8A01001EB410404EB73
:10BAE000011102EBC10191F8811001EB410202EB5F
:10BAF000011100EBC10080F87E30F3239DF8B40003
:10BB000040F2A11110FB01F00B4901EBC00000F560
:10BB100062709DF8A01001EB410202EB011100EBF5
:10BB2000C10090F8800040F2A11110FB01F0024921
:10BB300006E000009840002058450020BC3200205C
:10BB400001EBC00000F562709DF8B41040F2A11244
:10BB500011FB02F1FE4A02EBC10101F562719DF891
:10BB6000A02002EB420404EB021201EBC20191F8A7
:10BB7000811001EB410202EB011100EBC1004371A6
:10BB80009DF8B4100220FEF791FA9DF8B40000EB86
:10BB9000400101EB0010EF4901EB001130319DF83D
:10BBA000A00001EB0010807800F001029DF8B400C5
:10BBB00040F2A11110FB01F0E54901EBC00000F5D6
:10BBC00062709DF8A01001EB410303EB011100EB43
:10BBD000C100007E00F00100824279D09DF8B400DF
:10BBE00040F2A11110FB01F0D94901EBC00000F5B2
:10BBF00062709DF8A01001EB410202EB011100EB15
:10BC0000C100183009909DF8B40000EB400101EB31
:10BC10000011D04800EB011030309DF8A01000EB6F
:10BC20000110807809990A7860F300020A709DF883
:10BC3000B41001EB410000EB0110C64901EB00100C
:10BC400030309DF8A01000EB0110807800F001006A
:10BC5000E8BB9DF8B41001EB410000EB0110BD49B9
:10BC600001EB001030309DF8A01000EB011080783F
:10BC7000C0F3401068B39DF8B41040F2A11011FB5E
:10BC800000F0B34901EBC00000F562709DF8A01010
:10BC900001EB410202EB011100EBC10090F84600FC
:10BCA000B8B99DF8B41040F2A11011FB00F0A849FA
:10BCB00001EBC00000F562709DF8A01001EB41029D
:10BCC00002EB011100EBC100407B10B902E070E013
:10BCD000A9E23EE09DF8B41001EB410000EB011039
:10BCE0009C4901EB001030309DF8A01000EB0110D2
:10BCF0008078C0F3400060BB01229DF8B40040F2A0
:10BD0000A11110FB01F0924901EBC00101F5627134
:10BD10009DF8A00000EB400303EB001001EBC00016
:10BD20004273D9229DF8B40040F2A11110FB01F03A
:10BD3000874901EBC00101F562719DF8A00000EB9D
:10BD4000400303EB001001EBC0004271012201E04F
:10BD5000F0E314E09DF8B40040F2A11110FB01F0F3
:10BD60007B4901EBC00000F562709DF8A01001EB6B
:10BD7000410303EB011100EBC10080F846200022D3
:10BD80009DF8B40040F2A11110FB01F0704901EBE5
:10BD9000C00001E0FEE3FEE300F562709DF8A01034
:10BDA00001EB410303EB011100EBC10080F84520DA
:10BDB00034E29DF8B41040F2A11011FB00F0644988
:10BDC00001EBC00000F562709DF8A01001EB41028C
:10BDD00002EB011100EBC10090F84600B0B901225E
:10BDE0009DF8B40040F2A11110FB01F0584901EB9D
:10BDF000C00000F562709DF8A01001EB410303EB59
:10BE0000011100EBC10080F845202AE000229DF8D6
:10BE1000B40040F2A11110FB01F04D4901EBC0014B
:10BE200001F562719DF8A00000EB400303EB0010E8
:10BE300001EBC00080F845209DF8B41001EB4100F3
:10BE400000EB0110434901EB001130319DF8A000D7
:10BE500001EB0010801C0990007820F00102099885
:10BE600002703D4890F8E00790B100E067E29DF86D
:10BE7000B40000EB400101EB0010364901EB00106B
:10BE800030309DF8A01000EB0110807A02288FD18D
:10BE9000324890F8290001288AD13048D0F80C02A5
:10BEA0002E49498D88427DD29DF8B40040F2A111FF
:10BEB00010FB01F0264901EBC00000F562709DF80F
:10BEC000A01001EB410202EB011100EBC10090F860
:10BED000450001283BD19DF8B40040F2A11110FBB0
:10BEE00001F01B4901EBC00000F562709DF8A01045
:10BEF00001EB410202EB011100EBC10090F87F0061
:10BF000028BB9DF8B40000EB400101EB0010114983
:10BF100001EB001130319DF8A00001EB0010017819
:10BF20009DF8B40040F2A11210FB02F0084A02EBA7
:10BF3000C0004170C3229DF8B40040F2A11110FB73
:10BF400001F0034901EBC00101F5627108E080E0F6
:10BF50005845002098400020BC320020BC12002030
:10BF60009DF8A00000EB400303EB001001EBC000C4
:10BF7000427100229DF8B40000EB400101EB00107B
:10BF8000FE4901EB001130319DF8A00001EB0010DB
:10BF9000426001229DF8B40000EB400101EB00106B
:10BFA000F64900E0EAE001EB001130319DF8A00015
:10BFB00001EB0010C2729DF8B4100220FEF776F873
:10BFC000002139911CE000229DF8B40040F2A1113B
:10BFD00010FB01F0EA4901EBC00101F562719DF827
:10BFE000A00000EB400303EB001001EBC001473160
:10BFF000BDF8E4000A54BDF8E400401C81B2399158
:10C00000BDF8E4000628DEDB002039901CE00022A9
:10C010009DF8B40040F2A11110FB01F0D84901EBEA
:10C02000C00101F562719DF8A00000EB400303EB35
:10C03000001001EBC0016331BDF8E4000A54BDF803
:10C04000E400401C81B23991BDF8E4000F28DEDB2A
:10C05000E4E09DF8B41040F2A11011FB00F0C849D3
:10C0600001EBC00000F562709DF8A01001EB4102E9
:10C0700002EB011100EBC10090F8450001287DD1D1
:10C080009DF8B41040F2A11011FB00F0BC4901EB87
:10C09000C00101F562719DF8A00000EB400202EBC7
:10C0A000001001EBC00090F8801040F2A11011FBCD
:10C0B00000F0B34901EBC00101F562719DF8B400D5
:10C0C00040F2A11210FB02F0AD4A02EBC00000F5F5
:10C0D00062709DF8A02002EB420303EB021200EB1A
:10C0E000C20090F8810000EB400202EB001001EB6F
:10C0F000C00090F87E00032840D100239DF8B400D2
:10C1000040F2A11110FB01F09D4901EBC00101F5C6
:10C1100062719DF8A00000EB400202EB001001EB01
:10C12000C00090F8800040F2A11110FB01F094498A
:10C1300001EBC00101F562719DF8B40040F2A1125B
:10C1400010FB02F08E4A02EBC00202F562729DF80B
:10C15000A00000EB400404EB001002EBC00090F8DC
:10C16000810000EB400202EB001001EBC00080F800
:10C170007E309DF8B41001EB410000E04EE000EB92
:10C1800001107E4901EB001130319DF8A00001EB58
:10C19000001001789DF8B40040F2A11210FB02F0EB
:10C1A000774A02EBC0004170C3229DF8B40040F210
:10C1B000A11110FB01F0724901EBC00101F56271A0
:10C1C0009DF8A00000EB400303EB001001EBC00062
:10C1D000427100229DF8B40000EB400101EB001019
:10C1E000664901EB001130319DF8A00001EB001011
:10C1F000426002229DF8B40000EB400101EB001008
:10C200005E4901EB001130319DF8A00001EB0010F8
:10C21000C2729DF8B4100220FDF748FF9DF8B410DB
:10C220000220FDF743FF9DF8B41001EB410000EB45
:10C230000110524901EB001030309DF8A01000EBC6
:10C2400001108078C0F3400050B39DF8B41040F264
:10C25000A11011FB00F04A4901EBC00000F562702B
:10C260009DF8A01001EB410202EB011100EBC100AF
:10C270004079D52814D1D9229DF8B40040F2A111FB
:10C2800010FB01F03E4901EBC00000F562709DF823
:10C29000A01001EB410303EB011100EBC10042715F
:10C2A0009DF8B41040F2A11011FB00F0344901EBED
:10C2B000C00000F562709DF8A01001EB410202EB96
:10C2C000011100EBC1008078B22838D19DF8B4107C
:10C2D00001EB410000EB0110284901EB0010303068
:10C2E0009DF8A01000EB01108078C0F3400030BB37
:10C2F0009DF8B40000EB400101EB00101F4901EB79
:10C30000001030309DF8A01000EB01108078C0F3D1
:10C310004010A0B9E5229DF8B40040F2A11110FB35
:10C3200001F0174901EBC00000F562709DF8A01004
:10C3300001EB410303EB011100EBC10042719DF8D9
:10C34000B40000EB400101EB00100C4901EB0010C0
:10C3500030309DF8A01000EB011080780121B1EB86
:10C36000D01F7DD19DF8B40000EB400101EB00101F
:10C37000024901EB0010303004E00000984000203A
:10C38000584500209DF8A01000EB0110807800F0C7
:10C390000100002864D19DF8B40040F2A11110FB07
:10C3A00001F0F74901EBC00000F562709DF8A010A4
:10C3B00001EB410202EB011100EBC10090F84600D5
:10C3C00000284DD19DF8B40000EB400101EB0010B6
:10C3D000EC4901EB001030309DF8A01000EB01108B
:10C3E0008078C0F3C000D8BB9DF8B40000EB4001DA
:10C3F00001EB0010E34901EB001030309DF8A01074
:10C4000000EB0110407A00F0010048B39DF8B40041
:10C4100040F2A11110FB01F0D94901EBC00000F579
:10C4200062709DF8A01001EB410202EB011100EBDC
:10C43000C10090F8900000F0010088B99DF8B400A8
:10C4400040F2A11110FB01F0CD4901EBC00000F555
:10C4500062709DF8A01001EB410202EB011100E0B7
:10C460003FE000EBC10090F88200D0B3002039908B
:10C470002CE09DF8B40040F2A11110FB01F0C0497E
:10C4800001EBC00101F562719DF8A00000EB4002D4
:10C4900002EB001001EBC00000F18301BDF8E400E5
:10C4A0000A5C9DF8B40000EB400101EB0010B549B7
:10C4B00001EB00100E30BDF8E410405C824200D069
:10C4C00008E0BDF8E400401C81B23991BDF8E400F9
:10C4D0000628CEDB00BFBDF8E40006286CD13990F9
:10C4E0002EE069E09DF8B41040F2A11011FB00F0BD
:10C4F000A34901EBC00101F562719DF8A00000EBBA
:10C50000400202EB001001EBC00000F18301BDF816
:10C51000E4000A5C9DF8B40000EB400101EB001060
:10C52000984901EB00100E30BDF8E410405C8242E7
:10C5300001D009E09DE2BDF8E400401C81B23991D0
:10C54000BDF8E4000A28CDDB00BFBDF8E4000A28EE
:10C5500032D09DF8B41040F2A11011FB00F08849D0
:10C5600001EBC00000F562709DF8A01001EB4102E4
:10C5700002EB011100EBC10090300990007820F02F
:10C580000100401C0999087012229DF8B40040F285
:10C59000A11101E012E0CAE210FB01F0784901EBC1
:10C5A000C00000F562709DF8A01001EB410303EBA1
:10C5B000011100EBC100427101F02DBD9DF8B410D6
:10C5C00001EB410000EB01106E4901EB0010007B14
:10C5D000D0BBBDF8A400082800D0EDE700203990BA
:10C5E00028E09DF8B41001EB4100C0EBC110664992
:10C5F00001EBC001BDF8E400C01C085C00F00F00B6
:10C60000092800DD1AE09DF8B41001EB4100C0EBF1
:10C61000C1105D4901EBC001BDF8E400C01C085C1D
:10C6200000F0F000902800DD08E0BDF8E400401CB8
:10C6300081B23991BDF8E4000628D2DB00BFBDF815
:10C64000E400062801DAB7E76EE09DF8B41001EBCC
:10C650004100C0EBC1104C4901EBC000C07801049F
:10C660009DF8B40000EB4002C2EBC010464A02EB5A
:10C67000C000007941EA00219DF8B40000EB4002BF
:10C68000C2EBC010404A02EBC000407901439DF864
:10C69000B40040F2A11210FB02F0394A02EBC002D2
:10C6A00002F562729DF8A00000EB400303EB00105E
:10C6B00002EBC000C0F81A109DF8B41001EB410065
:10C6C000C0EBC110304901EBC000807901049DF836
:10C6D000B40000EB4002C2EBC0102B4A02EBC000DA
:10C6E000C07941EA00219DF8B40000EB4002C2EBA2
:10C6F000C010254A02EBC000007A01439DF8B40047
:10C7000040F2A11210FB02F01D4A02EBC00000F53E
:10C7100062709DF8A02002EB420303EB021200EBD3
:10C72000C200C0F81E10C6E0BDF8A4000A2800D060
:10C7300042E7002039902EE09DF8B40000EB400164
:10C74000C1EBC010104901EBC001BDF8E400C01CF2
:10C75000085C00F00F00092800DD20E09DF8B4001F
:10C7600000EB4001C1EBC010074901EBC001BDF86F
:10C77000E400C01C085C00F0F000902806DD0EE02C
:10C780005845002098400020F8870020BDF8E400BC
:10C79000401C81B23991BDF8E4000828CCDB00BF11
:10C7A000BDF8E400082800DA06E79DF8B40000EBC5
:10C7B0004001C1EBC010F94901EBC000C07801068F
:10C7C0009DF8B40000EB4002C2EBC010F34A02EB4C
:10C7D000C000007941EA00419DF8B40000EB40023E
:10C7E000C2EBC010ED4A02EBC000407941EA0021E3
:10C7F0009DF8B40000EB4002C2EBC010E74A02EB28
:10C80000C000807901439DF8B40040F2A11210FBF2
:10C8100002F0E34A02EBC00202F562729DF8A0004A
:10C8200000EB400303EB001002EBC000C0F81A104D
:10C830009DF8B40000EB4001C1EBC010D74901EBFB
:10C84000C000C07901069DF8B40000EB4002C2EBC5
:10C85000C010D24A02EBC000007A41EA00419DF8C4
:10C86000B40000EB4002C2EBC010CC4A02EBC000A7
:10C87000407A41EA00219DF8B40000EB4002C2EB8F
:10C88000C010C64A02EBC000807A01439DF8B40094
:10C8900040F2A11210FB02F0C14A02EBC00000F509
:10C8A00062709DF8A02002EB420303EB021200EB42
:10C8B000C200C0F81E109DF8B40040F2A11110FB98
:10C8C00001F0B74901EBC00101F562719DF8A000CC
:10C8D00000EB400202EB001011F830109DF8B4009C
:10C8E00040F2A11210FB02F0AD4A02EBC000407909
:10C8F000814234DA00219DF8B40040F2A11210FB0D
:10C9000002F0A74A02EBC000017104229DF8B400B6
:10C9100040F2A11110FB01F0A14901EBC00101F5AA
:10C9200062719DF8A00000EB400303EB001001F8DA
:10C930003020C5229DF8B40040F2A11110FB01F097
:10C94000974901EBC00000F562709DF8A01001EB63
:10C95000410303EB011100EBC100427188E09DF837
:10C96000B41001EB410000EB01108E4901EB001007
:10C9700030309DF8A01000EB01108078C0F340002B
:10C9800058B39DF8B41040F2A11011FB00F0844997
:10C9900001EBC00000F562709DF8A01001EB4102B0
:10C9A00002EB011100EBC1004079D92815D1D52245
:10C9B0009DF8B40040F2A11110FB01F0784901EBA1
:10C9C000C00000F562709DF8A01001EB410303EB7D
:10C9D000011100EBC10042714AE09DF8B41040F231
:10C9E000A11011FB00F06E4901EBC00000F5627070
:10C9F0009DF8A01001EB410202EB011100EBC10018
:10CA0000807B012834D100229DF8B40040F2A111AE
:10CA100010FB01F0624901EBC00101F562719DF864
:10CA2000A00000EB400303EB001001EBC000827399
:10CA3000B6229DF8B40040F2A11110FB01F0584954
:10CA400001EBC00101F562719DF8A00000EB40030D
:10CA500003EB001001EBC000427100219DF8B4000F
:10CA600040F2A11210FB02F04D4A02EBC00001712E
:10CA7000A2E5D5229DF8B40040F2A11110FB01F00F
:10CA8000474901EBC00101F562719DF8A00000EB80
:10CA9000400303EB001001EBC000427101219DF83F
:10CAA000B40040F2A11210FB02F03D4A02EBC000BC
:10CAB00001719DF8B41001EB4100C0EBC110374982
:10CAC00001EBC000C078592816D19DF8B41001EBD5
:10CAD000410000EB0110334901EB001030309DF8AC
:10CAE000A01000EB0110801C0990007820F02000BD
:10CAF00020300999087014E09DF8B41001EB410052
:10CB000000EB0110274901EB001030309DF8A01018
:10CB100000EB0110801C0990007820F02002099899
:10CB200002709DF8B4100220FDF7C0FA44E5D5224A
:10CB30009DF8B40040F2A11110FB01F0184901EB7F
:10CB4000C00000F562709DF8A01001EB410303EBFB
:10CB5000011100EBC10042712EE5D5229DF8B40011
:10CB600040F2A11110FB01F00D4901EBC00101F5EC
:10CB700062719DF8A00000EB400303EB001001EB95
:10CB8000C000427101219DF8B40040F2A11210FBD7
:10CB900002F0034A02EBC00001710DE5F8870020A6
:10CBA0005845002098400020D5229DF8B40040F25E
:10CBB000A11110FB01F0FE4901EBC00000F562700D
:10CBC0009DF8A01001EB410303EB011100EBC10044
:10CBD0004271F1E49DF8B41040F2A11011FB00F095
:10CBE000F34901EBC00000F56270BDF8D81001EB0D
:10CBF000410202EB011100EBC1008079012840D114
:10CC000000229DF8B40040F2A11110FB01F0E849A8
:10CC100001EBC00101F56271BDF8D80000EB4003E3
:10CC200003EB001001EBC0008271D5229DF8B40027
:10CC300040F2A11110FB01F0DD4901EBC00101F54B
:10CC400062719DF8A00000EB400303EB001001EBC4
:10CC5000C00042719DF8B41001EB410000EB0110DF
:10CC6000D44901EB001130319DF8A00001EB001018
:10CC7000801C0990007820F00400001D09990870BC
:10CC80001FE0C3229DF8B40040F2A11110FB01F097
:10CC9000C74901EBC00101F562719DF8A00000EBEE
:10CCA000400303EB001001EBC000427100219DF82E
:10CCB000B40040F2A11210FB02F0BD4A02EBC0002A
:10CCC000017179E49DF8B41040F2A11011FB00F05D
:10CCD000B74901EBC00000F56270BDF8D81001EB58
:10CCE000410202EB011100EBC1008079012840D123
:10CCF00000229DF8B40040F2A11110FB01F0AC49F4
:10CD000001EBC00101F56271BDF8D80000EB4003F2
:10CD100003EB001001EBC0008271D5229DF8B40036
:10CD200040F2A11110FB01F0A14901EBC00101F596
:10CD300062719DF8A00000EB400303EB001001EBD3
:10CD4000C00042719DF8B41001EB410000EB0110EE
:10CD5000984901EB001130319DF8A00001EB001063
:10CD6000801C0990007820F00400001D09990870CB
:10CD70001FE0C3229DF8B40040F2A11110FB01F0A6
:10CD80008B4901EBC00101F562719DF8A00000EB39
:10CD9000400303EB001001EBC000427100219DF83D
:10CDA000B40040F2A11210FB02F0814A02EBC00075
:10CDB000017112E49DF8B41001EB410000EB011089
:10CDC0007C4901EB0010007B50BB9DF8B41001EBD7
:10CDD0004100C0EBC110784901EBC00001799DF81A
:10CDE000B40000EB4002C2EBC010734A02EBC0007B
:10CDF000C07841EA00229DF8B40040F2A11110FB76
:10CE000001F06B4901EBC00000F562709DF8A010C5
:10CE100001EB410303EB011100EBC100426335E07C
:10CE20009DF8B40000EB4001C1EBC010624901EB7A
:10CE3000C000C07801049DF8B40000EB4002C2EBD2
:10CE4000C0105D4A02EBC000007941EA00219DF864
:10CE5000B40000EB4002C2EBC010574A02EBC00026
:10CE6000407901439DF8B40040F2A11210FB02F09A
:10CE70004F4A02EBC00000F562709DF8A02002EB63
:10CE8000420303EB021200EBC20041639DF8B400C1
:10CE900040F2A11110FB01F0454901EBC00101F581
:10CEA00062719DF8A00000EB400202EB001011F847
:10CEB00030109DF8B40040F2A11210FB02F03C4A81
:10CEC00002EBC0004079814234DA00219DF8B400C1
:10CED00040F2A11210FB02F0354A02EBC0000171D2
:10CEE00003229DF8B40040F2A11110FB01F030497B
:10CEF00001EBC00101F562719DF8A00000EB400359
:10CF000003EB001001F83020D9229DF8B40040F264
:10CF1000A11110FB01F0264901EBC00000F5627081
:10CF20009DF8A01001EB410303EB011100EBC100E0
:10CF3000427188E09DF8B40040F2A11110FB01F0AD
:10CF40001B4901EBC00000F56270BDF8D81001EB81
:10CF5000410202EB011100EBC1008079012852D19E
:10CF600000229DF8B40040F2A11110FB01F010491D
:10CF700001EBC00101F56271BDF8D80000EB400380
:10CF800003EB001001EBC0008271D9229DF8B400C0
:10CF900040F2A11110FB01F0054901EBC00101F5C0
:10CFA00062719DF8A00000EB400303EB001005E068
:10CFB0005845002098400020F887002001EBC00071
:10CFC00042719DF8B41001EB410000EB0110FE49E5
:10CFD00001EB001130319DF8A00001EB0010801C26
:10CFE0000990007820F00400001D099908700120C4
:10CFF0009DF8B41040F2A11211FB02F1F34A02EBCA
:10D00000C10108711FE0C5229DF8B40040F2A111D2
:10D0100010FB01F0ED4901EBC00101F562719DF8D3
:10D02000A00000EB400303EB001001EBC0004271D5
:10D0300000219DF8B40040F2A11210FB02F0E34A77
:10D0400002EBC000017113E500219DF8B40040F22D
:10D05000A11210FB02F0DD4A02EBC00001719DF845
:10D06000B41001EB410000EB0110D74901EB0011B6
:10D0700030319DF8A00001EB0010801C0990007871
:10D0800020F00400001D09990870D5229DF8B40015
:10D0900040F2A11110FB01F0CC4901EBC00000F5FA
:10D0A00062709DF8A01001EB410303EB011100EB4E
:10D0B000C1004271DCE49DF8B41001EB410000EBCB
:10D0C0000110C14901EB0010007BD0BBBDF8A400EA
:10D0D0000C2800D0CCE40021399128E09DF8B41050
:10D0E00001EB4100C0EBC110B94901EBC001BDF833
:10D0F000E400C01C085C00F00F00092800DD1AE005
:10D100009DF8B41001EB4100C0EBC110B04901EB38
:10D11000C001BDF8E400C01C085C00F0F0009028DD
:10D1200000DD08E0BDF8E400401C81B23991BDF893
:10D13000E4000A28D2DB00BFBDF8E4000A2801DAC7
:10D1400096E482E000202E902F90002139911EE07D
:10D15000DDE92E10000240EA11620902CDE92E122B
:10D160009DF8B41001EB4100C0EBC110984901EBF0
:10D17000C001BDF8E400C01C085CDDE92E34184392
:10D18000CDE92E04BDF8E400401C80B23990BDF812
:10D19000E4000528DCDB9DF8B400DDE92E1240F246
:10D1A000A11310FB03F0894B03EBC00303F562737B
:10D1B0009DF8A00000EB400404EB001003EBC0005E
:10D1C00040F8221F426000222E922F9200213991B6
:10D1D0001EE0DDE92E10000240EA11620902CDE9ED
:10D1E0002E129DF8B41001EB4100C0EBC11078493C
:10D1F00001EBC001BDF8E4000830085CDDE92E3425
:10D200001843CDE92E04BDF8E400401C80B23990EB
:10D21000BDF8E4000528DCDB9DF8B400DDE92E2133
:10D2200040F2A11310FB03F0684B03EBC00000F5C4
:10D2300062709DF8A03003EB430404EB031300EB92
:10D24000C30022308260C160BCE0BDF8A4000E289B
:10D2500000D00DE40020399028E09DF8B41001EBD7
:10D260004100C0EBC1105A4901EBC001BDF8E40018
:10D27000C01C085C00F00F00092800DD1AE09DF8D2
:10D28000B41001EB4100C0EBC110514901EBC001EA
:10D29000BDF8E400C01C085C00F0F000902800DD40
:10D2A00008E0BDF8E400401C81B23991BDF8E4000B
:10D2B0000C28D2DB00BFBDF8E4000C2800DA35E40E
:10D2C00000202E902F90002139911EE0DDE92E10D4
:10D2D000000240EA11620902CDE92E129DF8B41055
:10D2E00001EB4100C0EBC110394901EBC001BDF8B1
:10D2F000E400C01C085CDDE92E341843CDE92E049F
:10D30000BDF8E400401C80B23990BDF8E400062866
:10D31000DCDB9DF8B400DDE92E1240F2A11310FB16
:10D3200003F02A4B03EBC00303F562739DF8A000E2
:10D3300000EB400404EB001003EBC00040F8221F98
:10D34000426000222E922F92002139911EE0DDE9E9
:10D350002E10000240EA11620902CDE92E129DF85A
:10D36000B41001EB4100C0EBC110194901EBC00141
:10D37000BDF8E4000930085CDDE92E341843CDE93E
:10D380002E04BDF8E400401C80B23990BDF8E400E2
:10D390000628DCDB9DF8B400DDE92E1240F2A11373
:10D3A00010FB03F0094B03EBC00000F562709DF821
:10D3B000A03003EB430404EB031300EBC300223063
:10D3C0008160C26006E000009840002058450020BF
:10D3D000F88700209DF8B41040F2A11011FB00F076
:10D3E000FE4901EBC00101F562719DF8A00000EB60
:10D3F000400202EB001011F830109DF8B40040F22A
:10D40000A11210FB02F0F54A02EBC0004079814204
:10D410007ED19DF8B4009DF8A01001EB0010C2175A
:10D42000CDE92E02EE4890F8E00708B39DF8B4105D
:10D4300001EB410000EB0110EA4901EB0010303034
:10D440009DF8A01000EB0110807A022810D09DF802
:10D45000B41001EB410000EB0110E24901EB0010B8
:10D4600030309DF8A01000EB0110C07A00287DDD5F
:10D4700000229DF8B40000EB400101EB0010D949F7
:10D4800001EB001030309DF8A01000EB0110C272CB
:10D49000D548D0F80C020521B0FBF1F201FB1200D7
:10D4A00000EB4001D0482C3000EB41100D300990CA
:10D4B0009DF8B40040F2A11110FB01F0C74901EB47
:10D4C000C00000F562709DF8A01001EB410202EB74
:10D4D000011100EBC100223010220146089009988A
:10D4E000FAF7B3FEC048D0F80C020521B0FBF1F208
:10D4F00001FB120000EB4001BB482C3000EB411255
:10D500009DF8B40040F2A11110FB01F0B34900E016
:10D51000D0E201EBC00101F562719DF8A00000EBC3
:10D52000400303EB001001EBC00050F81A1F42F853
:10D53000011F40685060AC48D0F80C020521B0FBD8
:10D54000F1F201FB120000EB4001A7482C3000EB88
:10D5500041129DF8B40000EB400101EB0010A1491D
:10D5600001EB001130319DF8A00000E093E101EBE8
:10D570000010007810709C48D0F80C020521B0FB18
:10D58000F1F201FB120000EB400197482C3000EB58
:10D5900041119348F538026841F81D2F8088888032
:10D5A0009148D0F80C020521B0FBF1F201FB12000A
:10D5B00000EB40018C482C3000EB41129DF8B40088
:10D5C00040F2A11110FB01F0844901EBC00101F50B
:10D5D00062719DF8A00000EB400303EB001001EB2B
:10D5E000C000406BC2F809007F48D0F80C0205214A
:10D5F000B0FBF1F201FB120000EB40017A482C3045
:10D6000000EB41129DF8B40000EB400101EB00106B
:10D61000744901EB001130319DF8A00001EB0010BE
:10D620004068C2F8230000229DF8B40000EB4001DE
:10D6300001EB00106B4901EB001130319DF8A000A7
:10D6400001EB001042600021399154E06648D0F8A7
:10D650000C020521B0FBF1F201FB120000EB4001CE
:10D6600061482C3000EB41112731BDF8E4409DF8B2
:10D67000B40040F2A11210FB02F0584A02EBC002C3
:10D6800002F562729DF8A00000EB400303EB00106E
:10D6900002EBC00090F8800040F2A11210FB02F0F3
:10D6A0004E4A02EBC00202F562729DF8B40040F2ED
:10D6B000A11310FB03F0494B03EBC00303F56273A6
:10D6C0009DF8A00000EB400505EB001003EBC00047
:10D6D00090F8810000EB400303EB001002EBC00266
:10D6E0004732BDF8E400001D105C0855BDF8E400A9
:10D6F000401C81B23991BDF8E4000628A6DB002168
:10D70000399142E000239DF8B40040F2A11110FBD2
:10D7100001F0324901EBC00101F562719DF8A000F2
:10D7200000EB400202EB001001EBC00090F880001B
:10D7300040F2A11110FB01F0284901EBC00101F5F5
:10D7400062719DF8B40040F2A11210FB02F0234A6E
:10D7500002EBC00202F562729DF8A00000EB4004EB
:10D7600004EB001002EBC00090F8810000EB4002D7
:10D7700002EB001001EBC0014731BDF8E4000B548F
:10D78000BDF8E400401C81B23991BDF8E4000A28DC
:10D79000B8DB1548D0F80C020521B0FBF1F080B2DF
:10D7A000014609900220FBF793FC00210620FCF7BC
:10D7B0007DFC0D48D0F80C020B49498D884206D2F9
:10D7C0000948D0F80C02401C0749C1F80C0200219E
:10D7D0000520FCF76BFC9DF8B40007E058450020DD
:10D7E000BC32002098400020BC12002000EB400119
:10D7F00001EB0010FA4901EB001030309DF8A01049
:10D8000000EB0110801C0990007820F00400001D3E
:10D8100009990870F348D0F80C020521B0FBF1F229
:10D8200001FB120000EB4001EE482C3000EB4110F0
:10D83000D0F823202E9800EB4001EB4800EB41107C
:10D84000C0F823200020399020E0E648D0F80C02F0
:10D850000521B0FBF1F201FB120000EB4001E148B1
:10D860002C3000EB41102730BDF8E410425C2E98BC
:10D8700000EB4001DC4800EB41112731BDF8E4002A
:10D880000A54BDF8E400401C81B23991BDF8E400AF
:10D890000628DADB59E09DF8B40000EB400101EB0B
:10D8A0000010CF4901EB001030309DF8A01000EBC4
:10D8B0000110801C0990007820F0080008300999B8
:10D8C00008709DF8B40000EB400101EB0010C44962
:10D8D00001EB001030309DF8A01000EB0110426801
:10D8E0002E9800EB4001C04800EB4110C0F8232007
:10D8F0000020399025E09DF8B40040F2A11110FB02
:10D9000001F0BA4901EBC00101F562719DF8A00078
:10D9100000EB400202EB001001EBC0014731BDF803
:10D92000E4000A5C2E9800EB4001AF4800EB411187
:10D930002731BDF8E4000A54BDF8E400401C81B270
:10D940003991BDF8E4000628D5DB9DF8B40000EB62
:10D95000400101EB0010A24901EB001030309DF8AE
:10D96000A01000EB0110801C0990007820F020022C
:10D97000099802709DF8B4100220FCF797FB9DF8FF
:10D98000B40040F2A11110FB01F0984901EBC00076
:10D9900000F562709DF8A01001EB410202EB01114D
:10D9A00000EBC100223009902E9800EB40018E4818
:10D9B00000EB41100D30102208900999FAF745FC50
:10D9C0009DF8B40040F2A11110FB01F0874901EB72
:10D9D000C00101F562719DF8A00000EB400202EB6E
:10D9E000001001EBC0012E9800EB40027E4800EBD6
:10D9F000421051F81A2F40F8012F496841609DF8F4
:10DA0000B40000EB400101EB0010754901EB00117F
:10DA100030319DF8A00001EB001001782E9800EB4A
:10DA20004002714800EB421001702E9800EB40015B
:10DA30006D4800EB41116E48026841F81D2F808847
:10DA400088809DF8B40040F2A11110FB01F06749F5
:10DA500001EBC00101F562719DF8A00000EB4002EE
:10DA600002EB001001EBC000416B2E9800EB40026E
:10DA70005D4800EB4210C0F809102E9881B20820D2
:10DA80000991FCF713FB00229DF8B40040F2A111AC
:10DA900010FB01F0554901EBC00000F562709DF8E4
:10DAA000A01001EB410303EB011100EBC10080F872
:10DAB000462053E09DF8B40000EB400101EB00105C
:10DAC000474901EB001030309DF8A01000EB011029
:10DAD000801C0990007820F00400001D099908704E
:10DAE0009DF8B40000EB400101EB00103C4901EB54
:10DAF000001030309DF8A01000EB0110801C099040
:10DB0000007820F0800080300999087001209DF88D
:10DB1000B41040F2A11211FB02F1344A02EBC10130
:10DB200008719DF8B41040F2A11011FB00F01146ED
:10DB300001EBC00042799DF8B40040F2A11110FB46
:10DB400001F02A4901EBC00000F562709DF8A010B9
:10DB500001EB410303EB011100F83120D5229DF8C0
:10DB6000B40040F2A11110FB01F0204901EBC0000C
:10DB700000F562709DF8A01001EB410303EB011169
:10DB800000EBC100427146E2D5229DF8B40040F29C
:10DB9000A11110FB01F0154901EBC00000F5627006
:10DBA0009DF8A01001EB410303EB011100EBC10054
:10DBB000427130E2D5229DF8B40040F2A11110FB71
:10DBC00001F00A4901EBC00000F562709DF8A01059
:10DBD00001EB410303EB011100EBC10042711AE2BA
:10DBE00098400020BC120020D81400205845002086
:10DBF000C73100200121FE4880F804179DF8B410B9
:10DC000040F2A11011FB00F0FA4901EBC00101F54F
:10DC100062719DF8A00000EB400202EB001011F8C9
:10DC200030109DF8B40040F2A11210FB02F0F14A4E
:10DC300002EBC0004079814234DA00219DF8B40043
:10DC400040F2A11210FB02F0EA4A02EBC00001719F
:10DC500001229DF8B40040F2A11110FB01F0E5494A
:10DC600001EBC00101F562719DF8A00000EB4003DB
:10DC700003EB001001F8302011229DF8B40040F2AF
:10DC8000A11110FB01F0DB4901EBC00000F562704F
:10DC90009DF8A01001EB410303EB011100EBC10063
:10DCA000427160E09DF8B41040F2A11011FB00F049
:10DCB000D04901EBC00000F562709DF8A01001EBA7
:10DCC000410202EB011100EBC1008078B22835D18E
:10DCD00000219DF8B40040F2A11210FB02F0C54AE9
:10DCE00002EBC0000171B2229DF8B40040F2A11114
:10DCF00010FB01F0BF4901EBC00101F562719DF815
:10DD0000A00000EB400303EB001001EBC0004271E8
:10DD100000229DF8B40040F2A11110FB01F0B549BA
:10DD200001EBC00000F562709DF8A01001EB41030B
:10DD300003EB011100EBC100827014E0D5229DF8C5
:10DD4000B40040F2A11110FB01F0AA4901EBC000A0
:10DD500000F562709DF8A01001EB410303EB011187
:10DD600000EBC100427156E10021A14880F8041780
:10DD7000D5229DF8B40040F2A11110FB01F09D499D
:10DD800001EBC00000F562709DF8A01001EB4103AB
:10DD900003EB011100EBC10042713CE101229DF84F
:10DDA000B40040F2A11110FB01F0924901EBC00157
:10DDB00001F562719DF8A00000EB400303EB001039
:10DDC00001EBC00080F882200021399129E09DF804
:10DDD000B41001EB4100C0EBC110874901EBC00159
:10DDE000BDF8E400C01C0A5C9DF8B40040F2A1112B
:10DDF00010FB01F07F4901EBC00101F562719DF854
:10DE0000A00000EB400303EB001001EBC00000F1A9
:10DE10008301BDF8E4000A54BDF8E400401C81B25F
:10DE20003991BDF8E4000A28D1DBF4E09DF8B41084
:10DE300001EB4100C0EBC1106F4901EBC000C0789D
:10DE400001049DF8B40000EB4002C2EBC0106A4A26
:10DE500002EBC000007941EA00209DF8B41001EB0C
:10DE60004102C2EBC111644A02EBC1014979084386
:10DE7000B0F5E13F6ED19DF8B41001EB410000EB2D
:10DE800001105E4901EB001030309DF8A01000EB4E
:10DE90000110801C0990007820F00402099802709B
:10DEA00000229DF8B40040F2A11110FB01F051498D
:10DEB00001EBC00000F562709DF8A01001EB41037A
:10DEC00003EB011100EBC100A0F88E2013229DF896
:10DED000B40040F2A11110FB01F0464901EBC00073
:10DEE00000F562709DF8A01001EB410303EB0111F6
:10DEF00000EBC10042719DF8B41001EB410000EB52
:10DF000001103E4901EB0010407903464FF4805266
:10DF10004FF4E13109909DF8B40019F063FB9DF8CE
:10DF2000B41040F2A11011FB00F0324901EBC00126
:10DF300001F562719DF8A00000EB400202EB0010B9
:10DF400001EBC00090300990007820F00800083004
:10DF5000099908705FE09DF8B40000EB4001C1EB47
:10DF6000C010254901EBC00001799DF8B40000EB19
:10DF70004002C2EBC010204A02EBC000C07841EA68
:10DF800000229DF8B40040F2A11110FB01F01949E4
:10DF900001EBC00101F562719DF8A00000EB4003A8
:10DFA00003EB001001EBC000A0F88E209DF8B40038
:10DFB00040F2A11110FB01F00E4901EBC00101F587
:10DFC00062719DF8A00000EB400202EB001001EB33
:10DFD000C000B0F88E109DF8B40000EB400202EBD8
:10DFE0000010064A02EB0010408B814212DB07E072
:10DFF000BC32002058450020F887002098400020BF
:10E000000621A2F504729DF8B40002EB00129DF8FF
:10E01000A000115400BF00BF10F0FAB89DF8B40082
:10E0200000EB4001C1EBC010FE4911F8300004289C
:10E0300001D125900BE09DF8B40000EB4001C1EB4D
:10E04000C010F84911F83000152800D125909DF82E
:10E05000B40000EB4001C1EBC010F24901EBC0007D
:10E0600041789DF8B40000EB4002C2EBC010ED4ACD
:10E0700012F8300041EA002041F23001884202D11A
:10E08000A62025903DE09DF8B40000EB4001C1EBD7
:10E09000C010E44901EBC00041789DF8B40000EBEA
:10E0A0004002C2EBC010DF4A12F8300041EA002003
:10E0B00041F23101884202D1A720259021E09DF84C
:10E0C000B40000EB4001C1EBC010D64911F830009C
:10E0D000022816D19DF8B40000EB4001C1EBC0103E
:10E0E000D04901EBC00001799DF8B40000EB40027B
:10E0F000C2EBC010CB4A02EBC000C07841EA00215D
:10E1000025919DF8B40040F2A11110FB01F0C64921
:10E1100001EBC000817828910021C44A9DF8B40029
:10E1200002EB00129DF8A0001154C14890F828009D
:10E13000012815D19DF8B40000EB400101EB00105F
:10E14000BC4901EB001030309DF8A01000EB01102D
:10E15000801C0990007820F08000803009990870B8
:10E16000BDF8941043F23002881A91427ED009DC47
:10E1700004297CD015297BD0A62910D0A72942F0EC
:10E18000EF8268E1B0F5C06F73D0A0F201600028A3
:10E1900070D001286FD00428F1D101F077BE0021A2
:10E1A0009DF8B40040F2A11210FB02F09E4A02EB6F
:10E1B000C00001719DF8B40040F2A11110FB01F004
:10E1C000114601EBC00000F562709DF8A01001EB54
:10E1D000410202EB011110F83100052829DC06226A
:10E1E0009DF8B40040F2A11110FB01F08E4901EB43
:10E1F000C00101F562719DF8A00000EB400303EB44
:10E20000001001F83020A8229DF8B40040F2A111BE
:10E2100010FB01F0844901EBC00000F562709DF82D
:10E22000A01001EB410303EB011100EBC1004271AF
:10E230000FE19DF8B40040F2A11110FB01F07A4902
:10E2400001EBC00000F562709DF8A01001EB4102E7
:10E2500002EB011110F831000A2830DC0B229DF886
:10E26000B40040F2A11110FB01F005E0B9E138E281
:10E27000F4E3F4E3F4E3F4E36B4901EBC00101F5EB
:10E2800062719DF8A00000EB400303EB001001F861
:10E290003020A9229DF8B40040F2A11110FB01F03A
:10E2A000614901EBC00000F562709DF8A01001EB20
:10E2B000410303EB011100EBC1004271C9E09DF87D
:10E2C000B40040F2A11110FB01F0574901EBC0006E
:10E2D00000F562709DF8A01001EB410202EB011104
:10E2E00010F831000F2829DC10229DF8B40040F20C
:10E2F000A11110FB01F04C4901EBC00101F5627165
:10E300009DF8A00000EB400303EB001001F8302063
:10E31000A2229DF8B40040F2A11110FB01F0424985
:10E3200001EBC00000F562709DF8A01001EB410305
:10E3300003EB011100EBC10042718AE09DF8B400CB
:10E3400040F2A11110FB01F0374901EBC00000F5CC
:10E3500062709DF8A01001EB410202EB011100EB8D
:10E36000C1004079A52815D19DF8B40000EB40010B
:10E3700001EB00102F4901EB001030309DF8A01088
:10E3800000EB0110801C0990007820F00400001DB3
:10E39000099908709DF8B41040F2A11011FB00F02B
:10E3A000214901EBC00000F562709DF8A01001EB5F
:10E3B000410202EB011100EBC1008078A12848D096
:10E3C0009DF8B41040F2A11011FB00F0164901EBCA
:10E3D000C00101F562719DF8A00000EB400202EB64
:10E3E000001001EBC00082789DF8B40040F2A1114A
:10E3F00010FB01F00C4901EBC00101F562719DF8C1
:10E40000A00000EB400303EB001001EBC0004271E1
:10E41000A1229DF8B40040F2A11110FB01F00249C5
:10E420000AE00000F887002058450020883E0020C0
:10E43000BC1200209840002001EBC00000F5627083
:10E440009DF8A01001EB410303EB011100EBC100AB
:10E45000827002F085B900219DF8B40040F2A1124B
:10E4600010FB02F0FE4A02EBC00001719DF8B410EF
:10E4700040F2A11011FB00F0114601EBC00000F5C5
:10E4800062709DF8A01001EB410202EB011110F83F
:10E49000310008281FDC00219DF8B40040F2A112D1
:10E4A00010FB02F0EE4A02EBC000017108229DF859
:10E4B000B40040F2A11110FB01F0E94901EBC000EA
:10E4C00000F562709DF8A01001EB410303EB011110
:10E4D00000F8312028E09DF8B41040F2A11011FBA3
:10E4E00000F0DF4901EBC00000F562709DF8A0105C
:10E4F00001EB410202EB011110F831000B2813DC93
:10E500000C229DF8B40040F2A11110FB01F0D44997
:10E5100001EBC00000F562709DF8A01001EB410313
:10E5200003EB011100F831209DF8B41040F2A11066
:10E5300011FB00F0CA4901EBC00000F562709DF8C4
:10E54000A01001EB410202EB011100EBC100407988
:10E55000A42830D19DF8B41001EB410000EB01106C
:10E56000C04901EB001030309DF8A01000EB011005
:10E57000801C0990007820F0200020300999087054
:10E5800000229DF8B40040F2A11110FB01F0B44943
:10E5900001EBC00000F562709DF8A01001EB410393
:10E5A00003EB011100EBC10080F845209DF8B41089
:10E5B0000220FBF77BFDA1229DF8B40040F2A111DF
:10E5C00010FB01F0A64901EBC00000F562709DF858
:10E5D000A01001EB410303EB011100EBC1004271FC
:10E5E00037E70021399115E09DF8B41001EB4100A7
:10E5F000C0EBC1109C4901EBC001BDF8E400C01C98
:10E600000A5C16A9BDF8E4000A54BDF8E400401CF9
:10E6100081B23991BDF8E4000628E5DB062116A891
:10E6200028F0CAFC0021CDE93001DDE93021100AD3
:10E6300040EA0164309BE21841EB2120CDE908203B
:10E640004FF480724FF00003DDE90801F9F7BAFDDD
:10E650009DF8B40040F2A11110FB01F0804901EBDC
:10E66000C00000F562709DF8A01001EB410303EBC0
:10E67000011100EBC100027100209DF8B41040F2BE
:10E68000A11211FB02F1764A02EBC10108710422CA
:10E690009DF8B40040F2A11110FB01F0704901EBAC
:10E6A000C00000F562709DF8A01001EB410303EB80
:10E6B000011100F83120A7229DF8B40040F2A11109
:10E6C00010FB01F0664901EBC00000F562709DF897
:10E6D000A01001EB410303EB011100EBC1004271FB
:10E6E000B7E69DF8B41040F2A11011FB00F05C49B0
:10E6F00001EBC00000F562709DF8A01001EB410233
:10E7000002EB011110F83100042878DA00219DF89D
:10E71000B40040F2A11210FB02F0514A02EBC0001B
:10E720000171A1229DF8B40040F2A11110FB01F08B
:10E730004B4901EBC00101F562719DF8A00000EBAF
:10E74000400303EB001001EBC00042719DF8B410D0
:10E7500040F2A11011FB00F0414901EBC00101F5AD
:10E7600062719DF8A00000EB400202EB001001EB8B
:10E77000C00109910878401CC1B2099801709DF848
:10E78000B41040F2A11011FB00F0354901EBC000BC
:10E7900000F562709DF8A01001EB410202EB01113F
:10E7A00010F83100042828D10A229DF8B40040F264
:10E7B000A11110FB01F02A4901EBC00101F56271C2
:10E7C0009DF8A00000EB400303EB001001F830209F
:10E7D000A3229DF8B40040F2A11110FB01F02049E2
:10E7E00001EBC00000F562709DF8A01001EB410341
:10E7F00003EB011100EBC1004271E4E2FFE79DF879
:10E80000B41040F2A11011FB00F0154901EBC0005B
:10E8100000F562709DF8A01001EB410202EB0111BE
:10E8200010F8310004283BD100219DF8B40040F2DB
:10E83000A11210FB02F00A4A02EBC000017105228E
:10E840009DF8B40040F2A11110FB01F0044901EB66
:10E85000C00101F562719DF8A00000EB400305E0E6
:10E860005845002098400020F887002003EB001056
:10E8700001F83020A3229DF8B40040F2A11110FB52
:10E8800001F0FE4901EBC00000F562709DF8A01098
:10E8900001EB410303EB011100EBC100427192E275
:10E8A0009DF8B41040F2A11011FB00F0F34901EB08
:10E8B000C00000F562709DF8A01001EB410202EB70
:10E8C000011110F83100082834DC00219DF8B40053
:10E8D00040F2A11210FB02F0E84A02EBC000017105
:10E8E00009229DF8B40040F2A11110FB01F0E349A8
:10E8F00001EBC00101F562719DF8A00000EB40033F
:10E9000003EB001001F83020A7229DF8B40040F27C
:10E91000A11110FB01F0D94901EBC00000F56270B4
:10E920009DF8A01001EB410303EB011100EBC100C6
:10E93000427148E29DF8B41040F2A11011FB00F0C2
:10E94000CE4901EBC00000F562709DF8A01001EB0C
:10E95000410202EB011110F83100092834DC0021DA
:10E960009DF8B40040F2A11210FB02F0C34A02EB82
:10E97000C00001710A229DF8B40040F2A11110FB01
:10E9800001F0BE4901EBC00101F562719DF8A000E4
:10E9900000EB400303EB001001F83020A3229DF8A8
:10E9A000B40040F2A11110FB01F0B44901EBC0002A
:10E9B00000F562709DF8A01001EB410303EB01111B
:10E9C00000EBC1004271FEE19DF8B41040F2A110CD
:10E9D00011FB00F0A94901EBC00000F562709DF841
:10E9E000A01001EB410202EB011110F831000D28DB
:10E9F00038DC00219DF8B40040F2A11210FB02F0B7
:10EA00009E4A02EBC00001710E229DF8B40040F254
:10EA1000A11110FB01F0994901EBC00101F56271F0
:10EA20009DF8A00000EB400303EB001001F830203C
:10EA3000A1229DF8B40040F2A11110FB01F08F4912
:10EA400001EBC00000F562709DF8A01001EB4103DE
:10EA500003EB011100EBC1004271B4E1B4E1E8E164
:10EA60003DE21BE29DF8B41040F2A11011FB00F052
:10EA7000824901EBC00000F562709DF8A01001EB27
:10EA8000410202EB011110F831000E2834DC0021A4
:10EA90009DF8B40040F2A11210FB02F0774A02EB9D
:10EAA000C00001710F229DF8B40040F2A11110FBCB
:10EAB00001F0724901EBC00101F562719DF8A000FF
:10EAC00000EB400303EB001001F83020A3229DF877
:10EAD000B40040F2A11110FB01F0684901EBC00045
:10EAE00000F562709DF8A01001EB410303EB0111EA
:10EAF00000EBC100427166E19DF8B41040F2A11034
:10EB000011FB00F05D4901EBC00000F562709DF85B
:10EB1000A01001EB410202EB011110F831001028A6
:10EB20007DDC11229DF8B40040F2A11110FB01F030
:10EB3000524901EBC00101F562719DF8A00000EBA4
:10EB4000400303EB001001F83020A1229DF8B4002F
:10EB500040F2A11110FB01F0484901EBC00101F5A1
:10EB600062719DF8A00000EB400303EB001001EB85
:10EB7000C00042719DF8B40040F2A11110FB01F0F9
:10EB80003E4901EBC00101F562719DF8A00000EB68
:10EB9000400303EB001001EBC00082709DF8B4103D
:10EBA00001EB410000EB0110354901EB0011303160
:10EBB0009DF8A00001EB0010801C0990007820F067
:10EBC00080008030099908709DF8B41001EB410075
:10EBD00000EB01102A4901EB001030309DF8A01025
:10EBE00000EB0110801C0990007820F00400001D4B
:10EBF000099908709DF8B41001EB410000EB011079
:10EC00001F4901EB001030309DF8A01000EB0110FF
:10EC10008078C0F3401080B39DF8B41000E046E067
:10EC200001EB410000EB0110154901EB0010303001
:10EC30009DF8A01000EB0110801C0990007820F0D6
:10EC40002002099802709DF8B41001EB410000EB1E
:10EC500001100B4901EB001030309DF8A01000EBC3
:10EC600001108078C0F34000D8B99DF8B41001EBD2
:10EC7000410000EB0110024904E083E05845002008
:10EC80009840002001EB001030309DF8A01000EB00
:10EC90000110801C0990007820F0080008300999C4
:10ECA00008709DF8B4100220FBF700FA8BE09DF885
:10ECB000B41040F2A11011FB00F0FE4901EBC001BD
:10ECC00001F562719DF8A00000EB400202EB00101C
:10ECD00011F830109DF8B40040F2A11210FB02F0C0
:10ECE000F44A02EBC000407981426CD19DF8B41027
:10ECF00040F2A11011FB00F0114601EBC00000F53D
:10ED000062709DF8A01001EB410202EB011100EBD3
:10ED1000C1008078A12836D0A3229DF8B40040F22B
:10ED2000A11110FB01F0E34901EBC00101F5627193
:10ED30009DF8A00000EB400303EB001001EBC000C6
:10ED400042719DF8B41040F2A11011FB00F0D949B6
:10ED500001EBC00000F562709DF8A01001EB4102CC
:10ED600002EB011100EBC1008078A2282BD000201B
:10ED70009DF8B41040F2A11211FB02F1CD4A02EB52
:10ED8000C10108711FE0A1229DF8B40040F2A11159
:10ED900010FB01F0C74901EBC00101F562719DF85C
:10EDA000A00000EB400303EB001001EBC000427138
:10EDB00001219DF8B40040F2A11210FB02F0BD4AFF
:10EDC00002EBC00001710BE4A1229DF8B40040F2F7
:10EDD000A11110FB01F0B74901EBC00101F562710F
:10EDE0009DF8A00000EB400303EB001001EBC00016
:10EDF00082709DF8B40040F2A11110FB01F0AD4902
:10EE000001EBC00101F562719DF8A00000EB400329
:10EE100003EB001001EBC000427100219DF8B4002B
:10EE200040F2A11210FB02F0A24A02EBC0000171F5
:10EE300056E400219DF8B40040F2A11210FB02F04C
:10EE40009C4A02EBC000017109229DF8B40040F217
:10EE5000A11110FB01F0974901EBC00101F56271AE
:10EE60009DF8A00000EB400303EB001001F83020F8
:10EE7000A7229DF8B40040F2A11110FB01F08D49CA
:10EE800001EBC00000F562709DF8A01001EB41039A
:10EE900003EB011100EBC100427121E400219DF858
:10EEA000B40040F2A11210FB02F0824A02EBC00053
:10EEB0000171A7229DF8B40040F2A11110FB01F0EE
:10EEC0007C4901EBC00000F562709DF8A01001EBD9
:10EED000410303EB011100EBC100427173E7002114
:10EEE0009DF8B40040F2A11210FB02F0714A02EB4F
:10EEF000C0000171A7229DF8B40040F2A11110FBDF
:10EF000001F06C4901EBC00101F562719DF8A000B0
:10EF100000EB400303EB001001EBC00042719DF8D1
:10EF2000B40000EB4001C1EBC010634901EBC0002D
:10EF3000407930287ED19DF8B40040F2A11110FB39
:10EF400001F05C4901EBC00101F562719DF8A00080
:10EF500000EB400202EB001011F830109DF8B400F5
:10EF600040F2A11210FB02F0524A02EBC0004079BD
:10EF700081425FD19DF8B40040F2A11110FB01F075
:10EF8000114601EBC00000F562709DF8A01001EB86
:10EF9000410202EB011100EBC100C078312830D1F1
:10EFA0009DF8B40000EB400101EB0010434901EB78
:10EFB000001030309DF8A01000EB0110801C09906B
:10EFC000007820F020020998027000229DF8B40019
:10EFD00040F2A11110FB01F0364901EBC00000F531
:10EFE00062709DF8A01001EB410303EB011100EBEF
:10EFF000C10080F845209DF8B4100220FBF756F8B8
:10F0000057E09DF8B40040F2A11110FB01F029492E
:10F0100001EBC00000F562709DF8A01001EB410209
:10F0200002EB011100EBC100C078332841D19DF8FB
:10F03000B40000E06FE000EB400101EB00101F495D
:10F0400001EB001030309DF8A01000EB0110801C87
:10F050000990007820F020020998027001229DF8A2
:10F06000B40040F2A11110FB01F0124901EBC00005
:10F0700000F562709DF8A01001EB410303EB011154
:10F0800000EBC10080F84620A9229DF8B40040F2B0
:10F09000A11110FB01F0074901EBC00000F56270FF
:10F0A0009DF8A01001EB410303EB011100EBC1003F
:10F0B000827005E058450020F88700209840002025
:10F0C0009DF8B40000EB400101EB0010FE4901EB9C
:10F0D000001030309DF8A01000EB0110801C09904A
:10F0E000007820F00102099802709DF8B41001EB3D
:10F0F000410000EB0110F44901EB001030309DF8A5
:10F10000A01000EB0110801C0990007820F0020292
:10F1100009980270D6E39DF8B41001EB4100C0EBF2
:10F12000C110EA4901EBC000407931287ED19DF839
:10F13000B41040F2A11011FB00F0E54901EBC00151
:10F1400001F562719DF8A00000EB400202EB001097
:10F1500011F830109DF8B40040F2A11210FB02F03B
:10F16000DB4A02EBC000407981425FD19DF8B410C8
:10F1700040F2A11011FB00F0114601EBC00000F5B8
:10F1800062709DF8A01001EB410202EB011100EB4F
:10F19000C10090F8460058BB01229DF8B40040F22F
:10F1A000A11110FB01F0CA4901EBC00101F5627128
:10F1B0009DF8A00000EB400303EB001001EBC00042
:10F1C00080F845209DF8B41001EB410000EB0110E0
:10F1D000BD4901EB001130319DF8A00001EB00109A
:10F1E000801C0990007820F00100401C09990870EB
:10F1F0009DF8B41001EB410000EB0110B24901EBA6
:10F20000001030309DF8A01000EB0110801C099018
:10F21000007820F0020209980270AE4890F8E007EA
:10F2200090B19DF8B41001EB410000E005E200EB65
:10F230000110A54901EB001030309DF8A01000EB43
:10F240000110807A022877D1A34890F8290001287C
:10F25000F9D1A148D0F80C029F49498D88426BD260
:10F260009DF8B41040F2A11011FB00F0984901EB99
:10F27000C00000F562709DF8A01001EB410202EBA6
:10F28000011100EBC10090F84500012853D19DF811
:10F29000B41040F2A11011FB00F08D4901EBC00049
:10F2A00000F562709DF8A01001EB410202EB011124
:10F2B00000EBC10090F87F00E8BB01229DF8B4008C
:10F2C00000EB400101EB00107F4901EB00113031F0
:10F2D0009DF8A00001EB0010C27200229DF8B4005E
:10F2E00000EB400101EB0010774901EB00113031D8
:10F2F0009DF8A00001EB001042604FF010429DF815
:10F30000B40040F2A11110FB01F0714901EBC00102
:10F3100001F562719DF8A00000EB400303EB0010C3
:10F3200001EBC00082609DF8B41001EB410000EBDE
:10F330000110654901E071E06FE001EB001130312F
:10F340009DF8A00001EB001001789DF8B40040F298
:10F35000A11210FB02F05E4A02EBC00041709DF862
:10F36000B41040F2A11011FB00F0114601EBC001F6
:10F3700001F562719DF8A00000EB400202EB001065
:10F3800011F830109DF8B40040F2A11210FB02F009
:10F390004F4A02EBC000407981423ED100229DF8E5
:10F3A000B40040F2A11110FB01F0494901EBC0018A
:10F3B00001F562719DF8A00000EB400303EB001023
:10F3C00001EBC000C271A4229DF8B40040F2A1116B
:10F3D00010FB01F03E4901EBC00101F562719DF89F
:10F3E000A00000EB400303EB001001EBC0008270B3
:10F3F000A3229DF8B40040F2A11110FB01F03449A2
:10F4000001EBC00000F562709DF8A01001EB410314
:10F4100003EB011100EBC100427153E29DF8B410FF
:10F4200040F2A11011FB00F0294901EBC00000F5EA
:10F4300062709DF8A01001EB410202EB011100EB9C
:10F44000C10090F8450001287DD19DF8B41040F22C
:10F45000A11011FB00F01E4901EBC00101F5627122
:10F460009DF8A00000EB400202EB001001EBC00091
:10F4700090F8801040F2A11011FB00F0144901EB4C
:10F48000C00101F562719DF8B40040F2A11210FBB9
:10F4900002F00F4A02EBC00000F562709DF8A02058
:10F4A00002EB420303EB021200EBC20090F8810072
:10F4B00000EB400202EB001001EBC00090F87E0070
:10F4C000032840D1022209E098400020F88700205C
:10F4D00058450020BC320020BC1200209DF8B4002A
:10F4E00000EB400101EB0010F94901EB0011303154
:10F4F0009DF8A00001EB0010C2724FF010429DF881
:10F50000B40040F2A11110FB01F0F24901EBC0017F
:10F5100001F562719DF8A00000EB400303EB0010C1
:10F5200001EBC00082609DF8B41001EB410000EBDC
:10F530000110E74901EB001130319DF8A00001EB0B
:10F540000010017800E0B0E19DF8B40040F2A11293
:10F5500010FB02F0DF4A02EBC00041709DF8B410CE
:10F5600040F2A11011FB00F0114601EBC00101F5C2
:10F5700062719DF8A00000EB400202EB001011F850
:10F5800030109DF8B40040F2A11210FB02F0D14AF5
:10F5900002EBC000407981423ED100229DF8B400C8
:10F5A00040F2A11110FB01F0CA4901EBC00101F5C5
:10F5B00062719DF8A00000EB400303EB001001EB2B
:10F5C000C000C271A4229DF8B40040F2A11110FB4A
:10F5D00001F0C04901EBC00101F562719DF8A00086
:10F5E00000EB400303EB001001EBC0008270A3228C
:10F5F0009DF8B40040F2A11110FB01F0B54901EBF8
:10F60000C00000F562709DF8A01001EB410303EB10
:10F61000011100EBC100427100229DF8B40000EB23
:10F62000400101EB0010AA4901EB001030309DF8B9
:10F63000A01000EB0110426044E19DF8B41001EB12
:10F640004100C0EBC110A44901EBC0004079332850
:10F650007ED19DF8B41001EB410000EB01109C49F4
:10F6600001EB001030309DF8A01000EB0110801C61
:10F670000990007820F00100401C099908709DF85D
:10F68000B41001EB410000EB0110914901EB0010B7
:10F6900030309DF8A01000EB0110801C099000781C
:10F6A00020F02002099802709DF8B41001EB41008F
:10F6B00000EB0110864901EB001030309DF8A010DE
:10F6C00000EB0110801C0990007820F00200801CE3
:10F6D000099908709DF8B41040F2A11011FB00F0D8
:10F6E0007C4901EBC00042799DF8B40040F2A111C1
:10F6F00010FB01F0774901EBC00000F562709DF846
:10F70000A01001EB410303EB011100F831209DF83B
:10F71000B41001EB410000EB01106D4901EB00104A
:10F7200030309DF8A01000EB0110801C099000788B
:10F7300020F080008030099908709DF8B41001EB2A
:10F74000410000EB0110624901EB0010303000E095
:10F7500022E09DF8A01000EB01108078C0F340007B
:10F7600020B99DF8B4100220FAF7A0FCA2229DF85F
:10F77000B40040F2A11110FB01F0564901EBC000AA
:10F7800000F562709DF8A01001EB410303EB01113D
:10F7900000EBC100827095E09DF8B41001EB4100D0
:10F7A000C0EBC1104C4901EBC000407934287CD13A
:10F7B0009DF8B41001EB410000EB0110444901EB4E
:10F7C000001030309DF8A01000EB0110801C099053
:10F7D000007820F02002099802709DF8B41001EB27
:10F7E000410000EB01103A4901EB001030309DF868
:10F7F000A01000EB0110801C0990007820F002029C
:10F800000998027001229DF8B40040F2A11110FB8A
:10F8100001F0304901EBC00000F562709DF8A010C6
:10F8200001EB410303EB011100EBC10080F846201E
:10F83000A9229DF8B40040F2A11110FB01F0254966
:10F8400001EBC00000F562709DF8A01001EB4103D0
:10F8500003EB011100EBC10082709DF8B41040F27F
:10F86000A11011FB00F01B4901EBC00042799DF88B
:10F87000B40040F2A11110FB01F0164901EBC000E9
:10F8800000F562709DF8A01001EB410303EB01113C
:10F8900000F831209DF8B41001EB410000EB01109D
:10F8A0000B4901EB0010303000E00BE09DF8A01098
:10F8B00000EB0110801C0990007820F0800080305F
:10F8C0000999087000202E902F900021399128E08E
:10F8D0009840002058450020F8870020DDE92E10D0
:10F8E000000140EA11720901CDE92E129DF8B41011
:10F8F00001EB4100C0EBC110FE4901EBC001BDF8B6
:10F90000E400801D085C3038C117DDE92E24104367
:10F9100041EA0402CDE92E02BDF8E400401C80B2A9
:10F920003990BDF8E4000628D8DB9DF8B4002E9984
:10F9300040F2A11210FB02F0EF4A02EBC00202F506
:10F9400062729DF8A00000EB400303EB001002EB95
:10F95000C000C0F81A1000222E922F920021399177
:10F9600022E0DDE92E10000140EA11720901CDE923
:10F970002E129DF8B41001EB4100C0EBC110DD491F
:10F9800001EBC001BDF8E4000D30085C3038C11750
:10F99000DDE92E34184341EA0402CDE92E02BDF818
:10F9A000E400401C80B23990BDF8E4000428D8DBA4
:10F9B0009DF8B4002E9940F2A11210FB02F0CE4A3D
:10F9C00002EBC00202F562729DF8A00000EB40035A
:10F9D00003EB001002EBC000416300222E922F9235
:10F9E0000021399122E0DDE92E10000140EA117278
:10F9F0000901CDE92E129DF8B41001EB4100C0EBD6
:10FA0000C110BC4901EBC001BDF8E4001130085C35
:10FA10003038C117DDE92E34184341EA0402CDE93C
:10FA20002E02BDF8E400401C80B23990BDF8E4001D
:10FA30000628D8DB9DF8B4002E9940F2A11210FBE5
:10FA400002F0AD4A02EBC00202F562729DF8A0001E
:10FA500000EB400303EB001002EBC000C0F81E10E7
:10FA60009DF8B41001EB4100C0EBC110A14901EBBE
:10FA7000C00042799DF8B40040F2A11110FB01F0E2
:10FA80009D4901EBC00101F562719DF8A00000EBFA
:10FA9000400303EB001001EBC000C2709DF8B410EE
:10FAA00001EB410000EB0110944901EB00113031F2
:10FAB0009DF8A00001EB001082789DF8B40040F2A0
:10FAC000A11110FB01F08C4901EBC00101F562713D
:10FAD0009DF8A00000EB400303EB001001EBC00019
:10FAE00002769DF8B41040F2A11011FB00F082499B
:10FAF00001EBC00101F562719DF8A00000EB40022E
:10FB000002EB001011F830109DF8B40040F2A11281
:10FB100010FB02F0784A02EBC000407981427CDAA7
:10FB20009DF8B41040F2A11011FB00F0114601EB5A
:10FB3000C00000F562709DF8A01001EB410202EBDD
:10FB4000011110F831000F2867DD00219DF8B40085
:10FB500040F2A11210FB02F0674A02EBC0000171F3
:10FB6000A7229DF8B40040F2A11110FB01F06249F8
:10FB700001EBC00101F562719DF8A00000EB4003AC
:10FB800003EB001001EBC000427101219DF8B400AD
:10FB900040F2A11210FB02F0574A02EBC0000171C3
:10FBA0009DF8B41040F2A11011FB00F0114601EBDA
:10FBB000C00042799DF8B40040F2A11110FB01F0A1
:10FBC0004D4901EBC00101F562719DF8A00000EB09
:10FBD000400303EB001001F83020A1229DF8B4008F
:10FBE00040F2A11110FB01F0434901EBC00101F506
:10FBF00062719DF8A00000EB400303EB001001EBE5
:10FC0000C00042719DF8B41001EB410000EB0110FF
:10FC10003A4901EB0011303100E071E09DF8A0009D
:10FC200001EB0010801C0990007820F080008030EB
:10FC3000099908709DF8B41001EB410000EB011028
:10FC40002E4901EB001030309DF8A01000EB0110A0
:10FC5000801C0990007820F00400001D09990870AC
:10FC60009DF8B41001EB410000EB0110234901EBBA
:10FC7000001030309DF8A01000EB01108078C0F328
:10FC8000401088B99DF8B41001EB410000EB011061
:10FC90001A4901EB001030309DF8A01000EB011064
:10FCA0008078C0F3400058B39DF8B41001EB4100D8
:10FCB00000EB0110114901EB001030309DF8A0104D
:10FCC00000EB0110801C0990007820F020020998B8
:10FCD00002709DF8B41001EB410000EB01100749E0
:10FCE00001EB001030309DF8A01000EB0110801CDB
:10FCF000099006E0F8870020584500209840002031
:10FD0000C3E0007820F00202099802709DF8B40068
:10FD100000EB400101EB0010FE4901EB0010303018
:10FD20009DF8A01000EB0110801C0990007820F0D5
:10FD300008000830099908709DF8B4009DF8A010DB
:10FD400001EB0010C217CDE92E029DF8B41040F26D
:10FD5000A11011FB00F0F04901EBC00000F562704A
:10FD60009DF8A01001EB410202EB011100EBC10074
:10FD7000223009902E9800EB4001E84800EB41103A
:10FD80000D30102208900999F8F75FFA9DF8B41029
:10FD900040F2A11011FB00F0DF4901EBC00101F5B9
:10FDA00062719DF8A00000EB400202EB001001EB35
:10FDB000C0012E9800EB4002D84800EB421051F8E9
:10FDC0001A2F40F8012F496841609DF8B41001EBEB
:10FDD000410000EB0110CF4901EB001130319DF8DB
:10FDE000A00001EB001001782E9800EB4002CB48F8
:10FDF00000EB421001702E9800EB4001C74800EB69
:10FE00004111C748026841F81D2F808888809DF8FD
:10FE1000B41040F2A11011FB00F0BF4901EBC0018A
:10FE200001F562719DF8A00000EB400202EB0010AA
:10FE300001EBC000416B2E9800EB4002B74800EB8D
:10FE40004210C0F809109DF8B41001EB410000EB1E
:10FE50000110B04901EB001130319DF8A00001EB19
:10FE6000001041682E9800EB4002AC4800EB4210B5
:10FE7000C0F823102E9881B208200991FAF716F9DC
:10FE80009DF8B4100220FAF711F9FCE300202E903F
:10FE90002F900021399122E0DDE92E10000140EA87
:10FEA00011720901CDE92E129DF8B41001EB410049
:10FEB000C0EBC1109B4901EBC001BDF8E4000B3061
:10FEC000085C3038C117DDE92E24104341EA0402F2
:10FED000CDE92E02BDF8E400401C80B23990BDF897
:10FEE000E4000A28D8DB9DF8B400DDE92E1240F2C8
:10FEF000A11310FB03F0884B03EBC00303F56273FF
:10FF00009DF8A00000EB400404EB001003EBC000E0
:10FF100040F8221F426000222E922F920021399138
:10FF200022E0DDE92E10000140EA11720901CDE95D
:10FF30002E129DF8B41001EB4100C0EBC1107949BD
:10FF400001EBC001BDF8E4001530085C3038C11782
:10FF5000DDE92E34184341EA0402CDE92E02BDF852
:10FF6000E400401C80B23990BDF8E4000A28D8DBD8
:10FF70009DF8B400DDE92E2140F2A11310FB03F03F
:10FF8000654B03EBC00303F562739DF8A00000EB23
:10FF9000400404EB001003EBC00022308260C1601B
:10FFA00000219DF8B40040F2A11210FB02F05A4A61
:10FFB00002EBC00001719DF8B40040F2A11110FBEA
:10FFC00001F0114601EBC00000F562709DF8A01031
:10FFD00001EB410202EB011110F831000C2814DC96
:10FFE0000D229DF8B40040F2A11110FB01F04A4926
:10FFF00001EBC00000F562709DF8A01001EB410319
:020000040801F1
:1000000003EB011100F831207FE39DF8B40040F2CA
:10001000A11110FB01F0404901EBC00101F5627133
:100020009DF8A00000EB400202EB001011F8301028
:100030009DF8B40040F2A11210FB02F0364A02EB28
:10004000C00040798142DFD19DF8B4009DF8A01036
:1000500001EB0010C217CDE92E023148F53090F8BF
:10006000E00708B39DF8B40000EB400101EB00107D
:10007000284901EB001030309DF8A01000EB011072
:10008000807A022810D09DF8B40000EB400101EB0B
:100090000010204901EB001030309DF8A01000EB5B
:1000A0000110C07A00287CDD00229DF8B40000EB2E
:1000B000400101EB0010174901EB001030309DF8B2
:1000C000A01000EB0110C2721748D0F80C020521F5
:1000D000B0FBF1F201FB120000EB400112482C30A2
:1000E00000EB41100D3009909DF8B40040F2A111D1
:1000F00010FB01F0084901EBC00000F562709DF8AB
:10010000A01001EB410202EB011100EBC100223013
:1001100010220BE09840002058450020D814002001
:10012000C7310020F8870020BC120020014608904B
:100130000998F8F78AF8FE48D0F80C020521B0FBC0
:10014000F1F201FB120000EB4001F9482C3000EB0A
:1001500041129DF8B40040F2A11110FB01F0F549E5
:1001600001EBC00101F562719DF8A00000EB4003B6
:1001700003EB001001EBC00050F81A1F42F8011FFA
:1001800040685060EA48D0F80C020521B0FBF1F25B
:1001900001FB120000EB4001E5482C3000EB41125E
:1001A00000E094E19DF8B40000EB400101EB001089
:1001B000E14901EB001130319DF8A00001EB001086
:1001C00000781070DA48D0F80C020521B0FBF1F28B
:1001D00001FB120000EB4001D5482C3000EB41122E
:1001E0009DF8B40040F2A11110FB01F0D14901EBE0
:1001F000C00101F562719DF8A00000EB400303EB24
:10020000001001EBC000406BC2F80900C848D0F8EC
:100210000C020521B0FBF1F201FB120000EB4001E2
:10022000C3482C3000EB4111C448026841F81D2F2F
:1002300080888880BE48D0F80C020521B0FBF1F21E
:1002400001FB120000EB4001B9482C3000EB4112D9
:100250009DF8B40000EB400101EB0010B64901EB42
:10026000001130319DF8A00001EB00104068C2F889
:10027000230000229DF8B40000EB400101EB0010C8
:10028000AD4901EB001130319DF8A00001EB0010E9
:1002900042600021399154E0A548D0F80C020521B4
:1002A000B0FBF1F201FB120000EB4001A0482C3042
:1002B00000EB41112731BDF8E4409DF8B40040F255
:1002C000A11210FB02F09B4A02EBC00202F562721F
:1002D0009DF8A00000EB400303EB001002EBC00010
:1002E00090F8800040F2A11210FB02F0914A02EB5C
:1002F000C00202F562729DF8B40040F2A11310FB37
:1003000003F08C4B03EBC00303F562739DF8A00070
:1003100000EB400505EB001003EBC00090F88100F6
:1003200000EB400303EB001002EBC0024732BDF8C4
:10033000E400001D105C0855BDF8E400401C81B2CB
:100340003991BDF8E4000628A6DB0021399142E08E
:1003500000239DF8B40040F2A11110FB01F0754993
:1003600001EBC00101F562719DF8A00000EB4002B5
:1003700002EB001001EBC00090F8800040F2A111E8
:1003800010FB01F06B4901EBC00101F562719DF8B2
:10039000B40040F2A11210FB02F0664A02EBC00268
:1003A00002F562729DF8A00000EB400404EB00101F
:1003B00002EBC00090F8810000EB400202EB00105D
:1003C00001EBC0014731BDF8E4000B54BDF8E40077
:1003D000401C81B23991BDF8E4000A28B8DB5448CA
:1003E000D0F80C020521B0FBF1F080B20146099073
:1003F0000220F8F76DFE00210620F9F757FE4C4861
:10040000D0F80C024A49498D884206D24848D0F8B3
:100410000C02401C4649C1F80C0200210520F9F7E6
:1004200045FE9DF8B40000EB400101EB001042498D
:1004300001EB001030309DF8A01000EB0110801C83
:100440000990007820F00802099802703848D0F826
:100450000C020521B0FBF1F201FB120000EB4001A0
:1004600033482C3000EB4110D0F823202E9800EBBD
:100470004001334800EB4110C0F8232000203990A0
:1004800020E02B48D0F80C020521B0FBF1F201FB73
:10049000120000EB400126482C3000EB41102730C1
:1004A000BDF8E410425C2E9800EB4001244800EBBC
:1004B00041112731BDF8E4000A54BDF8E400401CA6
:1004C00081B23991BDF8E4000628DADB64E09DF8DA
:1004D000B40000EB400101EB0010174901EB0010E4
:1004E00030309DF8A01000EB0110801C09900078BE
:1004F00020F008000830099908709DF8B40000EB5E
:10050000400101EB00100C4901EB001030309DF868
:10051000A01000EB011042682E9800EB4001084843
:1005200000EB4110C0F823200020399030E000009B
:10053000BC1200205845002098400020C731002000
:10054000D81400209DF8B40040F2A11110FB01F076
:10055000FE4901EBC00101F562719DF8A00000EBBE
:10056000400202EB001001EBC0014731BDF8E4008E
:100570000A5C2E9800EB4001F54800EB4111273151
:10058000BDF8E4000A54BDF8E400401C81B2399182
:10059000BDF8E4000628D5DB00229DF8B40040F247
:1005A000A11110FB01F0E94901EBC00101F56271F5
:1005B0009DF8A00000EB400303EB001001EBC0002E
:1005C00080F846209DF8B4100220F9F76FFD9DF8E1
:1005D000B40040F2A11110FB01F0DC4901EBC001B5
:1005E00001F562719DF8A00000EB400202EB0010E3
:1005F00001EBC000223009902E9800EB4001D44856
:1006000000EB41110D3110220891DDE90801F7F7E7
:100610001CFE9DF8B40040F2A11110FB01F0CB4983
:1006200001EBC00101F562719DF8A00000EB4002F2
:1006300002EB001001EBC0012E9800EB4002C44811
:1006400000EB421051F81A2F40F8012F4968416021
:100650009DF8B40000EB400101EB0010BD4901EB37
:10066000001130319DF8A00001EB001001782E98A8
:1006700000EB4002B64800EB421001702E9800EBF0
:100680004001B34800E06BE000EB4111B248026862
:1006900041F81D2F808888809DF8B40040F2A11198
:1006A00010FB01F0A94901EBC00101F562719DF851
:1006B000A00000EB400202EB001001EBC000416B18
:1006C0002E9800EB4002A24800EB4210C0F809103F
:1006D0009DF8B40000EB400101EB00109D4901EBD7
:1006E000001130319DF8A00001EB001041682E98F8
:1006F00000EB4002964800EB4210C0F823102E9801
:1007000081B208200991F9F7D1FCA7229DF8B40025
:1007100040F2A11110FB01F08C4901EBC00101F581
:1007200062719DF8A00000EB400303EB001001EBA9
:10073000C0004271A2229DF8B40040F2A11110FB4A
:1007400001F0824901EBC00000F562709DF8A01035
:1007500001EB410303EB011100EBC100827000BF0C
:1007600000BF0DF055BD9DF8B41001EB4100C0EB8A
:10077000C1107A4911F83000042802D104212591D2
:100780000CE09DF8B41001EB4100C0EBC1107349BF
:1007900011F83000152801D1152125919DF8B410CC
:1007A00001EB4100C0EBC1106C4901EBC000417886
:1007B0009DF8B40000EB4002C2EBC010674A12F88B
:1007C000300041EA002041F23001884202D1A621E6
:1007D00025913DE09DF8B41001EB4100C0EBC11044
:1007E0005E4901EBC00041789DF8B40000EB400287
:1007F000C2EBC010594A12F8300041EA002041F221
:100800003101884202D1A721259121E09DF8B41041
:1008100001EB4100C0EBC110504911F83000022833
:1008200016D19DF8B41001EB4100C0EBC1104B494B
:1008300001EBC00001799DF8B40000EB4002C2EB6F
:10084000C010464A02EBC000C07841EA0021259161
:100850009DF8B41040F2A11011FB00F03B4901EBF0
:10086000C0008178289100213D4A9DF8B40002EB38
:1008700000129DF8A00011543A4890F82800012871
:1008800015D19DF8B41001EB410000EB0110314986
:1008900001EB001030309DF8A01000EB0110801C1F
:1008A0000990007820F08000803009990870BDF828
:1008B0009400A7287ED007DC04287CD015287BD0A4
:1008C000A62841F06D8762E0A0F55850303820B17D
:1008D000112872D01228F4D1FEE39DF8B41040F232
:1008E000A11011FB00F0194901EBC00000F5627086
:1008F0009DF8A01001EB410202EB011110F831004C
:1009000090BB00219DF8B40040F2A11210FB02F050
:100910000E4A02EBC000017101229DF8B40040F2C2
:10092000A11110FB01F0094901EBC00101F5627151
:100930009DF8A00000EB400303EB001001F830200D
:10094000A7229DF8B40040F2A1110EE05845002006
:10095000D814002098400020C7310020F8870020DC
:10096000883E0020BC1200200FE010FB01F0FE4981
:1009700001EBC00000F562709DF8A01001EB41038F
:1009800003EB011100EBC100427101F009BF00212E
:100990009DF8B40040F2A11210FB02F0F24A02EB03
:1009A000C00001719DF8B41040F2A11011FB00F0DD
:1009B000114603E0F9E060E1B0E2E4E201EBC000DF
:1009C00000F562709DF8A01001EB410202EB0111ED
:1009D00010F83100022829DC03229DF8B40040F20F
:1009E000A11110FB01F0E04901EBC00101F56271BA
:1009F0009DF8A00000EB400303EB001001F830204D
:100A0000A9229DF8B40040F2A11110FB01F0D649D3
:100A100001EBC00000F562709DF8A01001EB4103EE
:100A200003EB011100EBC1004271BDE09DF8B41071
:100A300040F2A11011FB00F0CB4901EBC00000F522
:100A400062709DF8A01001EB410202EB011110F859
:100A50003100052829DC06229DF8B40040F2A111DE
:100A600010FB01F0C04901EBC00101F562719DF876
:100A7000A00000EB400303EB001001F83020A2229D
:100A80009DF8B40040F2A11110FB01F0B64901EB52
:100A9000C00000F562709DF8A01001EB410303EB6C
:100AA000011100EBC10042717EE09DF8B41040F2EC
:100AB000A11011FB00F0AC4901EBC00000F5627021
:100AC0009DF8A01001EB410202EB011100EBC10007
:100AD0004079A52815D19DF8B41001EB410000EB39
:100AE0000110A24901EB001030309DF8A01000EB7E
:100AF0000110801C0990007820F00400001D099965
:100B000008709DF8B41040F2A11011FB00F0964956
:100B100001EBC00000F562709DF8A01001EB4102EE
:100B200002EB011100EBC1008078A1283CD09DF8B8
:100B3000B41040F2A11011FB00F08B4901EBC00191
:100B400001F562719DF8A00000EB400202EB00107D
:100B500001EBC00082789DF8B40040F2A11110FBB7
:100B600001F0814901EBC00101F562719DF8A0001F
:100B700000EB400303EB001001EBC0004271A12227
:100B80009DF8B40040F2A11110FB01F0764901EB91
:100B9000C00000F562709DF8A01001EB410303EB6B
:100BA000011100EBC1008270EFE69DF8B41040F235
:100BB000A11011FB00F06C4901EBC00000F5627060
:100BC0009DF8A01001EB410202EB011100EBC10006
:100BD0004079A42830D19DF8B41001EB410000EB1E
:100BE0000110624901EB001030309DF8A01000EBBD
:100BF0000110801C0990007820F020002030099915
:100C0000087000229DF8B40040F2A11110FB01F021
:100C1000554901EBC00000F562709DF8A01001EB92
:100C2000410303EB011100EBC10080F845209DF862
:100C3000B4100220F9F73AFA00219DF8B40040F20E
:100C4000A11210FB02F0484A02EBC0000171A12280
:100C50009DF8B40040F2A11110FB01F0424901EBF4
:100C6000C00000F562709DF8A01001EB410303EB9A
:100C7000011100EBC100427187E69DF8B41040F20B
:100C8000A11011FB00F0384901EBC00000F56270C3
:100C90009DF8A01001EB410202EB011110F83100A8
:100CA000012834DC00219DF8B40040F2A11210FBB1
:100CB00002F02D4A02EBC000017102229DF8B4003F
:100CC00040F2A11110FB01F0274901EBC00101F531
:100CD00062719DF8A00000EB400303EB001001F8E7
:100CE0003020A3229DF8B40040F2A11110FB01F0C6
:100CF0001D4901EBC00000F562709DF8A01001EBEA
:100D0000410303EB011100EBC100427105E19DF8C5
:100D1000B41040F2A11011FB00F0134901EBC00028
:100D200000F562709DF8A01001EB410202EB011189
:100D300010F83100042839DC00219DF8B40040F29D
:100D4000A11210FB02F0084A02EBC000017105225B
:100D50009DF8B40040F2A11110FB01F0024901EB33
:100D6000C00101F5627103E0584500209840002061
:100D70009DF8A00000EB400303EB001001F83020C9
:100D8000A3229DF8B40040F2A11110FB01F0FE492E
:100D900001EBC00000F562709DF8A01001EB41036B
:100DA00003EB011100EBC1004271B6E09DF8B410F5
:100DB00040F2A11011FB00F0F34901EBC00000F577
:100DC00062709DF8A01001EB410202EB011110F8D6
:100DD0003100062815DCA1229DF8B40040F2A111D3
:100DE00010FB01F0E84901EBC00000F562709DF8CE
:100DF000A01001EB410303EB011100EBC1004271B4
:100E00008BE09DF8B41040F2A11011FB00F0DE4918
:100E100001EBC00101F562719DF8A00000EB4002FA
:100E200002EB001011F830109DF8B40040F2A1124E
:100E300010FB02F0D44A02EBC000407981426CD131
:100E40009DF8B41040F2A11011FB00F0114601EB27
:100E5000C00000F562709DF8A01001EB410202EBAA
:100E6000011100EBC1008078A12836D0A3229DF8A3
:100E7000B40040F2A11110FB01F0C34901EBC00125
:100E800001F562719DF8A00000EB400303EB001038
:100E900001EBC00042719DF8B41040F2A11011FBAB
:100EA00000F0B94901EBC00000F562709DF8A01098
:100EB00001EB410202EB011100EBC1008078A22896
:100EC0002BD000209DF8B41040F2A11211FB02F1CA
:100ED000AD4A02EBC10108711FE0A1229DF8B400E8
:100EE00040F2A11110FB01F0A74901EBC00101F58F
:100EF00062719DF8A00000EB400303EB001001EBD2
:100F0000C000427101219DF8B40040F2A11210FB13
:100F100002F09D4A02EBC000017136E5A1229DF866
:100F2000B40040F2A11110FB01F0974901EBC001A0
:100F300001F562719DF8A00000EB400303EB001087
:100F400001EBC00042719DF8B40040F2A11110FB0A
:100F500001F08D4901EBC00101F562719DF8A0001F
:100F600000EB400303EB001001EBC0008270002196
:100F70009DF8B40040F2A11210FB02F0824A02EB8D
:100F8000C000017101E500219DF8B40040F2A112FA
:100F900010FB02F07C4A02EBC0000171A7229DF811
:100FA000B40040F2A11110FB01F0774901EBC00140
:100FB00001F562719DF8A00000EB400303EB001007
:100FC00001EBC00042719DF8B40000EB4001C1EBA1
:100FD000C0106E4901EBC000407930287DD19DF8EA
:100FE000B40040F2A11110FB01F0674901EBC00110
:100FF00001F562719DF8A00000EB400202EB0010C9
:1010000011F830109DF8B40040F2A11210FB02F06C
:101010005D4A02EBC000407981425ED19DF8B40088
:1010200000EB400101EB0010A2F5986101EB00100C
:1010300030309DF8A01000EB0110801C0990007862
:1010400020F00102099802709DF8B40000EB400105
:1010500001EB00104E4901EB001030309DF8A0105C
:1010600000EB0110801C0990007820F00202099822
:1010700002709DF8B40040F2A11110FB01F042494A
:1010800001EBC00000F562709DF8A01001EB410279
:1010900002EB011100EBC100C078312832D19DF87C
:1010A000B40000EB400101EB0010394901EB0010E6
:1010B00030309DF8A01000EB0110801C09900078E2
:1010C00020F020020998027000229DF8B40040F23E
:1010D000A11110FB01F001E0FEE340E02A4901EB21
:1010E000C00000F562709DF8A01001EB410303EB16
:1010F000011100EBC10080F845209DF8B4100220DA
:10110000F8F7D4FF9DF8B40040F2A11110FB01F0F4
:101110001D4901EBC00000F562709DF8A01001EBC5
:10112000410202EB011100EBC10090F846000128DA
:1011300014D1A9229DF8B40040F2A11110FB01F0D6
:10114000114901EBC00000F562709DF8A01001EBA1
:10115000410303EB011100EBC1008270DEE39DF857
:10116000B40000EB4001C1EBC010084901EBC00026
:10117000407931287ED19DF8B40040F2A11110FBD6
:1011800001F0014906E0000058450020F8870020E2
:101190009840002001EBC00101F562719DF8A000AC
:1011A00000EB400202EB001011F830109DF8B40083
:1011B00040F2A11210FB02F0FE4A02EBC00040799F
:1011C000814257D19DF8B40040F2A11110FB01F00B
:1011D000114601EBC00000F562709DF8A01001EB14
:1011E000410202EB011100EBC10090F8460058BB30
:1011F00001229DF8B40040F2A11110FB01F0ED496D
:1012000001EBC00101F562719DF8A00000EB400305
:1012100003EB001001EBC00080F845209DF8B400FE
:1012200000EB400101EB0010E34901EB001130310C
:101230009DF8A00001EB0010801C0990007820F0C0
:101240000100401C099908709DF8B40000EB4001B2
:1012500001EB0010D84901EB001030309DF8A010D0
:1012600000EB0110801C0990007820F00202099820
:10127000027000E00CE2D14890F8E00780B19DF8E0
:10128000B40000EB400101EB0010CB4901EB001072
:1012900030309DF8A01000EB0110807A022878D140
:1012A000C74890F829000128F9D1C548D0F80C02A8
:1012B000C349498D88426CD29DF8B40040F2A11117
:1012C00010FB01F0BB4901EBC00000F562709DF816
:1012D000A01001EB410202EB011100EBC10090F8FC
:1012E0004500012854D19DF8B40040F2A11110FB33
:1012F00001F0B04901EBC00000F562709DF8A0104C
:1013000001EB410202EB011100EBC10090F87F00FC
:10131000F0BB01229DF8B40000EB400101EB00108E
:10132000A54901EB001130319DF8A00001EB001040
:10133000C2724FF010429DF8B40040F2A11110FBB0
:1013400001F09C4901EBC00101F562719DF8A0001C
:1013500000EB400303EB001001EBC00082609DF83E
:10136000B40000EB400101EB0010934901EB0011C8
:1013700030319DF8A00001EB001001789DF8B40019
:1013800040F2A11210FB02F08A4A02EBC00001E019
:1013900070E005E141709DF8B40040F2A11110FB2E
:1013A00001F0114601EBC00101F562719DF8A0004A
:1013B00000EB400202EB001011F830109DF8B40071
:1013C00040F2A11210FB02F07A4A02EBC000407911
:1013D00081423ED100229DF8B40040F2A11110FBE1
:1013E00001F0744901EBC00101F562719DF8A000A4
:1013F00000EB400303EB001001EBC000C271A4221C
:101400009DF8B40040F2A11110FB01F0694901EB15
:10141000C00101F562719DF8A00000EB400303EBF1
:10142000001001EBC0008270A3229DF8B40040F2CE
:10143000A11110FB01F05F4901EBC00000F56270E3
:101440009DF8A01001EB410303EB011100EBC1007B
:10145000427100229DF8B40000EB400101EB001046
:10146000554901EB001030309DF8A01000EB011041
:10147000426053E29DF8B40040F2A11110FB01F06C
:101480004C4901EBC00000F562709DF8A01001EB23
:10149000410202EB011100EBC10090F84500012868
:1014A0007ED19DF8B40040F2A11110FB01F041493A
:1014B00001EBC00101F562719DF8A00000EB400254
:1014C00002EB001001EBC00090F8800040F2A11187
:1014D00010FB01F0374901EBC00101F562719DF885
:1014E000B40040F2A11210FB02F0324A02EBC0003D
:1014F00000F562709DF8A02002EB420303EB02129C
:1015000000EBC20090F8810000EB400202EB0010FB
:1015100001EBC00090F87E00032841D102229DF823
:10152000B40000EB400101EB0010234901EB001176
:1015300030319DF8A00001EB0010C2724FF0104254
:101540009DF8B40040F2A11110FB01F0194901EB24
:10155000C00101F562719DF8A00000EB400303EBB0
:10156000001001EBC00082609DF8B40000EB400168
:1015700001EB0010104901EB001130319DF8A00083
:1015800001EB001001789DF8B40040F2A11210FBAD
:1015900002F0084A02EBC00041709DF8B40000E080
:1015A0009BE140F2A11110FB01F0114601EBC001DB
:1015B00008E000005845002098400020BC32002080
:1015C000BC12002001F562719DF8A00000EB400202
:1015D00002EB001011F830109DF8B40040F2A11297
:1015E00010FB02F0FE4A02EBC000407981423ED17E
:1015F00000229DF8B40040F2A11110FB01F0F8495F
:1016000001EBC00101F562719DF8A00000EB400301
:1016100003EB001001EBC000C271A4229DF8B400DE
:1016200040F2A11110FB01F0ED4901EBC00101F501
:1016300062719DF8A00000EB400303EB001001EB8A
:10164000C0008270A3229DF8B40040F2A11110FBEB
:1016500001F0E34901EBC00000F562709DF8A010B5
:1016600001EB410303EB011100EBC10042710022C9
:101670009DF8B40000EB400101EB0010D94901EBEB
:10168000001030309DF8A01000EB0110426045E1E1
:101690009DF8B41001EB4100C0EBC110D24901EB41
:1016A000C000407933287DD19DF8B40000EB4001A3
:1016B00001EB0010CB4901EB001030309DF8A01079
:1016C00000EB0110801C0990007820F00100401C04
:1016D000099908709DF8B40000EB400101EB00107F
:1016E000C04901EB001030309DF8A01000EB011054
:1016F000801C0990007820F02002099802709DF863
:10170000B40000EB400101EB0010B64901EB001002
:1017100030309DF8A01000EB0110801C099000787B
:1017200020F00200801C099908709DF8B40040F276
:10173000A11110FB01F0AA4901EBC00042799DF80C
:10174000B40040F2A11110FB01F0A54901EBC0006B
:1017500000F562709DF8A01001EB410303EB01114D
:1017600000F831209DF8B41001EB410000EB0110AE
:101770009C4901EB001030309DF8A01000EB0110E7
:10178000801C0990007820F0800080300999087052
:101790009DF8B41001EB410000EB0110914901EB01
:1017A000001000E023E030309DF8A01000EB0110A5
:1017B0008078C0F3400020B99DF8B4100220F8F7FB
:1017C00075FCA2229DF8B40040F2A11110FB01F0BB
:1017D000834901EBC00000F562709DF8A01001EB99
:1017E000410303EB011100EBC100827096E09DF80C
:1017F000B41001EB4100C0EBC1107B4901EBC0000C
:101800004079342869D19DF8B41001EB410000EB18
:101810000110744901EB001030309DF8A01000EB6E
:101820000110801C0990007820F0200209980270B5
:101830009DF8B41001EB410000EB0110694901EB88
:10184000001030309DF8A01000EB0110801C0990B2
:10185000007820F002020998027001229DF8B4007D
:1018600040F2A11110FB01F05D4901EBC00000F551
:1018700062709DF8A01001EB410303EB011100EB36
:10188000C10080F84620A9229DF8B40040F2A111C1
:1018900010FB01F0524901EBC00000F562709DF8A9
:1018A000A01001EB410303EB011100EBC1008270BA
:1018B0009DF8B41040F2A11011FB00F0484901EB73
:1018C000C00042799DF8B40040F2A11110FB01F074
:1018D000434901EBC00001E0E3E21FE000F5627064
:1018E0009DF8A01001EB410303EB011100F831203A
:1018F0009DF8B41001EB410000EB0110394901EBF8
:10190000001030309DF8A01000EB0110801C0990F1
:10191000007820F0800080300999087000202E9017
:101920002F900021399122E0DDE92E10000140EADC
:1019300011720901CDE92E129DF8B41001EB41009E
:10194000C0EBC110284901EBC001BDF8E400801DC7
:10195000085C3038C117DDE92E34184341EA04022F
:10196000CDE92E02BDF8E400401C80B23990BDF8EC
:10197000E4000828D8DB9DF8B4002E9940F2A112AB
:1019800010FB02F0164A02EBC00202F562729DF8EB
:10199000A00000EB400303EB001002EBC000C0F816
:1019A0001A1000222E922F92002139912AE0DDE9AF
:1019B0002E10000140EA11720901CDE92E129DF8A6
:1019C000B41001EB4100C0EBC110074901EBC001AD
:1019D000BDF8E4000F30085C3038C11706E00000A5
:1019E0005845002098400020F8870020DDE92E347B
:1019F000184341EA0402CDE92E02BDF8E400401C80
:101A000080B23990BDF8E4000628D0DB9DF8B40020
:101A10002E9940F2A11210FB02F0FE4A02EBC00226
:101A200002F562729DF8A00000EB400303EB00108A
:101A300002EBC000416300222E922F9200213991C7
:101A400022E0DDE92E10000140EA11720901CDE922
:101A50002E129DF8B41001EB4100C0EBC110EE490D
:101A600001EBC001BDF8E4001530085C3038C11747
:101A7000DDE92E3440EA03022143CDE92E21BDF8F1
:101A8000E400401C81B23991BDF8E4000828D8DB9D
:101A90009DF8B4002E9940F2A11210FB02F0DD4A2D
:101AA00002EBC00202F562729DF8A00000EB400359
:101AB00003EB001002EBC000C0F81E109DF8B4103C
:101AC00001EB4100C0EBC110D34901EBC0004279EA
:101AD0009DF8B40040F2A11110FB01F0CD4901EBDB
:101AE000C00101F562719DF8A00000EB400303EB1B
:101AF000001001EBC000C2709DF8B41001EB410072
:101B000000EB0110C54901EB001130319DF8A00038
:101B100001EB001082789DF8B40040F2A11110FB97
:101B200001F0BC4901EBC00101F562719DF8A00014
:101B300000EB400303EB001001EBC00002769DF8C0
:101B4000B41040F2A11011FB00F0B24901EBC0014A
:101B500001F562719DF8A00000EB400202EB00105D
:101B600011F830109DF8B40040F2A11210FB02F001
:101B7000A84A02EBC000407981427DDA00219DF83D
:101B8000B40040F2A11210FB02F0A24A02EBC00026
:101B90000171A7229DF8B40040F2A11110FB01F0E1
:101BA0009C4901EBC00101F562719DF8A00000EBBA
:101BB000400303EB001001EBC000427101219DF8CE
:101BC000B40040F2A11210FB02F0924A02EBC000F6
:101BD00001719DF8B41040F2A11011FB00F0114604
:101BE00001EBC00042799DF8B40040F2A11110FB56
:101BF00001F0884901EBC00101F562719DF8A00078
:101C000000EB400303EB001001F83020A1229DF807
:101C1000B40040F2A11110FB01F07E4901EBC001BC
:101C200001F562719DF8A00000EB400303EB00108A
:101C300001EBC00042719DF8B41001EB410000EBD4
:101C40000110764901EB001130319DF8A00001EB45
:101C50000010801C0990007820F0800080300999E5
:101C600008709DF8B41001EB410000EB01106B49C6
:101C700001EB0010303000E05BE09DF8A01000EBBD
:101C80000110801C0990007820F00400001D0999C3
:101C900008709DF8B41001EB410000EB01105F49A2
:101CA00001EB001030309DF8A01000EB011080789F
:101CB000C0F34010E8B39DF8B41001EB410000EB15
:101CC0000110564901EB001030309DF8A01000EBD8
:101CD0000110801C0990007820F020020998027001
:101CE0009DF8B41001EB410000EB01104B4901EBF2
:101CF000001030309DF8A01000EB01108078C0F388
:101D00004000E8BB9DF8B41001EB410000EB01106E
:101D1000424901EB001030309DF8A01000EB01109B
:101D2000801C0990007820F00801083109980170A2
:101D300000E0B5E09DF8B4109DF8A00000EB0110A4
:101D4000C217CDE92E029DF8B41040F2A11011FB8C
:101D500000F0304901EBC00000F562709DF8A01062
:101D600001EB410202EB011100EBC10022300990AE
:101D70002E9800EB40012A4800EB41100D3000E0A6
:101D800089E0102208900999F6F75FFA9DF8B410DF
:101D900040F2A11011FB00F01E4901EBC00101F55A
:101DA00062719DF8A00000EB400202EB001001EB15
:101DB000C0012E9800EB4002194800EB421051F888
:101DC0001A2F40F8012F496841609DF8B41001EBCB
:101DD000410000EB0110114901EB001130319DF879
:101DE000A00001EB001001782E9800EB40020C4897
:101DF00000EB421001702E9800EB4001084800EB08
:101E000041110848026841F81D2F808888809DF89C
:101E1000B41009E058450020F887002098400020C1
:101E2000D8140020C731002040F2A11011FB00F0AF
:101E3000FE4901EBC00101F562719DF8A00000EBC5
:101E4000400202EB001001EBC000416B2E9800EB4A
:101E50004002F74800EB4210C0F809109DF8B4109A
:101E600001EB410000EB0110F24901EB00113031B0
:101E70009DF8A00001EB001041682E9800EB400295
:101E8000EB4800EB4210C0F823102E9881B20820D6
:101E90000991F8F70BF99DF8B4100220F8F706F94C
:101EA000FEE300202E902F900021399122E0DDE901
:101EB0002E10000140EA11720901CDE92E129DF8A1
:101EC000B41001EB4100C0EBC110DB4901EBC001D4
:101ED000BDF8E4000B30085C3038C117DDE92E3462
:101EE000184341EA0402CDE92E02BDF8E400401C8B
:101EF00080B23990BDF8E4000C28D8DB9DF8B4001E
:101F0000DDE92E1240F2A11310FB03F0C74B03EBE7
:101F1000C00303F562739DF8A00000EB400404EBDE
:101F2000001003EBC00040F8221F426000222E92F6
:101F30002F920021399122E0DDE92E10000140EAC4
:101F400011720901CDE92E129DF8B41001EB410088
:101F5000C0EBC110B84901EBC001BDF8E400173077
:101F6000085C3038C117DDE92E34184341EA040219
:101F7000CDE92E02BDF8E400401C80B23990BDF8D6
:101F8000E4000C28D8DB9DF8B400DDE92E1240F205
:101F9000A11310FB03F0A54B03EBC00303F5627321
:101FA0009DF8A00000EB400404EB001003EBC00020
:101FB00022308160C26000219DF8B40040F2A1127D
:101FC00010FB02F0994A02EBC00001719DF8B410B9
:101FD00040F2A11011FB00F0114601EBC00000F52A
:101FE00062709DF8A01001EB410202EB011110F8A4
:101FF0003100032814DC04229DF8B40040F2A11142
:1020000010FB01F0894901EBC00000F562709DF8FA
:10201000A01001EB410303EB011100F831207EE336
:102020009DF8B41040F2A11011FB00F07F4901EBC4
:10203000C00101F562719DF8A00000EB400202EBC7
:10204000001011F830109DF8B40040F2A11210FBFE
:1020500002F0764A02EBC00040798142DFD19DF860
:10206000B4009DF8A01001EB0010C217CDE92E02BC
:10207000724890F8E00708B39DF8B41001EB4100F6
:1020800000EB01106B4901EB001030309DF8A010FF
:1020900000EB0110807A022810D09DF8B41001EBFB
:1020A000410000EB0110634901EB001030309DF856
:1020B000A01000EB0110C07A00287DDD00229DF801
:1020C000B40000EB400101EB00105A4901EB001095
:1020D00030309DF8A01000EB0110C2725848D0F8C3
:1020E0000C020521B0FBF1F201FB120000EB4001F4
:1020F00053482C3000EB41100D3009909DF8B4008E
:1021000040F2A11110FB01F0484901EBC00000F5BD
:1021100062709DF8A01001EB410202EB011100EB8F
:10212000C10022301022014608900998F6F78DF878
:102130004348D0F80C020521B0FBF1F201FB12007C
:1021400000EB40013E482C3000EB41129DF8B400FA
:1021500040F2A11110FB01F0344901EBC00101F57F
:1021600062719DF8A00000EB400303EB001001EB4F
:10217000C00050F81A1F42F8011F406850603048F4
:10218000D0F80C020521B0FBF1F201FB120000EBCC
:1021900040012B482C3000EB41129DF8B40000EBBD
:1021A000400101EB0010234901EB001130319DF893
:1021B000A00001EB001000E095E1007810702048CD
:1021C000D0F80C020521B0FBF1F201FB120000EB8C
:1021D00040011B482C3000EB41129DF8B40040F246
:1021E000A11110FB01F0114901EBC00101F5627171
:1021F0009DF8A00000EB400303EB001001EBC000D2
:10220000406BC2F809000E48D0F80C020521B0FB63
:10221000F1F201FB120000EB400109482C3000EB09
:1022200041110648F53802680CE0000058450020CE
:10223000D814002098400020F8870020BC320020ED
:10224000BC12002041F81D2F80888880FE48D0F8FD
:102250000C020521B0FBF1F201FB120000EB400182
:10226000F9482C3000EB41129DF8B40000EB40011E
:1022700001EB0010F54901EB001130319DF8A00091
:1022800001EB00104068C2F8230000229DF8B40062
:1022900000EB400101EB0010EC4901EB0011303183
:1022A0009DF8A00001EB001042600021399154E03C
:1022B000E548D0F80C020521B0FBF1F201FB120059
:1022C00000EB4001E0482C3000EB41112731BDF814
:1022D000E4409DF8B40040F2A11210FB02F0DC4A89
:1022E00002EBC00202F562729DF8A00000EB400311
:1022F00003EB001002EBC00090F8800040F2A11246
:1023000010FB02F0D24A02EBC00202F562729DF8A5
:10231000B40040F2A11310FB03F0CD4B03EBC0035C
:1023200003F562739DF8A00000EB400505EB00107B
:1023300003EBC00090F8810000EB400303EB0010BA
:1023400002EBC0024732BDF8E400001D105C0855E6
:10235000BDF8E400401C81B23991BDF8E4000628C4
:10236000A6DB0021399142E000239DF8B40040F241
:10237000A11110FB01F0B64901EBC00101F562713A
:102380009DF8A00000EB400202EB001001EBC00042
:1023900090F8800040F2A11110FB01F0AC4901EB74
:1023A000C00101F562719DF8B40040F2A11210FB6A
:1023B00002F0A74A02EBC00202F562729DF8A0008B
:1023C00000EB400404EB001002EBC00090F8810029
:1023D00000EB400202EB001001EBC0014731BDF8F9
:1023E000E4000B54BDF8E400401C81B23991BDF803
:1023F000E4000A28B8DB9448D0F80C020521B0FBB1
:10240000F1F080B2014609900220F6F761FE00214A
:102410000620F7F74BFE8C48D0F80C028A49498D0C
:10242000884206D28848D0F80C02401C8649C1F880
:102430000C0200210520F7F739FE9DF8B41001EBDE
:10244000410000EB0110814901EB001030309DF894
:10245000A01000EB0110801C0990007820F0080209
:10246000099802707848D0F80C020521B0FBF1F20F
:1024700001FB120000EB400173482C3000EB4110CF
:10248000D0F823202E9800EB4001724800EB411059
:10249000C0F823200020399020E06B48D0F80C02CF
:1024A0000521B0FBF1F201FB120000EB4001664890
:1024B0002C3000EB41102730BDF8E410425C2E9820
:1024C00000EB4001634800EB41112731BDF8E40007
:1024D0000A54BDF8E400401C81B23991BDF8E40013
:1024E0000628DADB59E09DF8B41001EB410000EB5F
:1024F0000110564901EB001030309DF8A01000EBA0
:102500000110801C0990007820F00800083009991B
:1025100008709DF8B41001EB410000EB01104B492D
:1025200001EB001030309DF8A01000EB0110426864
:102530002E9800EB4001474800EB4110C0F82320E3
:102540000020399025E09DF8B41040F2A11011FB55
:1025500000F03F4901EBC00101F562719DF8A00058
:1025600000EB400202EB001001EBC0014731BDF867
:10257000E4000A5C2E9800EB4001364800EB411164
:102580002731BDF8E4000A54BDF8E400401C81B2D4
:102590003991BDF8E4000628D5DB00229DF8B4008F
:1025A00040F2A11110FB01F0294901EBC00101F536
:1025B00062719DF8A00000EB400303EB001001EBFB
:1025C000C00080F846209DF8B4100220F7F76EFD99
:1025D0009DF8B40040F2A11110FB01F01C4901EB81
:1025E000C00101F562719DF8A00000EB400202EB12
:1025F000001001EBC000223009902E9800EB400142
:10260000144800EB41110D3110220891DDE9080159
:10261000F5F71BFE9DF8B41040F2A11011FB00F07D
:102620000B4901EBC00101F562719DF8A00000EBC0
:10263000400202EB001001EBC0012E9800EB4002BB
:10264000044800EB421007E0BC1200209840002034
:1026500058450020D814002051F81A2F40F8012FB7
:10266000496841609DF8B41001EB410000EB011096
:10267000F94901EB001130319DF8A00001EB001089
:1026800001782E9800EB4002F44800EB42100170F4
:102690002E9800EB4001F14800EB4111F04800E0BA
:1026A0007EE0026841F81D2F808888809DF8B41074
:1026B00040F2A11011FB00F0EA4901EBC00101F565
:1026C00062719DF8A00000EB400202EB001001EBEC
:1026D000C000416B2E9800EB4002E04800EB421036
:1026E000C0F809109DF8B41001EB410000EB011097
:1026F000D94901EB001130319DF8A00001EB001029
:1027000041682E9800EB4002D44800EB4210C0F81C
:1027100023102E9881B208200991F7F7C7FC0022F8
:102720009DF8B40040F2A11110FB01F0CD4901EB7E
:10273000C00101F562719DF8A00000EB400303EBBE
:10274000001001EBC00080F84620A7229DF8B400DD
:1027500040F2A11110FB01F0C24901EBC00101F5EB
:1027600062719DF8A00000EB400303EB001001EB49
:10277000C0004271A2229DF8B40040F2A11110FBEA
:1027800001F0B84901EBC00000F562709DF8A0109F
:1027900001EB410303EB011100EBC100827000BFAC
:1027A00000BF0BF035BD0021AF4A9DF8B40002EB2D
:1027B00000129DF8A00011549DF8B41001EB4100E7
:1027C000C0EBC110A94901EBC000407870280ED1C0
:1027D0009DF8B41001EB4100C0EBC110A34901EB1F
:1027E000C0008078FA2802D1B121259142E09DF8FD
:1027F000B41001EB4100C0EBC1109C4901EBC000DB
:10280000407800F0F000C0280ED19DF8B41001EB24
:102810004100C0EBC110954901EBC0008078FA2857
:1028200002D1B621259125E09DF8B41001EB4100BD
:10283000C0EBC1108D4911F8300000F0F0005028B5
:1028400018D19DF8B41001EB4100C0EBC1108749CD
:1028500001EBC000407800F0F00030280AD19DF86C
:10286000B41001EB4100C0EBC110804901EBC00086
:10287000817825919DF8B41040F2A11011FB00F071
:10288000784901EBC000817828910021764A9DF8B3
:10289000B40002EB00129DF8A0001154744890F8A7
:1028A0002800012815D19DF8B41001EB410000EB80
:1028B0000110694901EB001030309DF8A01000EBC9
:1028C0000110801C0990007820F080008030099968
:1028D0000870BDF89400652874D004DC012809D084
:1028E000032805D17FE0B12802D0B62800D100E04E
:1028F0008BE18AE19DF8B41001EB4100C0EBC110FF
:102900005A4901EBC0000079012806D0022805D001
:10291000032804D0052864D102E062E061E060E0B1
:102920009DF8B41040F2A11011FB00F04D4901EBED
:10293000C00000F562709DF8A01001EB410202EBAF
:10294000011110F83100E0BB00219DF8B40040F205
:10295000A11210FB02F0434A02EBC00001710122F8
:102960009DF8B40040F2A11110FB01F03D4901EBCC
:10297000C00101F562719DF8A00000EB400303EB7C
:10298000001001F83020B6229DF8B40040F2A111E9
:1029900010FB01F0334901EBC00101F562719DF8B4
:1029A000A00000EB400303EB001001EBC0004271FC
:1029B000B2229DF8B40040F2A11110FB01F02949A8
:1029C00001E00DE037E001EBC00000F562709DF81A
:1029D000A01001EB410303EB011100EBC100827079
:1029E00000BF00BF11E19DF8B41001EB4100C0EB46
:1029F000C1101E4901EBC000C1791E4880F8031DBB
:102A00009DF8B41001EB410000EB0110124901EBFD
:102A1000001130319DF8A00001EB0010801C0990DE
:102A2000144890F8030DC2080998007862F300007A
:102A300009990870E9E09DF8B41001EB4100C0EB82
:102A4000C1100A4901EBC000007900F0F00098B90C
:102A5000B821259112E0000098400020D8140020F1
:102A6000C731002058450020883E0020F88700200C
:102A7000BC120020BC220020B921259100213991EF
:102A800020E09DF8B41001EB410000EB0110FE497D
:102A900001EB00113031BDF8E40001EB001041788A
:102AA0009DF8B40000EB4002C2EBC010F74A12F8E8
:102AB00030005038814200D112E0BDF8E400401CE3
:102AC00081B239919DF8B41001EB410000EB011087
:102AD000ED4901EB0010C179BDF8E4008142D0DC82
:102AE00000BF9DF8B41040F2A11011FB00F0E849BE
:102AF00001EBC00000F562709DF8A01001EB4102EF
:102B000002EB011110F83100012834D100219DF8A9
:102B1000B40040F2A11210FB02F0DD4A02EBC0004B
:102B2000017102229DF8B40040F2A11110FB01F0E6
:102B3000D74901EBC00101F562719DF8A00000EBDF
:102B4000400303EB001001F83020B9229DF8B400D7
:102B500040F2A11110FB01F0CD4901EBC00000F5DE
:102B600062709DF8A01001EB410303EB011100EB33
:102B7000C100427148E09DF8B41040F2A11011FB71
:102B800000F0C34901EBC00000F562709DF8A01091
:102B900001EB410202EB011110F83100012833D1A1
:102BA00000219DF8B40040F2A11210FB02F0B84AD7
:102BB00002EBC000017102229DF8B40040F2A111A5
:102BC00010FB01F0B24901EBC00101F562719DF803
:102BD000A00000EB400303EB001001F83020B92205
:102BE0009DF8B40040F2A11110FB01F0A84901EBDF
:102BF000C00000F562709DF8A01001EB410303EBEB
:102C0000011100EBC100427100BF00BFC9E59DF892
:102C1000B40000EB400101EB00109B4901EB0010F8
:102C2000007B20B101287CD002287BD1ECE29949BD
:102C30009DF8B40031F81000801F81B209919DF811
:102C4000B40000EB4001C1EBC010904901EBC000A3
:102C5000401C08900999F6F777FE0022CDE9300272
:102C60009DF8B40000EB4001C1EBC010874901EBB7
:102C7000C00288489DF8B41030F81100401F1118A8
:102C80000991042109981FF04DF9C217CDE92E02D0
:102C90002FA819C82E995940604001437ED17E4A21
:102CA0009DF8B40002EB001001709DF8B40000EB39
:102CB0004001C1EBC010754901EBC00001792591BD
:102CC000BDF89400312802D0452868D1FBE0714856
:102CD0009DF8B41030F811001838412190FBF1F044
:102CE000C217C1B2CDE92E026C4880F8AC100020AA
:102CF0003990DEE09DF8B40000EB4001C1EBC0105C
:102D0000624901EBC001BDF8E40000EB8010143013
:102D1000095C624AAD32BDF8E40011549DF8B4007C
:102D200001E0D3E06FE200EB4001C1EBC010574976
:102D300001EBC001BDF8E40000EB80101A30014443
:102D40000991082109981FF0ABF88DED0E0A534A3E
:102D5000B932BDF8E4000E9902EB001041609DF815
:102D6000B40000EB4001C1EBC010484901EBC001C9
:102D7000BDF8E40000EB80103230014409910821D5
:102D800009981FF08DF88DED0E0A444AB932BDF84E
:102D9000E4000E9902EB0010016001E095E093E081
:102DA0009DF8B40000EB4001C1EBC010374901EBC6
:102DB000C001BDF8E40000EB80103A3001440991F5
:102DC000082109981FF06CF88DED0E0A334AB932CC
:102DD000BDF8E4000E9902EB001081609DF8B4008C
:102DE00000EB4001C1EBC010284901EBC001BDF868
:102DF000E40000EB80104230014409910821099859
:102E00001FF04EF88DED0E0A244AB932BDF8E400E9
:102E10000E9902EB0010C1609DF8B40000EB400178
:102E200001EB0010184901EB00113031BDF8E4004E
:102E300001EB0010801C0990007820F080008030A9
:102E4000099908709DF8B40000EB4001C1EBC01077
:102E50000E4901EBC0010F4A9DF8B40032F8100092
:102E6000401E0A5C9DF8B40040F2A11110FB01F075
:102E7000074901EBC00101F562719DF8A00000EB6C
:102E8000400303EB00100BE098400020F88700207F
:102E90005845002078790020883E0020BC32002070
:102EA00001EBC00080F84420BDF8E400401C81B272
:102EB0003991BDF8E4000021DDE92E34C01AA141AA
:102EC000FFF618AF00E000BF00BFB4E29DF8B40009
:102ED00000EB4001C1EBC010FE4901EBC000407D9A
:102EE0009DF8B41001EB4102C2EBC111F94A02EBAB
:102EF000C101897D40EA0120C217CDE92E029DF86B
:102F0000B40000EB4001C1EBC010F24901EBC0017D
:102F1000099115210998F6F7FBFC0022CDE9300252
:102F2000DDE93042DDE92E106140504001437CD1A3
:102F30009DF8B40000EB4001C1EBC010E54911F869
:102F40003000401EC1B228910021E34A9DF8B40030
:102F500002EB00129DF8A0001154E04A9DF8A00079
:102F600011549FEDDF0A10EE101A0C329DF8A000EC
:102F700002EB001041609DF8B40000EB4001C1EB92
:102F8000C010D44901EBC00081799DF8B40000EB7A
:102F90004002C2EBC010CF4A02EBC000407941EAC8
:102FA000002000EE100AB8EEC00A9FEDCE1AC0EE67
:102FB000010A9DF8B40000EB4001C1EBC0101146BE
:102FC00001EBC00001799DF8B40000EB4002C2EBB8
:102FD000C010C04A02EBC000C07841EA002000EEF9
:102FE000100AB8EEC00A30EE800A10EE101ABB4A82
:102FF0000C329DF8A00002EB001001609DF8B400B7
:1030000000EB4001C1EBC010B24901EBC000817A76
:103010009DF8B40000EB4002C2EBC010AD4A02EBD9
:10302000C000407A41EA002000E0ECE000EE100A27
:10303000B8EEC00A9FEDAB1AC0EE010A9DF8B400CD
:1030400000EB4001C1EBC010114601EBC000017A5A
:103050009DF8B40000EB4002C2EBC0109D4A02EBA9
:10306000C000C07941EA002000EE100AB8EEC00AA4
:1030700030EE800A10EE101A984A0C329DF8A0002B
:1030800002EB001081609DF8B40000EB4001C1EB41
:10309000C010904901EBC000C07A00F0800038BB3E
:1030A0009DF8B40000EB4001C1EBC010894901EB71
:1030B000C000017B9DF8B40000EB4002C2EBC010E1
:1030C000844A02EBC000C07A41EA002000EE100AF8
:1030D000F8EEC00AB3EE001A80EE810A10EE100A74
:1030E0007E4A0C329DF8A01002EB0111C86047E047
:1030F0009DF8B40000EB4001C1EBC010754901EB35
:10310000C000017B9DF8B40000EB4002C2EBC01090
:10311000704A02EBC000C07A41EA0020404280B20F
:1031200000EE100AB8EEC00A8DED030A0398F5F719
:10313000F5FA9FED6D0B53EC102BCDE904019DEDDD
:10314000040B51EC100BF5F7CDF99FED690B53EC27
:10315000102BCDE906019DED060B51EC100BF5F798
:103160004CF9CDE908019DED080B51EC100BF5F77A
:10317000E8FA5A4A0C329DF8A01002EB0111C8601F
:103180009DF8B40000EB400101EB00105A4901EB3F
:10319000001030309DF8A01000EB0110801C099049
:1031A000007820F080008030099908709DF8B410F4
:1031B00001EB4100C0EBC110464901EBC000C27DEC
:1031C0009DF8B40040F2A11110FB01F04B4901EB56
:1031D000C00000F562709DF8A01001EB410303EB05
:1031E000011100EBC10080F844209DF8B41001EB00
:1031F000410000EB0110404901EB0010C179374854
:10320000AD3880F8AC1016E19DF8B41001EB410028
:10321000C0EBC1102F4901EBC000C0799DF8B4107C
:1032200001EB4102C2EBC1112A4A02EBC101097A4A
:1032300040EA0120C217CDE92E029DF8B41001EB3F
:103240004100C0EBC110234901EBC00109910721E6
:103250000998F6F75DFB0022CDE930022FA819C8C6
:103260002E995940604001437ED19DF8B41001EB86
:103270004100C0EBC110174911F83000401EC1B227
:1032800028910021144A9DF8B40002EB001001704F
:10329000124A9DF8A00011549DF8B41001EB4100B2
:1032A000C0EBC1100B4901EBC000817908460191C8
:1032B000F5F7AEF9CDE902019DED021B9FED100B74
:1032C00022F0D6FC8DED060B9DF8B41001EB410009
:1032D0001AE00000F8870020883E002069330020B3
:1032E0000000000000FF7F470000000000003040A9
:1032F0000000000000000000984000205845002019
:103300000000000000002440C0EBC110F64901EBB2
:10331000C00001799DF8B40000EB4002C2EBC01080
:10332000F14A02EBC000C07841EA002000EE100A2A
:10333000B8EEC00A8DED030A0398F5F7EFF9CDE971
:1033400004019DED060B53EC102B9DED040B51EC8D
:10335000100BF5F7C7F8CDE908019DED080B51EC0E
:10336000100BF5F7EEF900E064E0E04A9DF8A010DC
:1033700002EB011148601FED260A10EE100A9DF8BD
:10338000A01002EB011108601FED2B0A10EE100ACD
:103390009DF8A01002EB011188601FED2F0A10EEBE
:1033A000100A9DF8A01002EB0111C8609DF8B4103E
:1033B00001EB410000EB011002F6235101EB00107C
:1033C00030309DF8A01000EB0110801C09900078AF
:1033D00020F080008030099908709DF8B41001EB4E
:1033E0004100C0EBC110C04901EBC000427A9DF81A
:1033F000B40040F2A11110FB01F0BD4901EBC00087
:1034000000F562709DF8A01001EB410303EB011180
:1034100000EBC10080F844209DF8B41001EB41009E
:1034200000EB0110B34901EB0010C179AF48B93886
:1034300080F8AC1000BF00BF0AF0EABE9DF8B410DF
:1034400001EB4100C0EBC110A74901EBC000C178FE
:103450009DF8B40000EB4002C2EBC010A24A02EBA0
:10346000C000807841EA002129919DF8B41001EB59
:103470004100C0EBC110114601EBC001BDF8A40032
:10348000401C095C9DF8B40000EB4002C2EBC01088
:10349000954A02EBC002BDF8A400105C41EA00208E
:1034A000C217CDE92E029DF8B41001EB4100C0EB2C
:1034B000C1108D4901EBC0000990BDF8A410F6F7CA
:1034C00027FA0022CDE93002DDE93042DDE92E1095
:1034D00061405040014341F067869DF8B41001EB14
:1034E0004100C0EBC110804901EBC0004178289138
:1034F000002139911CE09DF8B41001EB410000EB74
:1035000001107C4901EB00113031BDF8E40001EB02
:10351000001041789DF8A000814204D1BDF8E4007C
:10352000C1B2289112E0BDF8E400401C81B239918B
:103530009DF8B41001EB410000EB01106D4901EB67
:103540000010C179BDF8E4008142D4DC00BF9DF8D1
:10355000B41001EB410000EB0110664901EB0010D3
:1035600030309DF8A01000EB0110801C099000780D
:1035700020F080008030099908709DF8B41001EBAC
:103580004100C0EBC110584901EBC0000079259003
:103590000020594A9DF8B41002EB01129DF8A010CA
:1035A0005054BDF89400F3287DD009DC05287BD069
:1035B00006280ED0F12878D0F22841F0F485F7E300
:1035C000F42873D0F62872D0F72871D0F828F4D1F7
:1035D000EFE30621109100213691EBE3BDF84000A6
:1035E000401C81B210919DF8B41001EB4100C0EB7A
:1035F000C1103D4901EBC001BDF84000095C2591B7
:10360000BDF84000401C81B21091BDF89400F12833
:1036100004D0F22872D0F32871D1FDE39DF8B410E4
:1036200001EB4100C0EBC1102F4901EBC001BDF817
:103630004000095C2991BDF84000401C81B2109106
:103640009DF8B41001EB410000EB0110294901EB9A
:10365000001130319DF8A020BDF8D800104401EBD6
:103660000010407A00F00100E8B39DF8B41040F279
:10367000A11011FB00F01E4901EBC00101F56271C0
:103680009DF8A020BDF8D800104400EB400202EBEA
:10369000001001EBC00090F8900000F0010010BB9A
:1036A0009DF8B41005E0FDE3FDE3FDE3FDE3FDE37C
:1036B000FDE340F2A11011FB00F00D4901EBC00148
:1036C00001F562719DF8A020BDF8D800104400EB10
:1036D000400202EB001001EBC00090F8820010B134
:1036E000002139913CE09EE0F887002075330020EE
:1036F0005845002098400020883E0020FCE3FAE373
:103700009DF8B41040F2A11011FB00F0FC4901EB50
:10371000C00101F562719DF8A020BDF8D8001044E9
:1037200000EB400202EB001001EBC00000F183014E
:10373000BDF8E4000A5C9DF8B40000EB400101EB29
:103740000010F04901EB00100E30BDF8E410405CB1
:10375000824200D008E0BDF8E400401C81B23991FB
:10376000BDF8E4000428CBDB00BFBDF8E40004286A
:1037700059D1042139912FE09DF8B41040F2A110E5
:1037800011FB00F0DE4901EBC00101F562719DF80B
:10379000A020BDF8D800104400EB400202EB00105E
:1037A00001EBC00000F18301BDF8E4000A5C9DF864
:1037B000B40000EB400101EB0010D24901EB001016
:1037C0000E30BDF8E410405C824200D008E0BDF845
:1037D000E400401C81B23991BDF8E4000A28CBDB3B
:1037E00000BFBDF8E4000A281DD09DF8B41040F2D7
:1037F000A11011FB00F0C24901EBC00101F562719B
:103800009DF8A020BDF8D800104400EB400202EB68
:10381000001001EBC00090300990007820F001000A
:10382000401C09990870BDF8A4000F287ED19DF8AE
:10383000B41001EB410000EB0110B24901EB0011A3
:1038400030319DF8A020BDF8D800104401EB0010E5
:10385000801C0990007820F00400001D0999087070
:10386000002039902DE09DF8B41001EB4100C0EB31
:10387000C110A54901EBC001BDF84020BDF8E4002E
:1038800010440A5C9DF8B40040F2A11110FB01F055
:103890009B4901EBC00101F562719DF8A030BDF8B4
:1038A000D800184400EB400303EB001001EBC0010B
:1038B0004731BDF8E4000A54BDF8E400401C81B271
:1038C0003991BDF8E4000A28CDDBBDF840000A308C
:1038D00081B21091002139912FE09DF8B41001EBD5
:1038E0004100C0EBC110884901EBC001BDF8402088
:1038F000BDF8E40010440A5C9DF8B40040F2A11148
:1039000010FB01F07E4901EBC00101F562719DF8E9
:10391000A030BDF8D800184400EB400303EB0010C2
:1039200001EBC0016031BDF8E40000E078E20A5428
:10393000BDF8E400401C81B23991BDF8E4000228D2
:10394000CBDBBDF84000801C81B210919DF8B41013
:1039500001EB4100C0EBC1106B4901EBC001BDF8A8
:103960004000085C01049DF8B40000EB4002C2EB8B
:10397000C010654A02EBC002BDF84000401C105C5C
:1039800041EA00219DF8B40000EB4002C2EBC010F8
:103990005D4A02EBC002BDF84000801C105C014390
:1039A0009DF8B40040F2A11210FB02F0544A02EB61
:1039B000C00202F562729DF8A030BDF8D80018442C
:1039C00000EB400303EB001002EBC0004167BDF8C1
:1039D0004000C01C81B210914C4890F8E007E8BB51
:1039E0000021399120E09DF8B41040F2A11011FBA4
:1039F00000F0434901EBC00101F562719DF8A02080
:103A0000BDF8D800104400EB400202EB001001EBBF
:103A1000C0004730BDF8E410405C00B108E0BDF8DC
:103A2000E400401C81B23991BDF8E4000A28DADBD9
:103A300000BFBDF8E4000A281BD140229DF8B40065
:103A400040F2A11110FB01F02D4901EBC00101F57D
:103A500062719DF8A030BDF8D80000E05AE018442B
:103A600000EB400303EB001001EBC00080F87E2068
:103A700066E19DF8B41040F2A11011FB00F020495E
:103A800001EBC00101F562719DF8A020BDF8D800DE
:103A9000104400EB400202EB001001EBC00090F874
:103AA0007E00B8BB00212A9121E10021379137E047
:103AB0009DF8B41040F2A11011FB00F0104901EB89
:103AC000C00101F562719DF8A020BDF8D800104436
:103AD00000EB400202EB001001EBC0014731BDF8E2
:103AE000DC00001D095C9DF8A80000EB40020848BE
:103AF00000EB4202BDF8DC00105C81420BD013E009
:103B00005845002098400020F8870020BC32002053
:103B10008834002014E1BDF8DC00401C81B23791EC
:103B2000BDF8DC000628C3DB00BFBDF8DC000628BA
:103B30007ED103229DF8B40040F2A11110FB01F0E8
:103B4000FE4901EBC00101F562719DF8A030BDF89E
:103B5000D800184400EB400303EB001001EBC00059
:103B600080F87E209DF8B41001EB410000EB0110BD
:103B7000F34901EB001130319DF8A020BDF8D800C9
:103B8000104401EB0010801C0990007820F0040222
:103B900009980270002039901FE020229DF8B4009F
:103BA00040F2A11110FB01F0E44901EBC00101F565
:103BB00062719DF8A030BDF8D800184400EB4003B6
:103BC00003EB001001EBC0015131BDF8E4000A54D1
:103BD000BDF8E400401C81B23991BDF8E4000F2823
:103BE000DBDB002139911FE020229DF8B40040F278
:103BF000A11110FB01F0D14901EBC00101F5627187
:103C00009DF8A030BDF8D800184400EB400303EB4A
:103C1000001001EBC0016331BDF8E4000A54BDF8A7
:103C2000E400401C81B23991BDF8E4000A2800E0AC
:103C300058E0D9DB00229DF8B40040F2A11110FB3E
:103C400001F0BE4901EBC00101F562719DF8A030A1
:103C5000BDF8D800184400EB400303EB001001EB63
:103C6000C00080F87820002139911FE000229DF8E3
:103C7000B40040F2A11110FB01F0B04901EBC0010A
:103C800001F562719DF8A030BDF8D800184400EB32
:103C9000400303EB001001EBC0017931BDF8E400F3
:103CA0000A54BDF8E400401C81B23991BDF8E4002B
:103CB0000528DBDB9DF8B41040F2A11011FB00F0E9
:103CC0009E4901EBC00101F562719DF8A020BDF88D
:103CD000D800104400EB400202EB001001EBC000E2
:103CE000406F0CE09DF8A800401CC1B22A91954895
:103CF000B0F8CA019DF8A81088423FF7D6AE00BFC1
:103D00009048B0F8CA019DF8A810884218D1402206
:103D10009DF8B40040F2A11110FB01F0874901EBBE
:103D2000C00101F562719DF8A030BDF8D8001844BB
:103D300000EB400303EB001001EBC00080F87E2095
:103D40009DF8B41040F2A11011FB00F07B4901EB8B
:103D5000C00101F562719DF8A020BDF8D8001044A3
:103D600000EB400202EB001001EBC00090F87E0077
:103D7000032804D011281ED0402850D134E0F2226C
:103D80009DF8B40040F2A11110FB01F06B4901EB6A
:103D9000C00101F562719DF8A030BDF8D80018444B
:103DA00000EB400303EB001001EBC000427136E072
:103DB000F1E3F1E316E1F3229DF8B40040F2A11122
:103DC00010FB01F05D4901EBC00101F562719DF846
:103DD000A030BDF8D800184400EB400303EB0010FE
:103DE00001EBC00042711AE0F2229DF8B40040F2EB
:103DF000A11110FB01F0514901EBC00101F5627105
:103E00009DF8A030BDF8D800184400EB400303EB48
:103E1000001001EBC00000E0C5E0427100BF6AE0A5
:103E20009DF8B40000EB400101EB0010444901EBA8
:103E3000001030309DF8A020BDF8D810114400EBE0
:103E40000110801C0990007820F00402099802708B
:103E50009DF8B40040F2A11110FB01F0374901EBCD
:103E6000C00000F562709DF8A020BDF8D810114484
:103E700001EB410202EB011100EBC10090F8900050
:103E800000F00100B8B300229DF8B40040F2A11187
:103E900010FB01F0294901EBC00101F562719DF8A9
:103EA000A03005E0FDE3FDE3ACE0FCE3FCE3FCE374
:103EB000BDF8D800184400EB400303EB001001EB01
:103EC000C000A0F88E2005229DF8B40040F2A11198
:103ED00010FB01F0194901EBC00101F562719DF879
:103EE000A030BDF8D800184400EB400303EB0010ED
:103EF00001EBC00042716FE0FFE79DF8B40040F2B3
:103F0000A11110FB01F00D4901EBC00101F5627137
:103F10009DF8A020BDF8D800104400EB400202EB51
:103F2000001001EBC00090F87E00402821D1002253
:103F30009DF8B40040F2A11106E0000058450020B1
:103F400098400020BC32002010FB01F0FE4901EB3C
:103F5000C00101F562719DF8A030BDF8D800184489
:103F600000EB400303EB001001EBC00080F87E2063
:103F700000BF00BFF1229DF8B40040F2A11110FB78
:103F800001F0F14901EBC00101F562719DF8A0302B
:103F9000BDF8D800184400EB400303EB001001EB20
:103FA000C000427118E0F1229DF8B40040F2A11166
:103FB00010FB01F0E44901EBC00101F562719DF8CD
:103FC000A030BDF8D800184400EB400303EB00100C
:103FD00001EBC000427100BF00BFBDF8D800401C1B
:103FE00081B236919DF8B40000EB4001C1EBC010E6
:103FF000D64901EBC0004179BDF8D80081423FF7B6
:10400000EDAAF4E39DF8B40040F2A11110FB01F019
:10401000CD4901EBC00000F562709DF8A01001EBE6
:10402000410202EB011110F8310048BB01229DF85A
:10403000B40040F2A11110FB01F0C34901EBC00133
:1040400001F562719DF8A00000EB400303EB001046
:1040500001F83020F4229DF8B40040F2A11110FBC9
:1040600001F0B94901EBC00000F562709DF8A010A5
:1040700001EB410303EB011100EBC1004271CDE004
:104080009DF8B40000EB400101EB0010B04901EBDA
:10409000001030309DF8A01000EB0110407A00F0C5
:1040A000010080B39DF8B40040F2A11110FB01F0B3
:1040B000A54901EBC00000F562709DF8A01001EB6E
:1040C000410202EB011100EBC10090F8900000F0FA
:1040D0000100C0B99DF8B40040F2A11110FB01F03D
:1040E000994901EBC00000F562709DF8A01001EB4A
:1040F000410202EB011100EBC10090F8820010B107
:10410000002139912DE089E09DF8B40040F2A11121
:1041100010FB01F08C4901EBC00101F562719DF8C3
:10412000A00000EB400202EB001001EBC00000F128
:104130008301BDF8E4000A5C9DF8B40000EB400187
:1041400001EB0010824901EB00100E30BDF8E410C5
:10415000405C824200D008E0BDF8E400401C81B21F
:104160003991BDF8E4000428CEDB00BFBDF8E400BF
:10417000042853D1042139912CE09DF8B40040F279
:10418000A11110FB01F0704901EBC00101F5627152
:104190009DF8A00000EB400202EB001001EBC00014
:1041A00000F18301BDF8E4000A5C9DF8B40000EB67
:1041B000400101EB0010664901EB00100E30BDF824
:1041C000E410405C824200D008E0BDF8E400401CEE
:1041D00081B23991BDF8E4000A28CEDB00BFBDF8FA
:1041E000E4000A281AD09DF8B40040F2A11110FB97
:1041F00001F0554901EBC00000F562709DF8A01078
:1042000001EB410202EB011100EBC100903009907B
:10421000007820F00100401C09990870BDF8A40046
:10422000112877D19DF8B40000EB400101EB00109C
:10423000474901EB001030309DF8A01000EB011051
:10424000801C0990007820F00400001D0999087076
:104250000020399028E09DF8B40000EB4001C1EB4C
:10426000C0103A4901EBC001BDF8E400401D0A5CF2
:104270009DF8B40040F2A11110FB01F0324901EBAE
:10428000C00101F562719DF8A00000EB400303EB53
:10429000001001EBC0014731BDF8E4000A54BDF83D
:1042A000E400401C81B23991BDF8E4000A28D2DB59
:1042B0000021399128E09DF8B40000EB4001C1EBEA
:1042C000C010224901EBC001BDF8E4000F300A5CC8
:1042D0009DF8B40040F2A11110FB01F01A4901EB66
:1042E000C00101F562719DF8A00000EB400303EBF3
:1042F000001001EBC0016031BDF8E4000A54BDF8C4
:10430000E400401C81B23991BDF8E4000228D2DB00
:10431000B0E2FFE7BDF8A40014287DD19DF8B400F9
:1043200000EB400101EB0010094901EB00103030B7
:104330009DF8A01000EB0110801C0990007820F07F
:104340000400001D099905E058450020F887002069
:104350009840002008700020399028E09DF8B400B3
:1043600000EB4001C1EBC010F84901EBC001BDF802
:10437000E400401D0A5C9DF8B40040F2A11110FB5E
:1043800001F0F34901EBC00101F562719DF8A00055
:1043900000EB400303EB001001EBC0014731BDF817
:1043A000E4000A54BDF8E400401C81B23991BDF824
:1043B000E4000A28D2DB0021399128E09DF8B400FE
:1043C00000EB4001C1EBC010E04901EBC001BDF8BA
:1043D000E4000F300A5C9DF8B40040F2A11110FB1C
:1043E00001F0DB4901EBC00101F562719DF8A0000D
:1043F00000EB400303EB001001EBC0016031BDF89E
:10440000E4000A54BDF8E400401C81B23991BDF8C3
:10441000E4000228D2DB00E02DE29DF8B40000EBBE
:104420004001C1EBC010C94901EBC000407C010450
:104430009DF8B40000EB4002C2EBC010C34A02EB8F
:10444000C000807C41EA00219DF8B40000EB4002EE
:10445000C2EBC010BD4A02EBC000C07C01439DF816
:10446000B40040F2A11210FB02F0B94A02EBC00006
:1044700000F562709DF8A02002EB420303EB0212EC
:1044800000EBC2004167B34890F8E007F0BB0021A1
:1044900039911DE09DF8B40040F2A11110FB01F02C
:1044A000AB4901EBC00101F562719DF8A00000EB82
:1044B000400202EB001001EBC0004730BDF8E410F1
:1044C000405C00B108E0BDF8E400401C81B23991C5
:1044D000BDF8E4000A28DDDB00BFBDF8E4000A28CF
:1044E00018D140229DF8B40040F2A11110FB01F058
:1044F000974901EBC00000F562709DF8A01001EB38
:10450000410303EB011100EBC10000E045E080F83E
:104510007E2050E19DF8B40040F2A11110FB01F0A3
:104520008B4901EBC00000F562709DF8A01001EB13
:10453000410202EB011100EBC10090F87E0060BB6C
:1045400000212A9111E1002137912CE09DF8B4005F
:1045500040F2A11110FB01F07D4901EBC00101F512
:1045600062719DF8A00000EB400202EB001001EB2D
:10457000C0014731BDF8DC00001D095C9DF8A800B2
:1045800000EB4002744800EB4202BDF8DC00105C16
:10459000814203D00BE0FDE3FDE30CE1BDF8DC005C
:1045A000401C81B23791BDF8DC000628CEDB00BF8D
:1045B000BDF8DC00062879D103229DF8B40040F252
:1045C000A11110FB01F0624901EBC00101F562711C
:1045D0009DF8A00000EB400303EB001001EBC000CE
:1045E00080F87E209DF8B40000EB400101EB001044
:1045F0005A4901EB001130319DF8A00001EB001089
:10460000801C0990007820F00402099802700020B4
:1046100039901CE020229DF8B40040F2A11110FB5B
:1046200001F04B4901EBC00101F562719DF8A0005A
:1046300000EB400303EB001001EBC0015131BDF86A
:10464000E4000A54BDF8E400401C81B23991BDF881
:10465000E4000F28DEDB002139911CE020229DF8C8
:10466000B40040F2A11110FB01F0394901EBC00187
:1046700001F562719DF8A00000EB400303EB001010
:1046800001EBC0016331BDF8E4000A54BDF8E40059
:10469000401C81B23991BDF8E4000A28DEDB00221B
:1046A00005E0FCE3FCE3FCE3FCE3E9E358E09DF810
:1046B000B40040F2A11110FB01F0254901EBC0014B
:1046C00001F562719DF8A00000EB400303EB0010C0
:1046D00001EBC00080F87820002139911CE0002215
:1046E0009DF8B40040F2A11110FB01F0184901EB54
:1046F000C00101F562719DF8A00000EB400303EBDF
:10470000001001EBC0017931BDF8E4000A54BDF896
:10471000E400401C81B23991BDF8E4000528DEDBDD
:104720009DF8B40040F2A11110FB01F0084901EB23
:10473000C00000F562709DF8A01001EB410202EB91
:10474000011100EBC100406F17E00000F887002066
:1047500058450020BC3200208834002098400020BA
:104760009DF8A800401CC1B22A91FE48B0F8CA11B9
:104770009DF8A80081423FF7E6AE00BFF948B0F8C7
:10478000CA019DF8A810884215D140229DF8B400B6
:1047900040F2A11110FB01F0F34901EBC00000F55C
:1047A00062709DF8A01001EB410303EB011100EBD7
:1047B000C10080F87E209DF8B40040F2A11110FBEA
:1047C00001F0E94901EBC00000F562709DF8A0100E
:1047D00001EB410202EB011100EBC10090F87E00F9
:1047E000032805D0112819D0402843D12CE045E3F7
:1047F000F2229DF8B40040F2A11110FB01F0DA4959
:1048000001EBC00000F562709DF8A01001EB4103C0
:1048100003EB011100EBC10042712BE0F3229DF884
:10482000B40040F2A11110FB01F0CF4901EBC00030
:1048300000F562709DF8A01001EB410303EB01113C
:1048400000EBC100427115E0F2229DF8B40040F285
:10485000A11110FB01F0C44901EBC00000F562702A
:104860009DF8A01001EB410303EB011100EBC10027
:10487000427100BF02E3BDF8A40006287DD19DF877
:10488000B40000EB4001C1EBC010B84901EBC0001F
:104890004079012872D10320B5490870F7229DF8AC
:1048A000B40040F2A11110FB01F0AF4901EBC001CF
:1048B00001F562719DF8A00000EB400303EB0010CE
:1048C00001EBC00042719DF8B40040F2A11110FB51
:1048D00001F0A54901EBC00101F562719DF8A0004E
:1048E00000EB400202EB001001EBC00090F88000EA
:1048F00000EB400101EB00109E4901EB001130314B
:104900009DF8B40040F2A11210FB02F0964A02EBAF
:10491000C00000F562709DF8A02002EB420303EB9B
:10492000021200EBC20090F8810001EB00108078C9
:10493000C0F34000F0B39DF8B41040F2A11011FB99
:1049400000F0894901EBC00000F562709DF8A010ED
:1049500001EB410202EB011100EBC10090F8801065
:1049600001EB410000EB0110824901EB001080795E
:10497000012804D00A287CD13FE027E2CDE0BA2309
:104980009DF8B40040F2A11110FB01F0764901EB53
:10499000C00101F562719DF8A00000EB400202EB3E
:1049A000001001EBC00090F8800040F2A11110FB54
:1049B00001F000E03AE16C4901EBC00101F56271E0
:1049C0009DF8B40040F2A11210FB02F0664A02EB1F
:1049D000C00000F562709DF8A02002EB420404EBD9
:1049E000021200EBC20090F8810000EB400202EBE3
:1049F000001001EBC00043713BE00B239DF8B400B5
:104A000040F2A11110FB01F0574901EBC00101F583
:104A100062719DF8A00000EB400202EB001001EB78
:104A2000C00090F8800040F2A11110FB01F04E4947
:104A300001EBC00101F562719DF8B40040F2A112D2
:104A400010FB02F0484A02EBC00000F562709DF8CE
:104A5000A02002EB420404EB021200EBC20090F82B
:104A6000810000EB400202EB001001EBC00043713B
:104A700000BF00BF9DF8B41040F2A11011FB00F080
:104A8000394901EBC00101F562719DF8A00000EB0E
:104A9000400202EB001001EBC00090F8801001EB27
:104AA000410000EB0110334901EB001130319DF85A
:104AB000B40040F2A11210FB02F02B4A02EBC0023C
:104AC00002F562729DF8A00000EB400303EB0010BA
:104AD00002EBC00090F8810001EB001002789DF815
:104AE000B40040F2A11110FB01F01F4901EBC0011D
:104AF00001F562719DF8A00000EB400303EB00108C
:104B000001EBC00090F8800040F2A11110FB01F011
:104B1000154901EBC0004270B0E19DF8B41001EB03
:104B20004100C0EBC110114901EBC00040790228DF
:104B30007CD104200E490870F8229DF8B40040F2A0
:104B4000A11110FB01F0084901EBC00101F56271F0
:104B50009DF8A00000EB400303EB001001EBC00048
:104B6000427109E0BC32002058450020F88700203F
:104B700019020020984000209DF8B41040F2A110C6
:104B800011FB00F0F94901EBC00101F562719DF8DC
:104B9000A00000EB400202EB001001EBC00090F817
:104BA000801001EB410000EB0110F14901EB001115
:104BB00030319DF8B40040F2A11210FB02F0EB4A34
:104BC00002EBC00000F562709DF8A02002EB4203EA
:104BD00003EB021200EBC20090F8810001EB001021
:104BE0008078C0F3400008B39DF8B41040F2A110E3
:104BF00011FB00F0DD4901EBC00000F562709DF88B
:104C0000A01001EB410202EB011100EBC10090F892
:104C1000800000EB400101EB0010D54901EB0010D2
:104C20008079012803D00A2879D13CE026E1B3231A
:104C30009DF8B40040F2A11110FB01F0CB4901EB4B
:104C4000C00101F562719DF8A00000EB400202EB8B
:104C5000001001EBC00090F8800040F2A11110FBA1
:104C600001F0C24901EBC00101F562719DF8B40089
:104C700040F2A11210FB02F0BC4A02EBC00000F5AA
:104C800062709DF8A02002EB420404EB021200EBDC
:104C9000C20090F8810000EB400202EB001001EB33
:104CA000C00043713BE00C239DF8B40040F2A11119
:104CB00010FB01F0AD4901EBC00101F562719DF8F7
:104CC000A00000EB400202EB001001EBC00090F8E6
:104CD000800040F2A11110FB01F0A44901EBC001DA
:104CE00001F562719DF8B40040F2A11210FB02F0D0
:104CF0009E4A02EBC00000F562709DF8A02002EB16
:104D0000420404EB021200EBC20090F8810000EBB9
:104D1000400202EB001001EBC000437100BF00BF76
:104D20009DF8B41040F2A11011FB00F08F4901EB87
:104D3000C00101F562719DF8A00000EB400202EB9A
:104D4000001001EBC00090F8801001EB410000EB77
:104D50000110874901EB001130319DF8B40040F299
:104D6000A11210FB02F0814A02EBC00202F562724E
:104D70009DF8A00000EB400303EB001002EBC00025
:104D800090F8810001EB001002789DF8B40040F229
:104D9000A11101E08FE072E010FB01F0734901EB1B
:104DA000C00000F562709DF8A01001EB410303EB19
:104DB000011100EBC10090F8800040F2A11110FB3E
:104DC00001F06A4901EBC000427057E09DF8B41051
:104DD00001EB410000EB0110654901EB00103030A0
:104DE0009DF8A01000EB0110801C0990007820F0C5
:104DF0000402099802709DF8B41040F2A11011FB52
:104E000000F05A4901EBC00000F562709DF8A01057
:104E100001EB410202EB011100EBC10090F89000A0
:104E200000F0010050B300229DF8B40040F2A1113F
:104E300010FB01F04D4901EBC00101F562719DF8D5
:104E4000A00000EB400303EB001001EBC000A0F852
:104E50008E2005229DF8B40040F2A11110FB01F054
:104E6000424901EBC00000F562709DF8A01001EB13
:104E7000410303EB011100EBC100427193E100BF5C
:104E8000F1229DF8B40040F2A11110FB01F0374966
:104E900001EBC00000F562709DF8A01003E04FE048
:104EA00005E191E066E001EB410303EB011100EB4A
:104EB000C100427177E19DF8B41040F2A11011FBDE
:104EC00000F02A4901EBC00000F562709DF8A010C7
:104ED00001EB410202EB011100EBC10090F87E00F2
:104EE000402816D100229DF8B40040F2A11110FB19
:104EF00001F01E4901EBC00000F562709DF8A010A2
:104F000001EB410303EB011100EBC10080F87E20AF
:104F100000BF00BFF1229DF8B40040F2A11110FBC8
:104F200001F0124901EBC00000F562709DF8A0107D
:104F300001EB410303EB011100EBC100427132E1CF
:104F4000F1229DF8B40040F2A11110FB01F00749D5
:104F500001EBC00000F562709DF8A01001EB410369
:104F600003EB011100EBC10042711CE15845002028
:104F70009840002003229DF8B40040F2A11110FBDC
:104F800001F0FE4901EBC00101F562719DF8A0003E
:104F900000EB400303EB001001F83020F1229DF8F4
:104FA000B40040F2A11110FB01F0F44901EBC00084
:104FB00000F562709DF8A01001EB410303EB0111B5
:104FC00000EBC1004271EEE002229DF8B40040F215
:104FD000A11110FB01F0E94901EBC00101F562717B
:104FE0009DF8A00000EB400303EB001001F8302017
:104FF000F6229DF8B40040F2A11110FB01F0DF4948
:1050000001EBC00101F562719DF8A00000EB4003C7
:1050100003EB001001EBC000427101229DF8B400C7
:1050200040F2A11110FB01F0D44901EBC00101F5E0
:1050300062719DF8A00000EB400303EB001001EB50
:10504000C00080F882200021399129E09DF8B41039
:1050500001EB4100C0EBC110C94901EBC001BDF833
:10506000E400401D0A5C9DF8B40040F2A11110FB61
:1050700001F0C24901EBC00101F562719DF8A00089
:1050800000EB400303EB001001EBC00000F18301D3
:10509000BDF8E4000A54BDF8E400401C81B2399127
:1050A000BDF8E4000A28D1DBBDF8A4007BE09DF840
:1050B000B41001EB4100C0EBC110B14901EBC000DD
:1050C00081799DF8B40000EB4002C2EBC010AC4AFD
:1050D00002EBC000407941EA00229DF8B40040F2A2
:1050E000A11110FB01F0A54901EBC00101F56271AE
:1050F0009DF8A00000EB400303EB001001EBC000A3
:10510000A0F88E209DF8B40040F2A11110FB01F030
:105110009A4901EBC00101F562719DF8A00000EB16
:10512000400202EB001001EBC000B0F88E109DF8B9
:10513000B40000EB400202EB0010924A02EB0010B8
:10514000408B81422EDBF1229DF8B40040F2A11188
:1051500010FB01F0894901EBC00101F562719DF876
:10516000A00000EB400303EB001001EBC000427114
:105170009DF8B40040F2A11110FB01F07F4901EB52
:10518000C00101F562719DF8A00000EB400202EB46
:10519000001001EBC00090300990007820F001026F
:1051A0000998027000BF00BF09F032B89DF8B40042
:1051B00000EB4001C1EBC010714901EBC000017967
:1051C0002891002136911CE09DF8B40000EB4001CD
:1051D00001EB00106B4901EB00113031BDF8D80034
:1051E00001EB001041789DF8A000814204D1BDF888
:1051F000D800C1B2289112E0BDF8D800401C81B29D
:1052000036919DF8B40000EB400101EB00105D49C0
:1052100001EB0010C179BDF8D8008142D4DC00BF99
:105220009DF8B40000EB4001C1EBC010544901EB04
:10523000C000C1782591BDF89400172834D2DFE86A
:1052400000F0330C0F331215181B1E333333333376
:105250003321242733332A2D30000721299123E0DD
:105260000721299120E0062129911DE0062029909F
:105270001AE00621299117E01221299114E0072153
:10528000299111E0092029900EE0062129910BE0D7
:105290000621299108E00B21299105E00B21299194
:1052A00002E02A21299100BF00BFBDF8A400001F21
:1052B000C1B209919DF8B40000EB4001C1EBC010F0
:1052C0002F4901EBC000C01C08900999F4F702F9BE
:1052D00037909DF8B40000EB4001C1EBC0102849A5
:1052E00001EBC001BDF8A400401E095CBDF8DC0064
:1052F000814270D19DF8B40000EB4001C1EBC010B9
:105300001F4901EBC0004078002864DD9DF8B4001F
:1053100000EB4001C1EBC010194901EBC001BDF821
:10532000A4000A5C9DF8B40040F2A11110FB01F04A
:10533000124901EBC00101F562719DF8A00000EB7C
:10534000400303EB001001EBC00080F84420002173
:105350000D4A9DF8B40002EB00129DF8A000115414
:105360000A4890F82800012821D19DF8B40000EBEC
:10537000400101EB001003490AE0000058450020FD
:10538000F887002098400020883E0020BC120020B2
:1053900001EB001030309DF8A01000EB0110801CD4
:1053A0000990007820F08000803009990870BDF8DD
:1053B000940007287ED00ADC07287CD2DFE810F0B2
:1053C0007B006506C7067B004F061206CA0C103824
:1053D0000728F2D200E0FDE3DFE810F02A0D140DFB
:1053E0006D006D0007000800F00600BFBDF89400D6
:1053F00014287DD19DF8B40000EB4001C1EBC01032
:10540000FE4901EBC000407901069DF8B40000EBB5
:105410004002C2EBC010F94A02EBC000807941EAB9
:1054200000419DF8B40000EB4002C2EBC010F34A0B
:1054300002EBC000C07941EA00219DF8B40000EB06
:105440004002C2EBC010ED4A02EBC000007A0143FB
:105450009DF8B40040F2A11210FB02F0E84A02EB02
:10546000C00202F562729DF8A00000EB400303EB5E
:10547000001002EBC000C0F81A109DF8B40040F212
:10548000A11110FB01F0DE4901EBC00101F56271D1
:105490009DF8A00000EB400202EB001001EBC00001
:1054A000D0F81A1008460991002111F0F9FBCDE956
:1054B0002E0101E0FEE3FEE39DF8B40000EB4001A5
:1054C00001EB0010CF4901EB0010007F00F0030159
:1054D0009DF8B40000EB400202EB0010C94A02EB59
:1054E0000010007FC0F3011001449DF8B40000E0FB
:1054F0006CE000EB400202EB0010C24A02EB00102D
:10550000007FC0F38100091A08460591F3F76FF890
:10551000CDE906019DED061B9FEDBB0B20F0A8FB1E
:105520008DED080B9DED080B51EC100BF3F7D1F846
:10553000CDE930019DF8B40040F2A11110FB01F05B
:10554000AF4901EBC00101F562719DF8A00000EBCD
:10555000400202EB001001EBC000416B08460791CE
:10556000002111F09DFBDDE92E32A0FB034501FB7C
:10557000035100FB021502220023DDE93001F2F79E
:1055800021FE20186941CDE90801DDE93023F2F759
:1055900019FECDE92E01DDE92E0112F035F90146A3
:1055A0009DF8B40040F2A11210FB02F0944A02EB05
:1055B000C00000F562709DF8A02002EB420303EBEF
:1055C000021200EBC200C0F81E1046E0BDF89400C5
:1055D000152842D19DF8B40000EB4001C1EBC0108A
:1055E000864901EBC000407901069DF8B40000EB4C
:1055F0004002C2EBC010814A02EBC000807941EA50
:1056000000419DF8B40000EB4002C2EBC0107B4AA1
:1056100002EBC000C07941EA00219DF8B40000EB24
:105620004002C2EBC010754A02EBC000007A014391
:105630009DF8B40040F2A11210FB02F0704A02EB98
:10564000C00000F562709DF8A02002EB420303EB5E
:10565000021200EBC200C0F81E109DF8B40000EB6F
:105660004001C1EBC010654901EBC000427A9DF8D2
:10567000B40040F2A11110FB01F0614901EBC0013F
:1056800001F562719DF8A00000EB400303EB0010F0
:1056900001EBC00080F894209DF8B40000EB4001BD
:1056A00001EB0010574901EB001030309DF8A010BD
:1056B00000EB0110801C09909DF8B40040F2A1118C
:1056C00010FB01F04E4901EBC00000F562709DF83F
:1056D000A02002EB420101EB021100EBC10090F8A7
:1056E0009400C2090998017862F3000101709DF8E5
:1056F000B40040F2A11110FB01F0414901EBC000E0
:1057000000F562709DF8A01001EB410202EB01115F
:1057100000EBC10090F8940000F00300012818D0BD
:105720009DF8B40040F2A11110FB01F0344901EBE7
:10573000C00000F562709DF8A01001EB410202EB81
:10574000011100EBC10090F8940000F00300032861
:105750002BD19DF8B40000EB400101EB001029496A
:1057600001EB001030309DF8A01000EB0110801C00
:105770000990007820F00201891C099801709DF8B9
:10578000B40000EB400101EB00101E4901EB0011D9
:1057900030319DF8A00001EB0010801C09900078CA
:1057A00020F020020998027014E09DF8B40000EB8C
:1057B000400101EB0010134901EB001030309DF85F
:1057C000A01000EB0110801C0990007820F002026C
:1057D000099802709DF8B40000EB400101EB001045
:1057E000084901EB001130319DF8A00001EB0010D9
:1057F0008078C0F340029DF8B40009E0F8870020EB
:10580000584500209840002000000000000024407F
:1058100040F2A11110FB01F0FE4901EBC00000F5C0
:1058200062709DF8A01001EB410303EB011100EB46
:10583000C100007EC0F3400082426CD09DF8B400ED
:1058400040F2A11110FB01F0F24901EBC00000F59C
:1058500062709DF8A01001EB410202EB011100EB18
:10586000C100183009909DF8B40000EB400101EB35
:105870000010E94901EB001030309DF8A01000EB5A
:105880000110807842080998007862F34100099974
:1058900008709DF8B40000EB400101EB0010DE49F8
:1058A00001EB001030309DF8A01000EB0110807863
:1058B000C0F3400050BB9DF8B40000EB400101EB89
:1058C0000010D54901EB001030309DF8A01000EB1E
:1058D0000110801C0990007820F0200209980270C5
:1058E00001229DF8B40040F2A11110FB01F0C9495A
:1058F00001EBC00000F562709DF8A01001EB4103C0
:1059000003EB011100EBC10080F846209DF8B410B4
:105910000220F4F7CBFB9DF8B40000EB400101EB53
:105920000010BD4901EB001130319DF8A00001EBE2
:105930000010807800F001029DF8B40040F2A1113F
:1059400010FB01F0B34901EBC00000F562709DF857
:10595000A01001EB410303EB011100EBC100007E3D
:1059600000F00100824265D09DF8B40040F2A11120
:1059700010FB01F0A74901EBC00000F562709DF833
:10598000A01001EB410202EB011100EBC100183045
:1059900009909DF8B40000EB400101EB00109E4916
:1059A00001EB001030309DF8A01000EB0110807862
:1059B00009990A7860F300020A709DF8B40000EBC0
:1059C000400101EB0010944901EB001030309DF8CC
:1059D000A01000EB0110807800F0010058BB9DF88A
:1059E000B40000EB400101EB00108B4901EB00100B
:1059F00030309DF8A01000EB0110801C0990007859
:105A000020F020020998027000229DF8B40040F2B4
:105A1000A11110FB01F07F4901EBC00000F562709D
:105A20009DF8A01001EB410303EB011100EBC10055
:105A300080F8452015E29DF8B40040F2A11110FB5A
:105A400001F0744901EBC00000F562709DF8A010F0
:105A500001EB410202EB011100EBC10090F846009E
:105A6000B0B901229DF8B40040F2A11110FB01F081
:105A7000684901EBC00000F562709DF8A01001EBD1
:105A8000410303EB011100EBC10080F845202AE03F
:105A900000229DF8B40040F2A11110FB01F05D4915
:105AA00001EBC00101F562719DF8A00000EB40031D
:105AB00003EB001001EBC00080F845209DF8B40016
:105AC00000EB400101EB0010534901EB00113031B4
:105AD0009DF8A00001EB0010801C0990007820F0D8
:105AE0000102099802704D4890F8E00780B19DF8D6
:105AF000B40000EB400101EB0010474901EB00103E
:105B000030309DF8A01000EB0110807A022862D19D
:105B1000434890F8290001287AD14148D0F80C0276
:105B20003F49498D884273D29DF8B40040F2A111DB
:105B300010FB01F0374901EBC00000F562709DF8E1
:105B4000A01001EB410202EB011100EBC10090F843
:105B5000450001283FD19DF8B40040F2A11110FB8F
:105B600001F02C4901EBC00000F562709DF8A01017
:105B700001EB410202EB011100EBC10090F87F0044
:105B800048BB01229DF8B40000EB400101EB00107E
:105B9000214901EB001130319DF8A00001EB00100C
:105BA000C2729DF8B40000EB400101EB00101A49ED
:105BB00001EB001130319DF8A00001EB00100178DD
:105BC0009DF8B40040F2A11210FB02F0114A02EB62
:105BD000C00001E0FEE316E1417005229DF8B4002B
:105BE00040F2A11110FB01F00A4901EBC00101F5DF
:105BF00062719DF8A00000EB400303EB001001EB85
:105C0000C000427100229DF8B40000EB400109E0A1
:105C100064E000005845002098400020BC3200207D
:105C2000BC12002001EB0010FE4901EB00113031E5
:105C30009DF8A00001EB001042609DF8B410022016
:105C4000F4F734FA002139911CE000229DF8B400E9
:105C500040F2A11110FB01F0F34901EBC00101F585
:105C600062719DF8A00000EB400303EB001001EB14
:105C7000C0014731BDF8E4000A54BDF8E400401CFF
:105C800081B23991BDF8E4001428DEDB00203990A0
:105C90001FE000229DF8B40040F2A11110FB01F0BA
:105CA000E14901EBC00101F562719DF8A00000EB34
:105CB000400301E05DE349E203EB001001EBC001AA
:105CC0006331BDF8E4000A54BDF8E400401C81B221
:105CD0003991BDF8E4000A28DBDBC2E09DF8B4008E
:105CE00040F2A11110FB01F0CF4901EBC00000F51B
:105CF00062709DF8A01001EB410202EB011100EB74
:105D0000C10090F8450001287DD19DF8B40040F213
:105D1000A11110FB01F0C44901EBC00101F5627152
:105D20009DF8A00000EB400202EB001001EBC00068
:105D300090F8800040F2A11110FB01F0BA4901EB8C
:105D4000C00101F562719DF8B40040F2A11210FB90
:105D500002F0B54A02EBC00000F562709DF8A02089
:105D600002EB420303EB021200EBC20090F8810049
:105D700000EB400202EB001001EBC00090F87E0047
:105D800003286ED102229DF8B40000EB400101EB24
:105D90000010A44901EB001130319DF8A00001EB87
:105DA0000010C2729DF8B40000EB400101EB00103E
:105DB0009C4901EB001130319DF8A00001EB00106F
:105DC00001789DF8B40040F2A11210FB02F0964A4F
:105DD00002EBC00041709DF8B40040F2A11110FB2D
:105DE00001F0114601EBC00101F562719DF8A000C0
:105DF00000EB400202EB001011F830109DF8B400E7
:105E000040F2A11200E02CE010FB02F0864A02EB07
:105E1000C0004079814214D105229DF8B40040F2BF
:105E2000A11110FB01F0804901EBC00000F5627088
:105E30009DF8A01001EB410303EB011100EBC10041
:105E4000427100229DF8B40000EB400101EB00100C
:105E5000744901EB001030309DF8A01000EB0110E8
:105E600042609DF8B40040F2A11110FB01F06E49B0
:105E700001EBC00000F562709DF8A01001EB41023B
:105E800002EB011110F83100012814DC02229DF808
:105E9000B40040F2A11110FB01F0634901EBC00016
:105EA00000F562709DF8A01001EB410303EB0111B6
:105EB00000F8312095E09DF8B40040F2A11110FBEC
:105EC00001F0594901EBC00000F562709DF8A01087
:105ED00001EB410202EB011110F83100022834DC21
:105EE00000219DF8B40040F2A11210FB02F04E4ACE
:105EF00002EBC000017103229DF8B40040F2A11131
:105F000010FB01F0484901EBC00101F562719DF8F9
:105F1000A00000EB400303EB001001F83020072243
:105F20009DF8B40040F2A11110FB01F03E4901EBD5
:105F3000C00000F562709DF8A01001EB410303EB77
:105F4000011100EBC10042714BE09DF8B40040F23A
:105F5000A11110FB01F0344901EBC00101F56271A0
:105F60009DF8A00000EB400202EB001011F8301089
:105F70009DF8B40040F2A11210FB02F02A4A02EB95
:105F8000C000407981422CD19DF8B40040F2A111AB
:105F900010FB01F0114601EBC00000F562709DF8A6
:105FA000A01001EB410202EB011100EBC10090F8DF
:105FB0009400C0F34010A0B116229DF8B40040F246
:105FC000A11110FB01F0184901EBC00000F562704F
:105FD0009DF8A01001EB410303EB011100EBC100A0
:105FE0004271B3E014229DF8B40040F2A11110FBFD
:105FF00001F00D4901EBC00101F562719DF8A000AF
:1060000000EB400303EB001001EBC00042710121E3
:106010009DF8B40040F2A11210FB02F0024A02EB1C
:10602000C00003E0984000205845002001719DF811
:10603000B40000EB400101EB0010A2F5986101EB08
:10604000001130319DF8A00001EB0010801C099078
:10605000007820F0200020300999087076E01422A2
:106060009DF8B40040F2A11110FB01F0FE4901EBD4
:10607000C00000F562709DF8A01001EB410303EB36
:10608000011100EBC100427160E09DF8B40040F2E4
:10609000A11110FB01F0F44901EBC00000F56270A2
:1060A000BDF8D81001EB410202EB011100EBC10079
:1060B000807901282AD100229DF8B40040F2A11174
:1060C00010FB01F0E84901EBC00101F56271BDF878
:1060D000D80000EB400303EB001001EBC00082711D
:1060E00014229DF8B40040F2A11110FB01F0DE492A
:1060F00001EBC00000F562709DF8A01001EB4103B8
:1061000003EB011100EBC10042711FE000219DF87B
:10611000B40040F2A11210FB02F0D34A02EBC0001F
:10612000017105229DF8B40040F2A11110FB01F0AD
:10613000CD4901EBC00000F562709DF8A01001EBA5
:10614000410303EB011100EBC1004271FEE30121A9
:106150009DF8B40040F2A11210FB02F0C24A02EB1B
:10616000C000017114229DF8B40040F2A11110FB8F
:1061700001F0BD4901EBC00101F562719DF8A0007D
:1061800000EB400303EB001001EBC00042719DF8EF
:10619000B40000EB400101EB0010B44901EB001129
:1061A00030319DF8A00001EB0010801C09900078B0
:1061B00020F00400001D09990870C7E300202E900C
:1061C0002F90002139911FE0DDE92E10000240EAF6
:1061D00011620902CDE92E129DF8B40000EB4001D6
:1061E000C1EBC010A24901EBC001BDF8E400401DA5
:1061F000085CDDE92E3440EA0302CDE92E24BDF827
:10620000E400401C81B23991BDF8E4000328DBDBD7
:10621000DDE92E0111F0F8FA01469DF8B40040F2D4
:10622000A11210FB02F0904A02EBC00202F562726A
:106230009DF8A00000EB400303EB001002EBC00050
:10624000C0F81E1000222E922F92002139911EE0DC
:10625000DDE92E10000240EA11620902CDE92E129A
:106260009DF8B40000EB4001C1EBC010804901EB88
:10627000C001BDF8E4000830085CDDE92E341843A5
:10628000CDE92E04BDF8E400401C80B23990BDF881
:10629000E4000328DCDBDDE92E0111F0B5FA01464C
:1062A0009DF8B40040F2A11210FB02F06E4A02EB1E
:1062B000C00202F562729DF8A00000EB400303EB00
:1062C000001002EBC000C0F81A1000222E922F928C
:1062D000002139911EE0DDE92E10000240EA116232
:1062E0000902CDE92E129DF8B40000EB4001C1EB8C
:1062F000C0105F4901EBC001BDF8E4001330085C39
:10630000DDE92E341843CDE92E04BDF8E400401C2D
:1063100080B23990BDF8E4000328DCDB9DF8B400BE
:106320002E9940F2A11210FB02F04F4A02EBC0027C
:1063300002F562729DF8A00000EB400303EB001031
:1063400002EBC000416307229DF8B40040F2A111A6
:1063500010FB01F0444901EBC00000F562709DF8AC
:10636000A01001EB410303EB011100EBC1004271EE
:10637000ECE200202E902F90002139911FE0DDE902
:106380002E10000240EA11620902CDE92E129DF89A
:10639000B40000EB4001C1EBC010354901EBC00176
:1063A000BDF8E400401D085CDDE92E3440EA03023C
:1063B000CDE92E24BDF8E400401C81B23991BDF82E
:1063C000E4000428DBDBDDE92E0111F01DFA9DF865
:1063D000B42000E0FEE340F2A11312FB03F2224BD3
:1063E00003EBC20303F562739DF8A02002EB4204A5
:1063F00004EB021203EBC20222329060D160002152
:106400002E912F91002039901EE0DDE92E10000220
:1064100040EA11620902CDE92E129DF8B40000EBAA
:106420004001C1EBC010124901EBC001BDF8E4000E
:106430000930085CDDE92E341843CDE92E04BDF89F
:10644000E400401C80B23990BDF8E4000428DCDB95
:10645000DDE92E0111F0D8F99DF8B42040F2A11326
:1064600012FB03F2004B05E0584500209840002045
:10647000F887002003EBC20303F562739DF8A020A8
:1064800002EB420404EB021203EBC20242F8220FB9
:1064900051609DF8B40040F2A11110FB01F0FE49DB
:1064A00001EBC00000F562709DF8A01001EB410205
:1064B00002EB011110F831009DF8B41040F2A11266
:1064C00011FB02F1F44A02EBC101497988427CD107
:1064D0009DF8B40040F2A11110FB01F0114601EB50
:1064E000C00000F562709DF8A01001EB410202EBC4
:1064F000011100EBC10090F89400C0F34010A8B166
:1065000017229DF8B40040F2A11110FB01F0E249FE
:1065100001EBC00000F562709DF8A01001EB410393
:1065200003EB011100EBC100427114E014229DF84D
:10653000B40040F2A11110FB01F0D74901EBC000FB
:1065400000F562709DF8A01001EB410303EB01110F
:1065500000EBC10042719DF8B4009DF8A01001EB62
:106560000010C217CDE92E02CC4890F8E00708B31E
:106570009DF8B40000EB400101EB0010C84901EBAD
:10658000001030309DF8A01000EB0110807A022836
:1065900010D09DF8B40000EB400101EB0010C049A1
:1065A00001EB001030309DF8A01000EB0110C07A14
:1065B00000287CDD00229DF8B40040F2A11110FB00
:1065C00001F0B54901EBC00100E02FE301F5627174
:1065D0009DF8A00000EB400303EB001001EBC000AE
:1065E00080F846209DF8B40000EB400101EB00105C
:1065F000AB4901EB001130319DF8A00001EB001018
:10660000C272A848D0F80C020521B0FBF1F201FBE0
:10661000120000EB4001A3482C3000EB41100D307C
:1066200009909DF8B40040F2A11110FB01F09A49C5
:1066300001EBC00000F562709DF8A01001EB410273
:1066400002EB011100EBC10022301022014608903C
:106650000998F1F7FAFD9348D0F80C020521B0FB38
:10666000F1F201FB120000EB40018E482C3000EBF0
:1066700041129DF8B40040F2A11110FB01F08649CF
:1066800001EBC00101F562719DF8A00000EB400331
:1066900003EB001001EBC00050F81A1F42F8011F75
:1066A000406850607F48D0F80C02052100E0AAE164
:1066B000B0FBF1F201FB120000EB400179482C30F5
:1066C00000EB41129DF8B40000EB400101EB00101B
:1066D000734901EB001130319DF8A00001EB00106F
:1066E000007810706F48D0F80C020521B0FBF1F271
:1066F00001FB120000EB40016A482C3000EB411214
:106700009DF8B40040F2A11110FB01F0624901EBC9
:10671000C00101F562719DF8A00000EB400303EB9E
:10672000001001EBC000406BC2F809005D48D0F8D2
:106730000C020521B0FBF1F201FB120000EB40015D
:1067400058482C3000EB41115448F538026841F8A4
:106750001D2F808888805348D0F80C020521B0FB9B
:10676000F1F201FB120000EB40014E482C3000EB2F
:1067700041129DF8B40000EB400101EB00104849C4
:1067800001EB001130319DF8A00001EB00104068D2
:10679000C2F8230000229DF8B40000EB400101EB99
:1067A00000103F4901EB001130319DF8A00001EBD2
:1067B000001042600021399154E03A48D0F80C02B0
:1067C0000521B0FBF1F201FB120000EB400135485E
:1067D0002C3000EB41112731BDF8E4409DF8B400A6
:1067E00040F2A11210FB02F02B4A02EBC00202F5AC
:1067F00062729DF8A00000EB400303EB001002EB77
:10680000C00090F8800040F2A11210FB02F0224A72
:1068100002EBC00202F562729DF8B40040F2A113CF
:1068200010FB03F01C4B03EBC00303F562739DF8F0
:10683000A00000EB400505EB001003EBC00090F852
:10684000810000EB400303EB001002EBC002473273
:10685000BDF8E400001D105C0855BDF8E400401CC4
:1068600081B23991BDF8E4000628A6DB00203990FA
:106870004BE000239DF8B40040F2A11110FB01F0A1
:10688000054901EBC00101F562719DF8A00000EB24
:10689000400202EB001007E058450020BC32002007
:1068A00098400020BC12002001EBC00090F880004E
:1068B00040F2A11110FB01F0FE4901EBC00101F50E
:1068C00062719DF8B40040F2A11210FB02F0F94A87
:1068D00002EBC00202F562729DF8A00000EB4004DA
:1068E00004EB001002EBC00090F8810000EB4002C6
:1068F00002EB001001EBC0014731BDF8E4000B547E
:10690000BDF8E400401C81B23991BDF8E4000A28CA
:10691000AFDBE948D0F80C020521B0FBF1F080B202
:10692000014609900220F2F7D3FB00210620F3F77D
:10693000BDFBE148D0F80C02DF49498D884208D2FE
:10694000DD48D0F80C02401CDB4900E001E2C1F850
:106950000C0200210520F3F7A9FB9DF8B40000EB21
:10696000400101EB0010D54901EB001030309DF8DB
:10697000A01000EB0110801C0990007820F00802A4
:1069800009980270CC48D0F80C020521B0FBF1F256
:1069900001FB120000EB4001C7482C3000EB411016
:1069A000D0F823202E9800EB4001C54800EB4110A1
:1069B000C0F823200020399020E0BF48D0F80C0216
:1069C0000521B0FBF1F201FB120000EB4001BA48D7
:1069D0002C3000EB41102730BDF8E410425C2E98BB
:1069E00000EB4001B64800EB41112731BDF8E4004F
:1069F0000A54BDF8E400401C81B23991BDF8E400AE
:106A00000628DADB6FE000229DF8B40040F2A11105
:106A100010FB01F0A74901EBC00101F562719DF87F
:106A2000A00000EB400303EB001001EBC00080F876
:106A300046209DF8B40000EB400101EB00109F4997
:106A400001EB001130319DF8A00001EB0010801C1B
:106A50000990007820F008000830099908709DF826
:106A6000B40000EB400101EB0010944901EB001071
:106A700030309DF8A01000EB011042682E9800EB1A
:106A800040018F4800EB4110C0F8232000203990CE
:106A900025E09DF8B40040F2A11110FB01F08549FA
:106AA00001EBC00101F562719DF8A00000EB40020E
:106AB00002EB001001EBC0014731BDF8E4000A5CB5
:106AC0002E9800EB40017E4800EB41112731BDF8C4
:106AD000E4000A54BDF8E400401C81B23991BDF8CD
:106AE000E4000628D5DB9DF8B4100220F3F7DEFAA7
:106AF0009DF8B40040F2A11110FB01F06D4901EBCB
:106B0000C00101F562719DF8A00000EB400202EBAC
:106B1000001001EBC000223009902E9800EB4001DC
:106B2000674800EB41100D30102208900999F1F7E9
:106B30008CFB9DF8B40040F2A11110FB01F05D49FF
:106B400001EBC00101F562719DF8A00000EB40026D
:106B500002EB001001EBC0012E9800EB40025848F8
:106B600000EB421051F81A2F40F8012F496841609C
:106B70009DF8B40000EB400101EB00104F4901EB20
:106B8000001130319DF8A00001EB001001782E9823
:106B900000EB40024A4800EB421001702E9800EBD7
:106BA0004001474800EB41114648026841F81D2F5B
:106BB000808888809DF8B40040F2A11110FB01F09C
:106BC0003C4901EBC00101F562719DF8A00000EBAA
:106BD000400200E043E102EB001001EBC000416B1A
:106BE0002E9800EB4002364800EB4210C0F8091026
:106BF0009DF8B40000EB400101EB00102F4901EBC0
:106C0000001130319DF8A00001EB001041682E9872
:106C100000EB40022A4800EB4210C0F823102E98E7
:106C200081B208200991F3F741FA92E09DF8B4008F
:106C300040F2A11110FB01F01E4901EBC00101F56A
:106C400062719DF8A00000EB400202EB001011F809
:106C500030109DF8B40040F2A11210FB02F0154A6A
:106C600002EBC0004079814273DA9DF8B40000EB7A
:106C7000400101EB0010114901EB001030309DF88C
:106C8000A01000EB0110801C0990007820F0040097
:106C9000001D099908709DF8B40000EB400101EB5C
:106CA0000010064901EB001030309DF8A01000EBF9
:106CB000011009E058450020BC1200209840002037
:106CC000D8140020C7310020801C0990007820F0E3
:106CD000800080300999087001209DF8B41040F2BE
:106CE000A11211FB02F1FE4A02EBC10108719DF8ED
:106CF000B40040F2A11110FB01F0114601EBC000FD
:106D000042799DF8B40040F2A11110FB01F0F44962
:106D100001EBC00000F562709DF8A01001EB41038B
:106D200003EB011100F8312014229DF8B40040F269
:106D3000A11110FB01F0EA4901EBC00000F56270FF
:106D40009DF8A01001EB410303EB011100EBC10022
:106D5000427183E00121E34880F804179DF8B400F4
:106D600040F2A11110FB01F0DD4901EBC00101F57A
:106D700062719DF8A00000EB400202EB001011F8D8
:106D800030109DF8B40040F2A11210FB02F0D44A7A
:106D900002EBC0004079814233DA00219DF8B40053
:106DA00040F2A11210FB02F0CD4A02EBC0000171CB
:106DB00001229DF8B40040F2A11110FB01F0C84976
:106DC00001EBC00101F562719DF8A00000EB4003EA
:106DD00003EB001001F8302014229DF8B40040F2BB
:106DE000A11110FB01F0BE4901EBC00000F562707B
:106DF0009DF8A01001EB410303EB011100EBC10072
:106E000042712BE014229DF8B40040F2A11110FB56
:106E100001F0B34901EBC00101F562719DF8A000DA
:106E200000EB400303EB001001EBC000427115E0E2
:106E300014229DF8B40040F2A11110FB01F0A84902
:106E400001EBC00000F562709DF8A01001EB41035A
:106E500003EB011100EBC100427100BF00BF07F05E
:106E6000D7B99DF8B40040F2A11110FB01F09C4984
:106E700001EBC000817828919DF8B40000EB40013F
:106E8000C1EBC010984911F8301029919DF8B40059
:106E900040F2A11110FB01F0914901EBC00101F595
:106EA00062719DF8A00000EB400202EB001001EBC4
:106EB000C000417925919DF8B40000EB4001C1EB81
:106EC000C010894901EBC0010991BDF8A4100998CF
:106ED000F3F784FE37909DF8B40000EB4001C1EB5E
:106EE000C010814901EBC001BDF8A400095CBDF8E8
:106EF000DC00814241F067879DF8B40000EB40015F
:106F0000C1EBC010784901EBC0004078002841F384
:106F10005A870021754A9DF8B40002EB00129DF8D3
:106F2000A0001154BDF8940089287DD00EDC1428EF
:106F300001F0298705DC082877D0102841F0428726
:106F4000FBE3152872D08028F8D1F8E38B286ED0A7
:106F50008C286DD08E286CD08F28EFD1BDF8A4007E
:106F60000D2867D19DF8B40000EB4001C1EBC010C3
:106F70005D4901EBC00041785D4880F8041D9DF833
:106F8000B40000EB4001C1EBC010574901EBC00059
:106F9000C17A574880F8051D9DF8B40040F2A11150
:106FA00010FB01F04E4901EBC00000F562709DF846
:106FB000A01001EB410202EB011110F8310003288F
:106FC0007EDC4B4890F8050D00287ADD9DF8B40072
:106FD00040F2A11110FB01F0414901EBC00101F5A4
:106FE00062719DF8A00000EB400202EB001001EB83
:106FF000C00109910878401CC1B2099801709DF840
:10700000B40040F2A11110FB01F0354901EBC000C2
:1070100000F562709DF8A01001EB410202EB011136
:1070200010F83100042806E0FEE3FEE3FEE3FEE391
:10703000FEE3FEE3FEE344DB9DF8B40000EB400119
:1070400001EB00102B4901EB001030309DF8A0102F
:1070500000EB0110801C0990254890F8050DC0F345
:107060000010C0F101000999097860F30001099846
:1070700001701F4890F8040DC0F3C00078BB9DF864
:10708000B40000EB400101EB00101A4901EB0010C5
:1070900030309DF8A01000EB01108078C0F3401054
:1070A000E8B19DF8B40000EB400101EB001011497C
:1070B00001EB001030309DF8A01000EB011001E052
:1070C0006BE007E1801C0990007820F00200801C32
:1070D000099908709DF8B40040F2A1110CE027E076
:1070E00058450020BC320020F8870020883E002050
:1070F000BC2200209840002010FB01F0FE4901EB6B
:10710000C00000F562709DF8A01001EB410202EB97
:10711000011100EBC10018300990007820F0020046
:10712000801C099908709DF8B4100220F2F7BEFF88
:1071300000219DF8B40040F2A11210FB02F0EE4ACB
:1071400002EBC000017104229DF8B40040F2A111CD
:1071500010FB01F0E84901EBC00101F562719DF8F7
:10716000A00000EB400303EB001001F830208C225C
:107170009DF8B40040F2A11110FB01F0DE4901EBD3
:10718000C00000F562709DF8A01001EB410303EB15
:10719000011100EBC10042719CE09DF8B40040F287
:1071A000A11110FB01F0D44901EBC00101F562719E
:1071B0009DF8A00000EB400202EB001011F8301027
:1071C0009DF8B40040F2A11210FB02F0CA4A02EB93
:1071D000C000407981427DD19DF8B40000EB4001B0
:1071E00001EB0010A2F5986101EB001030309DF822
:1071F000A01000EB0110801C0990C04890F8050D0C
:10720000C0F30010C0F101010998027861F3000297
:1072100002709DF8B40000EB400101EB0010B8498A
:1072200001EB001130319DF8A00001EB0010801C33
:107230000990B24890F8040DC2080998017862F3E9
:10724000410101709DF8B40000EB400101EB00101A
:10725000AB4901EB001130319DF8A00001EB0010AB
:107260008078C0F340029DF8B40040F2A11110FBF9
:1072700001F0A14901EBC00000F562709DF8A0107B
:1072800001EB410303EB011100EBC100007EC0F3F1
:10729000400082426CD09DF8B40040F2A11110FB76
:1072A00001F0954901EBC00000F562709DF8A01057
:1072B00001EB410202EB011100EBC1001830099013
:1072C0009DF8B41001EB410000EB01108C4901EB7B
:1072D000001100E0C6E330319DF8A00001EB001082
:1072E000807842080998017862F3410101709DF8A5
:1072F000B40000EB400101EB0010814901EB0010EC
:1073000030309DF8A01000EB01108078C0F34000F1
:1073100048BB01229DF8B40040F2A11110FB01F01E
:10732000754901EBC00101F562719DF8A00000EB09
:10733000400303EB001001EBC00042739DF8B40062
:1073400040F2A11110FB01F06B4901EBC00000F508
:1073500062709DF8A01001EB410303EB011100EBFB
:10736000C10080F846209DF8B4100220F2F79EFE7E
:107370009DF8B40000EB400101EB0010604901EB07
:10738000001130319DF8A00001EB0010807800F072
:1073900001029DF8B40040F2A11110FB01F0564922
:1073A00001EBC00000F562709DF8A01001EB4103F5
:1073B00003EB011100EBC100007E00F001008242EE
:1073C00079D09DF8B40040F2A11110FB01F04A49B8
:1073D00001EBC00000F562709DF8A01001EB4102C6
:1073E00002EB011100EBC100183009909DF8B400C8
:1073F00000EB400101EB0010414901EB001130317D
:107400009DF8A00001EB001081780998027861F3E3
:10741000000202709DF8B40000EB400101EB001087
:10742000374901EB001030309DF8A01000EB01103F
:10743000807800F00100E8BB9DF8B40000EB40014B
:1074400001EB00102E4901EB001030309DF8A01028
:1074500000EB01108078C0F3401068B39DF8B400D1
:1074600040F2A11110FB01F0234901EBC00000F52F
:1074700062709DF8A01001EB410202EB011100EBDC
:10748000C10090F84600B8B99DF8B40040F2A111CF
:1074900010FB01F0184901EBC00000F562709DF887
:1074A000A01001EB410202EB011100EBC100407B97
:1074B00010B902E05BE05FE242E09DF8B40000EB4F
:1074C000400101EB00100E4901EB001030309DF837
:1074D000A01000EB01108078C0F3400080BB0122B7
:1074E0009DF8B40040F2A11110FB01F0024901EB3C
:1074F000C00101F5627105E058450020BC22002062
:10750000984000209DF8A00000EB400303EB001022
:1075100001EBC00042739DF8B40040F2A11110FBD2
:1075200001F0FE4901EBC00000F562709DF8A0106B
:1075300001EB410303EB011100EBC10080F8462091
:1075400000229DF8B40040F2A11110FB01F0F349B4
:1075500001EBC00000F562709DF8A01001EB410343
:1075600003EB011100EBC10080F84520FFE19DF81D
:10757000B40040F2A11110FB01F0E84901EBC0009A
:1075800000F562709DF8A01001EB410202EB0111C1
:1075900000EBC10090F84600B0B901229DF8B4009C
:1075A00040F2A11110FB01F0DC4901EBC00000F535
:1075B00062709DF8A01001EB410303EB011100EB99
:1075C000C10080F845202AE000229DF8B40040F276
:1075D000A11110FB01F0D14901EBC00101F562716D
:1075E0009DF8A00000EB400303EB001001EBC0008E
:1075F00080F845209DF8B40000EB400101EB00103D
:10760000C74901EB001130319DF8A00001EB0010DB
:10761000801C0990007820F0010209980270C1488E
:1076200090F8E00780B19DF8B40000EB400101EB59
:107630000010BB4901EB001030309DF8A01000EBAA
:107640000110807A022879D1B74890F829000128E2
:1076500074D1B548D0F80C02B349498D88426DD237
:107660009DF8B40040F2A11110FB01F0AB4901EB11
:10767000C00000F562709DF8A01001EB410202EB22
:10768000011100EBC10090F84500012854D19DF88C
:10769000B40040F2A11110FB01F0A04901EBC000C1
:1076A00000F562709DF8A01001EB410202EB0111A0
:1076B00000EBC10090F87F00F0BB01229DF8B40000
:1076C00000EB400101EB0010954901EB0011303156
:1076D0009DF8A00001EB0010C2729DF8B40000EB11
:1076E000400101EB00108E4901EB001130319DF893
:1076F000A00001EB001001789DF8B40040F2A11247
:1077000010FB02F0854A02EBC000417008229DF890
:10771000B40040F2A11110FB01F0804901EBC0015F
:1077200001F562719DF8A00000EB400303EB00102F
:1077300001EBC000427103E060E024E3F6E0FDE30A
:1077400000229DF8B40000EB400101EB00107449E9
:1077500001EB001130319DF8A00001EB00104260F8
:107760009DF8B4100220F2F7A1FC002139911CE031
:1077700000229DF8B40040F2A11110FB01F067490E
:1077800001EBC00101F562719DF8A00000EB400320
:1077900003EB001001EBC0014731BDF8E4000A54CF
:1077A000BDF8E400401C81B23991BDF8E400142812
:1077B000DEDB002039901CE000229DF8B40040F28E
:1077C000A11110FB01F0554901EBC00101F56271F7
:1077D0009DF8A00000EB400303EB001001EBC0019B
:1077E0006331BDF8E4000A54BDF8E400401C81B2E6
:1077F0003991BDF8E4000A28DEDBB8E09DF8B4005A
:1078000040F2A11110FB01F0444901EBC00000F56A
:1078100062709DF8A01001EB410202EB011100EB38
:10782000C10090F8450006E0C7E27FE2FEE32AE3EC
:1078300091E3FCE379E2012878D19DF8B40040F2AD
:10784000A11110FB01F0354901EBC00101F5627196
:107850009DF8A00000EB400202EB001001EBC0001D
:1078600090F8800040F2A11110FB01F02B4901EBD0
:10787000C00101F562719DF8B40040F2A11210FB45
:1078800002F0264A02EBC00000F562709DF8A020CD
:1078900002EB420303EB021200EBC20090F88100FE
:1078A00000EB400202EB001001EBC00090F87E00FC
:1078B00003285CD102229DF8B40000EB400101EBEB
:1078C0000010174901EB001130319DF8A00001EBC9
:1078D0000010C2729DF8B40000EB400101EB0010F3
:1078E0000F4901EB001130319DF8A00001EB0010B1
:1078F00001789DF8B40040F2A11210FB02F0074A93
:1079000002EBC000417008229DF8B40040F2A111C2
:1079100010FB01F0014901EBC00108E058450020CF
:1079200098400020BC320020BC1200201FE001F56E
:1079300062719DF8A00000EB400303EB001001EB27
:10794000C000427100229DF8B40000EB400101EB41
:107950000010FE4901EB001130319DF8A00001EB51
:10796000001042609DF8B4100220F2F79FFB9DF8D2
:10797000B4100220F2F79AFB9DF8B40040F2A11176
:1079800010FB01F0F24901EBC00000F562709DF8B8
:10799000A01001EB410202EB011100EBC100807865
:1079A000802838D19DF8B40000EB400101EB0010B5
:1079B000E64901EB001030309DF8A01000EB0110FB
:1079C0008078C0F3400030BB9DF8B40000EB40016C
:1079D00001EB0010DD4901EB001030309DF8A010E4
:1079E00000EB01108078C0F34010A0B915229DF87B
:1079F000B40040F2A11110FB01F0D54901EBC00029
:107A000000F562709DF8A01001EB410303EB01113A
:107A100000EBC10042719DF8B40000EB400101EBA6
:107A20000010CA4901EB001030309DF8A01000EBA7
:107A300001108078C0F34000A8B18F229DF8B400F7
:107A400040F2A11110FB01F0C14901EBC00000F5AB
:107A500062709DF8A01001EB410303EB011100EBF4
:107A6000C10042714AE09DF8B40040F2A11110FB40
:107A700001F0B74901EBC00000F562709DF8A0105D
:107A800001EB410202EB011100EBC100807B0128F8
:107A900034D100229DF8B40040F2A11110FB01F096
:107AA000AB4901EBC00101F562719DF8A00000EB4C
:107AB000400303EB001001EBC00082738C229DF8A1
:107AC000B40040F2A11110FB01F0A14901EBC0018B
:107AD00001F562719DF8A00000EB400303EB00107C
:107AE00001EBC000427100219DF8B40040F2A112E8
:107AF00010FB02F0964A02EBC00001719DF8B40041
:107B000000EB400101EB0010904901EB0010007BFD
:107B1000F0BB9DF8B40000EB4001C1EBC0108D49F3
:107B200001EBC000807801049DF8B40000EB400236
:107B3000C2EBC010874A02EBC000C07841EA0021C6
:107B40009DF8B40000EB4002C2EBC010814A02EB8A
:107B5000C00000790843C117CDE908010FF054FEB9
:107B60009DF8B41040F2A11211FB02F1784A02EB29
:107B7000C10202F562729DF8A01001EB410303EB14
:107B8000011102EBC101C1F81E009DF8B40000E034
:107B90003AE000EB4001C1EBC0106E4901EBC000C0
:107BA000407900049DF8B41001EB4102C2EBC11111
:107BB000684A02EBC101897940EA01209DF8B410BE
:107BC00001EB4102C2EBC111624A02EBC101C9796A
:107BD0000843C117CDE908010FF016FE9DF8B41057
:107BE00040F2A11211FB02F1594A02EBC10101F569
:107BF00062719DF8A02002EB420303EB021201EB3D
:107C0000C201C1F81A0090E09DF8B40000EB4001F9
:107C1000C1EBC0104F4901EBC000807801069DF810
:107C2000B40000EB4002C2EBC0104A4A02EBC000B5
:107C3000C07841EA00419DF8B40000EB4002C2EB7D
:107C4000C010444A02EBC000007941EA00219DF8CF
:107C5000B40000EB4002C2EBC0103E4A02EBC00091
:107C600040790843C117CDE908010FF0CDFD014669
:107C70009DF8B40040F2A11210FB02F0344A02EB6E
:107C8000C00202F562729DF8A00000EB400303EB16
:107C9000001002EBC000C0F81E109DF8B40000EB0D
:107CA0004001C1EBC0102B4901EBC00080790106F7
:107CB0009DF8B40000EB4002C2EBC010254A02EB75
:107CC000C000C07941EA00419DF8B40000EB4002D9
:107CD000C2EBC0101F4A02EBC000007A41EA00214B
:107CE0009DF8B40000EB4002C2EBC010194A02EB51
:107CF000C000407A0843C117CDE908010FF084FDA8
:107D00009DF8B41040F2A11211FB02F1104A02EBEF
:107D1000C10101F562719DF8A02002EB420303EB63
:107D2000021201EBC201C1F81A0023E2BDF8A4005F
:107D3000032827D18F229DF8B40040F2A11110FB37
:107D400001F0034901EBC00106E00000984000206B
:107D500058450020F887002001F562719DF8A000C9
:107D600000EB400303EB001001EBC0004271012166
:107D70009DF8B40040F2A11210FB02F0FE4A02EBA3
:107D8000C0000171F6E1BDF8A400032814D18F22D0
:107D90009DF8B40040F2A11110FB01F0F64901EB8F
:107DA000C00000F562709DF8A01001EB410303EBE9
:107DB000011100EBC1004271DCE1BDF8A400032811
:107DC00060D19DF8B40040F2A11110FB01F0EA4926
:107DD00001EBC00000F56270BDF8D81001EB410264
:107DE00002EB011100EBC100807901282AD10022A9
:107DF0009DF8B40040F2A11110FB01F0DE4901EB47
:107E0000C00101F56271BDF8D80000EB400303EB3F
:107E1000001001EBC00082718F229DF8B40040F287
:107E2000A11110FB01F0D44901EBC00000F5627014
:107E30009DF8A01001EB410303EB011100EBC10021
:107E400042711FE008229DF8B40040F2A11110FB1E
:107E500001F0C94901EBC00101F562719DF8A00074
:107E600000EB400303EB001001EBC0004271002166
:107E70009DF8B40040F2A11210FB02F0BE4A02EBE2
:107E8000C000017176E1BDF8A400032862D19DF81D
:107E9000B40040F2A11110FB01F0B74901EBC000A2
:107EA00000F56270BDF8D81001EB410202EB011140
:107EB00000EBC100807901282AD100229DF8B4008E
:107EC00040F2A11110FB01F0AB4901EBC00101F53B
:107ED0006271BDF8D80000EB400303EB001001EB2A
:107EE000C00082718F229DF8B40040F2A11110FBF6
:107EF00001F0A14901EBC00000F562709DF8A010EF
:107F000001EB410303EB011100EBC100427121E0E1
:107F100008229DF8B40040F2A11110FB01F096492F
:107F200001EBC00101F562719DF8A00000EB400378
:107F300003EB001001EBC000427100E020E10021E2
:107F40009DF8B40040F2A11210FB02F08A4A02EB45
:107F5000C00001710EE1BDF8A400082868D19DF8A9
:107F6000B40000EB4001C1EBC010844901EBC0003C
:107F7000807801069DF8B40000EB4002C2EBC0100F
:107F80007E4A02EBC000C07841EA00419DF8B4008F
:107F900000EB4002C2EBC010784A02EBC00000794F
:107FA00041EA00219DF8B40000EB4002C2EBC01092
:107FB000724A02EBC00040790843C117CDE90801BD
:107FC0000FF022FC9DF8B41040F2A11211FB02F157
:107FD000694A02EBC10202F562729DF8A01001EB42
:107FE000410303EB011102EBC10148639DF8B400AA
:107FF00040F2A11110FB01F05F4901EBC00000F558
:1080000062709DF8A01001EB410202EB011110F823
:1080100031209DF8B40040F2A11110FB01F0564947
:1080200001EBC0004079824238DA02E0FEE3E1E091
:10803000A0E000219DF8B40040F2A11210FB02F074
:108040004D4A02EBC000017105229DF8B40040F2D8
:10805000A11110FB01F0484901EBC00101F562716B
:108060009DF8A00000EB400303EB001001F8302066
:108070008E229DF8B40040F2A11110FB01F03E49A0
:1080800001EBC00000F562709DF8A01001EB410308
:1080900003EB011100EBC10042716BE09DF8B400ED
:1080A00040F2A11110FB01F0334901EBC00000F5D3
:1080B0006270BDF8D81001EB410202EB011100EB38
:1080C000C1008079012835D100229DF8B40040F22A
:1080D000A11110FB01F0284901EBC00101F562710B
:1080E000BDF8D80000EB400303EB001001EBC0002B
:1080F00082718F229DF8B40040F2A11110FB01F0B3
:108100001D4901EBC00101F562719DF8A00000EB73
:10811000400303EB001001EBC000427101219DF808
:10812000B40040F2A11210FB02F0134A02EBC000AF
:1081300001711FE08E229DF8B40040F2A11110FBE6
:1081400001F00D4901EBC00101F562719DF8A0003D
:1081500000EB400303EB001001EBC0004271002173
:108160009DF8B40040F2A11210FB02F0024A02EBAB
:10817000C0000171EFE3000058450020F88700209F
:10818000BDF8A400032834D100219DF8B40040F2CA
:10819000A11210FB02F0FE4A02EBC00001710122A5
:1081A0009DF8B40040F2A11110FB01F0F84901EB79
:1081B000C00101F56271BDF8D80000EB400303EB8C
:1081C000001001EBC00082718C229DF8B40040F2D7
:1081D000A11110FB01F0EE4901EBC00101F5627144
:1081E0009DF8A00000EB400303EB001001EBC00082
:1081F0004271B0E3BDF8A4000F287CD19DF8B40013
:1082000000EB400101EB0010E24901EB0010007BA4
:10821000E8BB00202E902F90002139911FE0DDE96E
:108220002E10000240EA11620902CDE92E129DF8DB
:10823000B41001EB4100C0EBC110D74901EBC00104
:10824000BDF8E400C0F10600085CDDE92E341843F7
:10825000CDE92E04BDF8E400401C80B23990BDF891
:10826000E4000528DBDB9DF8B400DDE92E2140F2B7
:10827000A11310FB03F0C64B03EBC00303F56273BD
:108280009DF8A00000EB400404EB001000E04AE081
:1082900003EBC00040F8222F416000222E922F9263
:1082A0000021399120E0DDE92E10000240EA116240
:1082B0000902CDE92E129DF8B41001EB4100C0EB8C
:1082C000C110B54901EBC001BDF8E400C0F10B00DD
:1082D000085CDDE92E3440EA0302CDE92E24BDF826
:1082E000E400401C81B23991BDF8E4000528DADBD6
:1082F0009DF8B40000E0FCE3DDE92E1240F2A1138A
:1083000010FB03F0A24B03EBC00000F562709DF878
:10831000A03003EB430404EB031300EBC300223053
:108320008160C26085E000202E902F90002139915D
:1083300020E0DDE92E10000240EA11620902CDE9D9
:108340002E129DF8B41001EB4100C0EBC110924910
:1083500001EBC001BDF8E400C0F10700085CDDE9F5
:108360002E3440EA0302CDE92E24BDF8E400401C7F
:1083700081B23991BDF8E4000628DADB9DF8B4003B
:10838000DDE92E1240F2A11310FB03F0804B03EB4A
:10839000C00303F562739DF8A00000EB400404EBFA
:1083A000001003EBC00040F8221F426000222E9212
:1083B0002F920021399120E0DDE92E10000240EAE1
:1083C00011620902CDE92E129DF8B41001EB4100B3
:1083D000C0EBC110704901EBC001BDF8E400C0F171
:1083E0000D00085CDDE92E3440EA0302CDE92E24BD
:1083F000BDF8E400401C81B23991BDF8E4000628C4
:10840000DADB9DF8B400DDE92E1240F2A11310FB77
:1084100003F05F4B03EBC00000F562709DF8A030E5
:1084200003EB430404EB031300EBC3002230816031
:10843000C2609DF8B41040F2A11011FB00F0544945
:1084400001EBC00101F562719DF8A00000EB400254
:1084500002EB001011F830109DF8B40040F2A112A8
:1084600010FB02F04A4A02EBC000407981427DD104
:108470009DF8B4009DF8A01001EB0010C217CDE9E3
:108480002E02464890F8E00708B39DF8B41001EBBF
:10849000410000EB01103F4901EB001030309DF826
:1084A000A01000EB0110807A022810D09DF8B410C3
:1084B00001EB410000EB0110364901EB00103030B8
:1084C0009DF8A01000EB0110C07A00285FDD0022AB
:1084D0009DF8B40000EB400101EB00102D4901EBC9
:1084E000001030309DF8A01000EB0110C2722C4833
:1084F000D0F80C020521B0FBF1F201FB120000EBF9
:10850000400127482C3000EB41100D3009909DF8B8
:10851000B41040F2A11011FB00F01D4901EBC000A6
:1085200000F562709DF8A01001EB410202EB011111
:1085300000EBC10022301022014608900998EFF7A5
:1085400084FE1748D0F80C020521B0FBF1F201FBC4
:10855000120000EB400112482C3000EB41129DF854
:10856000B40040F2A11110FB01F000E0F8E208496C
:1085700001EBC00101F562719DF8A00000EB400322
:1085800003EB001001EBC00050F81A1F0AE0B2E143
:108590005845002098400020F8870020BC32002079
:1085A000BC12002042F8011F40685060FE48D0F81D
:1085B0000C020521B0FBF1F201FB120000EB4001BF
:1085C000F9482C3000EB41129DF8B40000EB40015B
:1085D00001EB0010F54901EB001130319DF8A000CE
:1085E00001EB001000781070EF48D0F80C02052164
:1085F000B0FBF1F201FB120000EB4001EA482C3025
:1086000000EB4111EA48026841F81D2F80888880FC
:10861000E548D0F80C020521B0FBF1F201FB120095
:1086200000EB4001E0482C3000EB41129DF8B40013
:1086300040F2A11110FB01F0DE4901EBC00101F590
:1086400062719DF8A00000EB400303EB001001EB0A
:10865000C000406BC2F80900D348D0F80C020521D5
:10866000B0FBF1F201FB120000EB4001CE482C30D0
:1086700000EB41129DF8B40000EB400101EB00104B
:10868000CA4901EB001130319DF8A00001EB001048
:108690004068C2F8230000229DF8B40000EB4001BE
:1086A00001EB0010C14901EB001130319DF8A00031
:1086B00001EB001042600021399154E0BA48D0F833
:1086C0000C020521B0FBF1F201FB120000EB4001AE
:1086D000B5482C3000EB41112731BDF8E4409DF83E
:1086E000B40040F2A11210FB02F0B24A02EBC00249
:1086F00002F562729DF8A00000EB400303EB00104E
:1087000002EBC00090F8800040F2A11210FB02F0D2
:10871000A84A02EBC00202F562729DF8B40040F272
:10872000A11310FB03F0A34B03EBC00303F562732B
:108730009DF8A00000EB400505EB001003EBC00026
:1087400090F8810000EB400303EB001002EBC00245
:108750004732BDF8E400001D105C0855BDF8E40088
:10876000401C81B23991BDF8E4000628A6DB002048
:10877000399042E000239DF8B40040F2A11110FBB3
:1087800001F08C4901EBC00101F562719DF8A00078
:1087900000EB400202EB001001EBC00090F88000FB
:1087A00040F2A11110FB01F0824901EBC00101F57B
:1087B00062719DF8B40040F2A11210FB02F07D4AF4
:1087C00002EBC00202F562729DF8A00000EB4004CB
:1087D00004EB001002EBC00090F8810000EB4002B7
:1087E00002EB001001EBC0014731BDF8E4000B546F
:1087F000BDF8E400401C81B23991BDF8E4000A28BC
:10880000B8DB6948D0F80C020521B0FBF1F080B26A
:10881000014609900220F0F75BFC00210620F1F7E9
:1088200045FC6148D0F80C025F4900E002E2498D46
:10883000884206D25C48D0F80C02401C5A49C1F864
:108840000C0200210520F1F731FC9DF8B41001EB7A
:10885000410000EB0110554901EB001030309DF84C
:10886000A01000EB0110801C0990007820F0080295
:10887000099802704C48D0F80C020521B0FBF1F2C7
:1088800001FB120000EB400147482C3000EB411087
:10889000D0F823202E9800EB4001474800EB411010
:1088A000C0F823200020399020E03F48D0F80C0287
:1088B0000521B0FBF1F201FB120000EB40013A4848
:1088C0002C3000EB41102730BDF8E410425C2E98AC
:1088D00000EB4001384800EB41112731BDF8E400BE
:1088E0000A54BDF8E400401C81B23991BDF8E4009F
:1088F0000628DADB66E09DF8B41001EB410000EBDE
:1089000001102A4901EB001030309DF8A01000EB57
:108910000110801C0990007820F0080008300999A7
:1089200008709DF8B41001EB410000EB01101F49E5
:1089300001EB001030309DF8A01000EB01104268F0
:108940002E9800EB40011C4800EB4110C0F823209A
:108950000020399026E015E29DF8B41040F2A110F5
:1089600011FB00F0134901EBC00101F562719DF8A4
:10897000A00000EB400202EB001001EBC001473108
:10898000BDF8E4000A5C2E9800EB40010A4800EBB9
:1089900041112731BDF8E4000A54BDF8E400401C41
:1089A00081B239910AE00000BC12002098400020FA
:1089B000C731002058450020D8140020BDF8E4003D
:1089C0000628C9DB9DF8B41001EB410000EB011053
:1089D000FE4901EB001030309DF8A01000EB0110B3
:1089E000801C0990007820F02002099802709DF800
:1089F000B4100220F1F75AFB9DF8B41040F2A11018
:108A000011FB00F0F24901EBC00000F562709DF827
:108A1000A01001EB410202EB011100EBC10022307A
:108A200009902E9800EB4001EA4800EB41100D3010
:108A3000102208900999EFF708FC9DF8B41040F255
:108A4000A11011FB00F0E24901EBC00101F56271D8
:108A50009DF8A00000EB400202EB001001EBC0010A
:108A60002E9800EB4002DB4800EB421051F81A2F21
:108A700040F8012F496841609DF8B40000EB4001C7
:108A800001EB0010D14901EB001130319DF8A0003D
:108A900001EB001001782E9800EB4002CD4800EB6E
:108AA000421001702E9800EB4001CA4800EB4111C2
:108AB000C948026841F81D2F808888809DF8B4005D
:108AC00040F2A11110FB01F0C14901EBC00101F519
:108AD00062719DF8A00000EB400202EB001001EB78
:108AE000C000416B2E9800EB4002BA4800EB4210E8
:108AF00000E09EE0C0F809109DF8B40000EB4001D2
:108B000001EB0010B14901EB001130319DF8A000DC
:108B100001EB001041682E9800EB4002AD4800EBDD
:108B20004210C0F823102E9881B208200991F1F765
:108B3000BDFA00229DF8B40040F2A11110FB01F033
:108B4000A34901EBC00000F562709DF8A01001EB95
:108B5000410303EB011100EBC10080F8462053E014
:108B60009DF8B40000EB400101EB0010974901EBC8
:108B7000001030309DF8A01000EB0110801C09900F
:108B8000007820F00401091D099801709DF8B400D7
:108B900000EB400101EB00108C4901EB001130317A
:108BA0009DF8A00001EB0010801C0990007820F0D7
:108BB000800080300999087001209DF8B41040F2BF
:108BC000A11211FB02F1824A02EBC10108719DF86A
:108BD000B40040F2A11110FB01F0114601EBC000FE
:108BE00042799DF8B40040F2A11110FB01F07849E0
:108BF00001EBC00000F562709DF8A01001EB41038D
:108C000003EB011100F831208F229DF8B40040F2EF
:108C1000A11110FB01F06E4901EBC00000F562707C
:108C20009DF8A01001EB410303EB011100EBC10023
:108C30004271C7E0BDF8A400032857D1012166485E
:108C4000F53080F804179DF8B40040F2A11110FB34
:108C500001F05F4901EBC00101F562719DF8A000D0
:108C600000EB400202EB001011F830109DF8B40048
:108C700040F2A11210FB02F0554A02EBC00040790D
:108C8000814234DA00219DF8B40040F2A11210FBB9
:108C900002F04F4A02EBC000017101229DF8B400BE
:108CA00040F2A11110FB01F0494901EBC00101F5AF
:108CB00062719DF8A00000EB400303EB001001F887
:108CC00030208F229DF8B40040F2A11110FB01F07A
:108CD0003F4901EBC00000F562709DF8A01001EB68
:108CE000410303EB011100EBC10042714AE09DF822
:108CF000B40040F2A11110FB01F0354901EBC000B6
:108D000000F562709DF8A01001EB410202EB011129
:108D100000EBC1008078802834D100219DF8B40098
:108D200040F2A11210FB02F0294A02EBC0000171CF
:108D300080229DF8B40040F2A11110FB01F02449FB
:108D400001EBC00101F562719DF8A00000EB40034A
:108D500003EB001001EBC000427100229DF8B4004B
:108D600040F2A11110FB01F0194901EBC00000F520
:108D700062709DF8A01001EB410303EB011100EBC1
:108D8000C10082701EE0BDF8A400032819D10021A3
:108D90001148F53080F804178F229DF8B40040F296
:108DA000A11110FB01F00A4901EBC00000F562704F
:108DB0009DF8A01001EB410303EB011100EBC10092
:108DC000427100BF00BF05F023BA000098400020A8
:108DD00058450020D8140020C73100209DF8B40069
:108DE00000EB4001C1EBC010FE4911F8300004282F
:108DF00001D125900BE09DF8B40000EB4001C1EBE0
:108E0000C010F84911F83000152800D125909DF8C0
:108E1000B40000EB4001C1EBC010F24901EBC0000F
:108E200041789DF8B40000EB4002C2EBC010ED4A5F
:108E300012F8300041EA002041F23001884202D1AC
:108E4000A62025903DE09DF8B40000EB4001C1EB69
:108E5000C010E44901EBC00041789DF8B40000EB7C
:108E60004002C2EBC010DF4A12F8300041EA002095
:108E700041F23101884202D1A720259021E09DF8DE
:108E8000B40000EB4001C1EBC010D64911F830002E
:108E9000022816D19DF8B40000EB4001C1EBC010D0
:108EA000D04901EBC00001799DF8B40000EB40020D
:108EB000C2EBC010CB4A02EBC000C07841EA0021EF
:108EC00025919DF8B40040F2A11110FB01F0C649B4
:108ED00001EBC000C17827919DF8B40040F2A111C8
:108EE00010FB01F0C04901EBC00108319DF89C0066
:108EF000C0EBC00001EBC00082789DF8B40040F2E6
:108F0000A11110FB01F0B84901EBC00108319DF837
:108F10009C00C0EBC00001EBC000C0781044C1B29F
:108F200028910021B14A9DF8B40002EB00129DF88F
:108F30009C00115439913AE09DF8B40040F2A1111F
:108F400010FB01F0A84901EBC00108319DF89C001D
:108F5000C0EBC00001EBC00002799DF8B40040F204
:108F6000A11110FB01F0A04901EBC00108319DF8EF
:108F70009C00C0EBC00001EBC0008178BDF8E400AC
:108F8000084400EB400101EB00119DF8B40040F2F1
:108F9000A11310FB03F0944B03EBC00000F56270CB
:108FA00000F83120BDF8E400401C81B239919DF8F1
:108FB000B40040F2A11110FB01F08B4901EBC0019C
:108FC00008319DF89C00C0EBC00011F83010BDF8CE
:108FD000E4008142B0DCBDF8941043F23002881AFC
:108FE00091427DD009DC04297BD015297AD0A629AD
:108FF00010D0A72942F07D8450E1B0F5C06F72D047
:10900000A0F2016000286FD001286ED00428F1D1B1
:1090100001F0A5BF00219DF8B40040F2A11210FBA1
:1090200002F0714A02EBC00001719DF8B40040F2F9
:10903000A11110FB01F0114601EBC00008309DF8B2
:109040009C10C1EBC10100EBC1000079052824DCB4
:1090500006229DF8B40040F2A11110FB01F0624914
:1090600001EBC00108319DF89C00C0EBC00001EB92
:10907000C0000271A8229DF8B40040F2A11110FBBB
:1090800001F0594901EBC00008309DF89C10C1EB7C
:10909000C10100EBC1004271FEE09DF8B40040F256
:1090A000A11110FB01F0504901EBC00008309DF800
:1090B0009C10C1EBC10100EBC10000790A282BDC38
:1090C0000B229DF8B40040F2A11110FB01F04649BB
:1090D00001EBC00108319DF89C00C0EBC00005E029
:1090E00094E113E2FEE3FEE3FEE3FEE301EBC000E6
:1090F0000271A9229DF8B40040F2A11110FB01F009
:10910000394901EBC00008309DF89C10C1EBC1014A
:1091100000EBC1004271BFE09DF8B40040F2A11124
:1091200010FB01F0304901EBC00008309DF89C10A5
:10913000C1EBC10100EBC10000790F2824DC102233
:109140009DF8B40040F2A11110FB01F0264901EB9B
:10915000C00108319DF89C00C0EBC00001EBC000CD
:109160000271A2229DF8B40040F2A11110FB01F09F
:109170001D4901EBC00008309DF89C10C1EBC101F6
:1091800000EBC100427187E09DF8B40040F2A111EC
:1091900010FB01F0144901EBC00008309DF89C1051
:1091A000C1EBC10100EBC1004079A5282DD19DF88C
:1091B000B40040F2A11110FB01F00B4901EBC0011A
:1091C00008319DF89C00C0EBC00001EBC000C178E5
:1091D0009DF8B40000EB400202EB0010044A02EBE1
:1091E000001007E0F887002058450020883E002046
:1091F00098400020303000EB0110801C099000786E
:1092000020F00400001D099908709DF8B40040F298
:10921000A11110FB01F0FD4901EBC00008309DF8E1
:109220009C10C1EBC10100EBC1008079A12833D0B3
:109230009DF8B40040F2A11110FB01F0F34901EBDD
:10924000C00108319DF89C00C0EBC00001EBC000DC
:1092500082799DF8B40040F2A11110FB01F0EB49B6
:1092600001EBC00108319DF89C00C0EBC00001EB90
:10927000C0004271A1229DF8B40040F2A11110FB80
:1092800001F0E24901EBC00008309DF89C10C1EBF1
:10929000C10100EBC100827102F02BBB00219DF8DF
:1092A000B40040F2A11210FB02F0D84A02EBC00059
:1092B00001719DF8B40040F2A11110FB01F01146BC
:1092C00001EBC00008309DF89C10C1EBC10100EB20
:1092D000C100007908281DDC00219DF8B40040F28F
:1092E000A11210FB02F0C94A02EBC0000171082272
:1092F0009DF8B40040F2A11110FB01F0C34901EB4D
:10930000C00008309DF89C10C1EBC10100EBC1000A
:10931000027124E09DF8B40040F2A11110FB01F0AD
:10932000BA4901EBC00008309DF89C10C1EBC101A7
:1093300000EBC10000790B2811DC0C229DF8B40071
:1093400040F2A11110FB01F0B04901EBC000083060
:109350009DF89C10C1EBC10100EBC10002719DF8AA
:10936000B40040F2A11110FB01F0A84901EBC000CC
:1093700008309DF89C10C1EBC10100EBC1004079A1
:10938000A42830D19DF8B40000EB400101EB00109F
:109390009F4901EB001030309DF8A01000EB011048
:1093A000801C0990007820F0200020300999087076
:1093B00000229DF8B40040F2A11110FB01F0934986
:1093C00001EBC00000F562709DF8A01001EB4103B5
:1093D00003EB011100EBC10080F845209DF8B410AB
:1093E0000220F0F763FEA1229DF8B40040F2A11123
:1093F00010FB01F0854901EBC00008309DF89C107E
:10940000C1EBC10100EBC100427145E7002039907A
:1094100015E09DF8B40000EB4001C1EBC0107D49A0
:1094200001EBC001BDF8E400C01C095C16AABDF840
:10943000E4001154BDF8E400401C81B23991BDF83C
:10944000E4000628E5DB062116A81DF0B5FD002185
:10945000CDE93001DDE93021100A40EA0164309B9A
:10946000E21841EB2120CDE908204FF480724FF043
:109470000003DDE90801EEF7A5FE9DF8B40040F217
:10948000A11110FB01F0614901EBC00000F5627011
:109490009DF89C1001EB410303EB011100EBC100AF
:1094A000027100209DF8B41040F2A11211FB02F1EC
:1094B000564A02EBC101087104229DF8B40040F243
:1094C000A11110FB01F0514901EBC00000F56270E1
:1094D0009DF89C1001EB410303EB011100F83120D2
:1094E000A7229DF8B40040F2A11110FB01F04749FA
:1094F00001EBC00000F562709DF89C1001EB410388
:1095000003EB011100EBC1004271C5E69DF8B40008
:1095100040F2A11110FB01F03C4901EBC000083002
:109520009DF89C10C1EBC10100EBC100007904283B
:1095300072DA00219DF8B40040F2A11210FB02F093
:10954000324A02EBC0000171A1229DF8B40040F242
:10955000A11110FB01F02D4901EBC00108319DF86C
:109560009C00C0EBC00001EBC00042719DF8B4004C
:1095700040F2A11110FB01F0244901EBC0000830BA
:109580009DF89C10C1EBC10100EBC100001D0990CA
:109590000078401CC2B2099802709DF8B40040F2F5
:1095A000A11110FB01F0194901EBC00008309DF832
:1095B0009C10C1EBC10100EBC1000079042823D14C
:1095C0000A229DF8B40040F2A11110FB01F00F49EE
:1095D00001EBC00108319DF89C00C0EBC00001EB1D
:1095E000C0000271A3229DF8B40040F2A11110FB4B
:1095F00001F0064901EBC00008309DF89C10C1EB5A
:10960000C10100EBC1004271EBE205E058450020CA
:1096100098400020F88700209DF8B40040F2A11186
:1096200010FB01F0FE4901EBC00008309DF89C10D2
:10963000C1EBC10100EBC100007904282FD100214A
:109640009DF8B40040F2A11210FB02F0F44A02EBC4
:10965000C000017105229DF8B40040F2A11110FB79
:1096600001F0EF4901EBC00108319DF89C00C0EB0F
:10967000C00001EBC0000271A3229DF8B40040F2CB
:10968000A11110FB01F0E64901EBC00008309DF884
:109690009C10C1EBC10100EBC1004271A1E29DF839
:1096A000B40040F2A11110FB01F0DD4901EBC00054
:1096B00008309DF89C10C1EBC10100EBC10000799E
:1096C00008282FDC00219DF8B40040F2A11210FB05
:1096D00002F0D34A02EBC000017109229DF8B400E8
:1096E00040F2A11110FB01F0CD4901EBC00108319E
:1096F0009DF89C00C0EBC00001EBC0000271A722E6
:109700009DF8B40040F2A11110FB01F0C44901EB37
:10971000C00008309DF89C10C1EBC10100EBC100F6
:1097200042715EE29DF8B40040F2A11110FB01F01D
:10973000BB4901EBC00008309DF89C10C1EBC10192
:1097400000EBC100007909282FDC00219DF8B4004E
:1097500040F2A11210FB02F0B14A02EBC00001710D
:109760000A229DF8B40040F2A11110FB01F0AC49AF
:1097700001EBC00108319DF89C00C0EBC00001EB7B
:10978000C0000271A3229DF8B40040F2A11110FBA9
:1097900001F0A34901EBC00008309DF89C10C1EB1B
:1097A000C10100EBC10042711BE29DF8B40040F220
:1097B000A11110FB01F09A4901EBC00008309DF89F
:1097C0009C10C1EBC10100EBC10000790D282FDC1A
:1097D00000219DF8B40040F2A11210FB02F0904A63
:1097E00002EBC00001710E229DF8B40040F2A111FD
:1097F00010FB01F08A4901EBC00108319DF89C0083
:10980000C0EBC00001EBC0000271A1229DF8B400C2
:1098100040F2A11110FB01F0814901EBC0000830BA
:109820009DF89C10C1EBC10100EBC1004271D8E171
:109830009DF8B40040F2A11110FB01F0784901EB52
:10984000C00008309DF89C10C1EBC10100EBC100C5
:1098500000790E282FDC00219DF8B40040F2A112FF
:1098600010FB02F06E4A02EBC00001710F229DF85E
:10987000B40040F2A11110FB01F0694901EBC001F5
:1098800008319DF89C00C0EBC00001EBC0000271E4
:10989000A3229DF8B40040F2A11110FB01F0604931
:1098A00001EBC00008309DF89C10C1EBC10100EB3A
:1098B000C100427195E19DF8B40040F2A11110FB86
:1098C00001F0574901EBC00008309DF89C10C1EB36
:1098D000C10100EBC100007910287DDC11229DF848
:1098E000B40003E07EE1ACE1F9E1DAE140F2A1117C
:1098F00010FB01F04A4901EBC00108319DF89C00C2
:10990000C0EBC00001EBC0000271A1229DF8B400C1
:1099100040F2A11110FB01F0414901EBC0010831F7
:109920009DF89C00C0EBC00001EBC00042719DF8A7
:10993000B40040F2A11110FB01F0394901EBC00164
:1099400008319DF89C00C0EBC00001EBC0008271A3
:109950000021399156E09DF8B40040F2A11110FBAE
:1099600001F02F4901EBC00108319DF89C00C0EBCC
:10997000C00001EBC0008178BDF8E40001449DF80F
:10998000B40000EB400202EB0010264A02EB00108C
:10999000303000EB0110801C0990007820F080012D
:1099A0008031099801709DF8B40040F2A11110FBBC
:1099B00001F01B4901EBC00108319DF89C00C0EB90
:1099C000C00001EBC0008178BDF8E40001449DF8BF
:1099D000B40000EB400200E085E002EB0010114A09
:1099E00002EB0010303000EB0110801C0990007871
:1099F00020F00400001D09990870BDF8E400401C27
:109A000080B239909DF8B40040F2A11110FB01F032
:109A1000034901EBC00108319DF89C0004E00000FF
:109A20005845002098400020C0EBC00011F83010CD
:109A3000BDF8E40081428EDC9DF8B40000EB4001EB
:109A400001EB0010FE4901EB001030309DF8A01032
:109A500000EB01108078C0F34010E8B39DF8B4002B
:109A600000EB400101EB0010F54901EB0010303034
:109A70009DF8A01000EB0110801C0990007820F0E8
:109A80002002099802709DF8B40000EB400101EB40
:109A90000010EB4901EB001030309DF8A01000EBF6
:109AA00001108078C0F34000A8B99DF8B40000EB25
:109AB000400101EB0010E24901EB001030309DF84D
:109AC000A01000EB0110801C0990007820F0080025
:109AD00008300999087000E065E09DF8B410022094
:109AE000F0F7E4FA7DE09DF8B40040F2A11110FB1C
:109AF00001F0D44901EBC00108319DF89C00C0EB96
:109B0000C00001EBC00001799DF8B40040F2A11241
:109B100010FB02F0CB4A02EBC0004079814260D1D9
:109B20009DF8B40040F2A11110FB01F0114601EBC9
:109B3000C00008309DF89C10C1EBC10100EBC100D2
:109B40008079A12830D0A3229DF8B40040F2A11161
:109B500010FB01F0BB4901EBC00108319DF89C00EE
:109B6000C0EBC00001EBC00042719DF8B40040F2B0
:109B7000A11110FB01F0B34901EBC00008309DF8C2
:109B80009C10C1EBC10100EBC1008079A22828D054
:109B900000219DF8B40040F2A11210FB02F0A94A86
:109BA00002EBC00001711CE0A1229DF8B40040F25C
:109BB000A11110FB01F0A34901EBC00108319DF890
:109BC0009C00C0EBC00001EBC000427101219DF878
:109BD000B40040F2A11210FB02F09A4A02EBC0005E
:109BE000017112E4A1229DF8B40040F2A11110FB12
:109BF00001F0944901EBC00108319DF89C00C0EBD5
